:100000000C947A0D0C94A7620C94AB0D0C94AB0D70
:100010000C94AB0D0C9497510C94E45F0C94AB0DC5
:100020000C94AB0D0C94AB0D0C94AB0D0C94AB0D70
:100030000C94AB0D0C94AB0D0C94AB0D0C94AB0D60
:100040000C94AB0D0C943D820C941B510C94AB0D95
:100050000C94AB0D0C94AB0D0C94AB0D0C9462890D
:100060000C94AB0D0C94E8570C94BF570C94AB0D4B
:100070000C94AB0D0C94AB0D0C94AB0D0C94AB0D20
:100080000C94513C0C94AB0D0C94AB0D0C94AB0D3B
:100090000C9496570C946D570C94AB0D0C94AB0DBF
:1000A0000C94AB0D0C94AB0D0C94AB0D0C94AB0DF0
:1000B0000C94AB0D0C941E420C94AB0D0C94AB0D38
:1000C0000C94AB0D0C94AB0D0C94AB0D0C944457ED
:1000D0000C941B570C94AB0D0C94F2560C94C9560F
:1000E0000C94AB0D89188C189318961899189C18B5
:1000F000A318AA18AD18B418BB18C218841EB21ED3
:10010000E91E201FFB1F322060208E205421542125
:100110005421542154215421542154215421542137
:100120005421542154215421542154215421542127
:100130005421542154215421542154215421542117
:10014000542154215421571F8F1FC61FBC20F42057
:100150002B21522358235E2364236A2370237623A2
:100160007C23822388238E239423A623AC23B223CB
:10017000CA23D023D623DC23E223E823EE23F4236F
:10018000FA23002406240C241224182424243024C6
:1001900036243C2442245A24602466246C2472248D
:1001A000782468256E25742586258C259225A4251E
:1001B000AA25B025B625BC25C225DA25E0250A26C4
:1001C000102616261C2634263A2640264626DB26EE
:1001D000DB26DB26DB26DB26DB26DB26DB265C2696
:1001E000602664266A266E26722676267A267E2663
:1001F00082268826A626AC26B22648247E2484247D
:100200008A24902496249C24222628262E264C26B6
:1002100052265826B826BE26C426C825CE25A22496
:10022000A824AE24B424BA24C0247A2598252A24EC
:100230009A23A0234E245424CA26D026D6261E2430
:10024000E625EC25F225F825FE250426C624CC2437
:10025000D224D824DE24E424EA24F024F624FC2446
:10026000022508250E2514251A25202526252C25AE
:1002700038253E2544254A25502556255C256225EE
:100280009A2694268E26A02680259E25B823BE2356
:10029000C423D4253225A22D7F2D582DBF2D162EF7
:1002A000DE2D0D2EFC2DC72EAA2E832E172FE42E09
:1002B000E42E062FEF2E9B349B34B5349B34C2348E
:1002C000DB34F63411354B4254425C427042824278
:1002D00094429F42BB45EF45244644467946E14659
:1002E000F146194865476E47A247D747E447194882
:1002F000AD468A4CA14CB84CCF4CE64C144D2B4D1E
:10030000424D594D784D904DA74DC64DDC4DFD4C9D
:10031000C253C553B453B853BE53FC53C953CD5302
:10032000D353D753DB53E153E553E953FC53EF5316
:10033000F353F753525957595C5966597059E95953
:100340007A5982598A5994599E59A859B759C1590D
:10035000E959CB59D559DF5905A84CCDB2D44EB97E
:100360003836A9020C50B9918688083CA6AAAA2A58
:10037000BE000000803F3400330032004E6F6E65D7
:100380000053746F70706564004E65757472616CB3
:10039000205475726E004D6F76696E6720526576D7
:1003A00065727365004D6F76696E6720466F727770
:1003B000617264004272616B696E670054414E4B1A
:1003C00020524553544F5245440025004865616C06
:1003D0007468204C6576656C3A2000564548494360
:1003E0004C452052455041495220434F4D504C45B9
:1003F00054450054414E4B2044455354524F5945A7
:10040000440025004865616C7468204C6576656C15
:100410003A2000290056454849434C452052455052
:1004200041495220535441525445442028005245DA
:1004300050414952204F5045524154494F4E20435C
:10044000414E43454C4C45440029004D41434849E9
:100450004E452047554E20484954212028005245FA
:1004600050414952204F5045524154494F4E20432C
:10047000414E43454C4C454400290043414E4E4FAC
:100480004E2048495421202800547572726574200A
:10049000726F746174696F6E206973206E6F74205F
:1004A0006F66207479706520536572766F2E204ECA
:1004B0006F20736574757020617661696C61626C20
:1004C000652E004E6F207374656572696E672073C8
:1004D0006572766F2061737369676E65642C207234
:1004E000652D636865636B2076656869636C65205C
:1004F000747970652E0054757272657420656C6530
:10050000766174696F6E206973206E6F74206F66F8
:10051000207479706520536572766F2E204E6F209F
:10052000736574757020617661696C61626C652EAB
:1005300000546F70204C65667400546F70204365E2
:100540006E74657200546F70205269676874004D54
:100550006964646C65204C656674004D6964646C04
:10056000652043656E746572004D6964646C652036
:10057000526967687400426F74746F6D204C6566D1
:100580007400426F74746F6D2043656E7465720001
:10059000426F74746F6D20526967687400464952E7
:1005A0004D574152452056455253494F4E3A20002F
:1005B0006942757300534275730050504D004E6F81
:1005C0006E6520446574656374656400417A696D85
:1005D0007574682020202000456C65766174696F11
:1005E0006E2020005475726E2020202020202000D4
:1005F0005468726F74746C652020200053746963B2
:100600006B202020202020204D696E2020202043B8
:10061000656E7465722020204D6178202020204472
:1006200065616462616E64202052657665727365EF
:100630006400524144494F20494E464F202D20002E
:100640004E4F542044455445435445440049474E79
:100650004F52454400416E616C6F670044696769A1
:1006600074616C00417578204368616E2E202020F3
:100670004D696E20202020204D61782020202020F0
:1006800054797065004368616E6E656C7320757493
:10069000696C697A65643A20004368616E6E656CC6
:1006A000732064657465637465643A20002028448F
:1006B000697361626C656429002028456E61626C13
:1006C000656429004D656368616E6963616C2072C1
:1006D00065636F696C00416972736F6674004D6584
:1006E0006368616E6963616C2042617272656C3A25
:1006F000200020284D31290020284D3229002028B3
:1007000042290042617272656C20456C65766174A5
:10071000696F6E3A20200020284D30290020284D96
:1007200031290020284129005475727265742052C5
:100730006F746174696F6E3A2020200020416D70E3
:10074000732900202843757272656E74204C696DA0
:1007500069743A20004472697665204D6F746F7237
:10076000733A202020202020004D4F544F52205417
:10077000595045530054616E6B202854616D69795E
:100780006120444D44290054616E6B2028444B4C39
:100790004D2047656172626F78290043617200489D
:1007A000616C66747261636B0054616E6B00554ED0
:1007B0004B4E4F574E00596573004E6F0029002570
:1007C0002C20446563656C65726174696F6E206688
:1007D0006163746F72200020284B69636B626163F0
:1007E0006B2073706565642000547261636B2052E6
:1007F00065636F696C20456E61626C65643A2020A8
:1008000020004E2F4120666F722076656869636C08
:10081000652074797065005475726E204D6F646543
:100820003A202020202020202020202020202000CE
:100830004E2F4120666F722076656869636C652073
:100840007479706500596573202854616D69796108
:1008500029002500202D20004E65757472616C20E2
:100860005475726E20416C6C6F7765643A2020205D
:100870000020736563005472616E736D69737369F0
:100880006F6E2044656C61793A2020202020002082
:1008900073656300456E67696E65205061757365A9
:1008A0002054696D653A20202020202000207365A7
:1008B000630053686966742054696D653A2020208E
:1008C00020202020202020202020004175746F6DE2
:1008D00061746963004D616E75616C005472616E84
:1008E000736D697373696F6E20547970653A202057
:1008F00020202020002500596573202D20005265FE
:100900007665727365205370656564204C696D6906
:100910007465643A2020002500596573202D20005D
:10092000466F7277617264205370656564204C690C
:100930006D697465643A202000206D7329002520BC
:100940007468726F74746C6520666F722000202862
:10095000004D6F746F72204E7564676520456E613F
:10096000626C65643A202020200029004E6F6E657D
:10097000004E6F6E65002C205072657365743A20CE
:10098000002900202841646A757374656420746FBF
:10099000200020284C6576656C3A2000446563652C
:1009A0006C2052616D7020456E61626C65643A2006
:1009B000202020200029004E6F6E65004E6F6E656E
:1009C000002C205072657365743A2000290020289D
:1009D00041646A757374656420746F200020284C2C
:1009E0006576656C3A2000416363656C2052616DE9
:1009F0007020456E61626C65643A202020202000E2
:100A00004163746976652044726976696E67205027
:100A1000726F66696C653A200056656869636C653B
:100A200020547970653A202020202020202020208A
:100A3000200044524956452053455454494E47538B
:100A40000020736563005265636F696C2064656C98
:100A500061793A20202020202020202020202020E2
:100A6000202020202020002500596573202D200003
:100A700042617272656C20456C65766174696F6E57
:100A8000205370656564204C696D697465643A2013
:100A9000002500596573202D20005475727265740D
:100AA00020526F746174696F6E20537065656420A5
:100AB0004C696D697465643A202000545552524562
:100AC000542053455454494E475300556E6B6E6F36
:100AD000776E004865617679004D656469756D00D3
:100AE0004C6967687400437573746F6D00556E6B65
:100AF0006E6F776E004E6F6E65004F70656E2050A2
:100B0000616E7A65720054616D6979612053706518
:100B1000630020736563207265636F76657279295F
:100B200000207365632072656C6F61642C20002067
:100B30004D4720686974732C20002063616E6E6FCE
:100B40006E20686974732C200028005765696768F7
:100B50007420436C6173733A20202020200044618C
:100B60006D6167652050726F66696C653A20202060
:100B700000596573202800416363657074204D47F8
:100B80002044616D6167653A200059657320280033
:100B900053656E64204D4720495220436F64653A87
:100BA0002020004E2F4100526570616972656420FB
:100BB00062793A202020202020004E2F41004869F1
:100BC000742050726F746F636F6C20323A20202053
:100BD00000290020285465616D2000466972652057
:100BE00050726F746F636F6C3A202020200046694A
:100BF00072652050726F746F636F6C3A20202020F2
:100C0000004973205265706169722054616E6B3FB8
:100C100020202000495220262054616E6B20426122
:100C200074746C696E672044697361626C656400FA
:100C3000424154544C4520494E464F00554E4B4E70
:100C40004F574E0042656E6564696E692054425389
:100C5000204D6963726F0042656965722055534D7E
:100C60002D52432D320054616967656E20536F75B4
:100C70006E642043617264004F70656E2050616E37
:100C80007A657220536F756E64204361726400420E
:100C9000656E6564696E6920544253204D696E69C2
:100CA00000536F756E6420636172643A2000534F85
:100CB000554E44204341524400556E6B6E6F776E23
:100CC0000042617272656C20456C65766174696F73
:100CD0006E20436F6D6D616E640054757272657441
:100CE00020526F746174696F6E20436F6D6D616E19
:100CF00064005374656572696E6720436F6D6D6142
:100D00006E640056656869636C6520537065656440
:100D100000456E67696E65205370656564005468B0
:100D2000726F74746C6520436F6D6D616E640053F7
:100D300070656564206465637265617365732062C4
:100D4000656C6F772000537065656420696E63720F
:100D500065617365732061626F76652000547572FA
:100D60006E2053746F70706564004C656674205417
:100D700075726E205374617274656400526967689D
:100D800074205475726E20537461727465640056D9
:100D9000656869636C652053746F70706564004D9D
:100DA0006F76696E672052657665727365004D6F68
:100DB00076696E6720466F727761726400456E6770
:100DC000696E652053746F7000456E67696E6520AB
:100DD00053746172740043616E6E6F6E2052656C65
:100DE0006F616465640056656869636C652044657D
:100DF0007374726F7965640043616E6E6F6E204824
:100E00006974004272616B6573204170706C696532
:100E100064005661726961626C6500290020286F68
:100E2000662000506F732000417578204368616E22
:100E30006E656C20005661726961626C65004F6E70
:100E4000004F6666004200410045787465726E612D
:100E50006C20496E7075742000070809090B0C0C92
:100E60000B0C0C54757272657420537469636B209B
:100E70002D200046756E6374696F6E202300202D4F
:100E80003E20002073656300547572726574206D96
:100E90006F76656D656E742064656C61793A2020AB
:100EA000004E6F6E650059657300547572726574FB
:100EB00020737469636B2066756E6374696F6E73FB
:100EC0003A200046554E4354494F4E20545249470C
:100ED000474552530076206375746F66662900207B
:100EE00028004C564320456E61626C65643A2020B0
:100EF00020202020007600566F6C746167653A20D0
:100F000020202020202020202000596573004E6FD3
:100F10000042617474657279204465746563746518
:100F2000643A200042415454455259005365726955
:100F3000616C203320547820426175643A2020008F
:100F40004175782053657269616C20426175643A1D
:100F5000202020004D6F746F722053657269616CA0
:100F600020426175643A20005553422053657269EE
:100F7000616C20426175643A202020004241554452
:100F800020524154455300212000464143544F52C2
:100F90005920524553455421200054616967656EBC
:100FA0002056322F563300536F6E7900524354410E
:100FB000204D616368696E652047756E00436C6102
:100FC000726B204D616368696E652047756E0052D3
:100FD0004354412052657061697200494255205264
:100FE000657061697200436C61726B20526570615B
:100FF0006972004F70656E50616E7A65720056734B
:1010000054616E6B00464F560054616967656E20EF
:1010100056310048656E67204C6F6E670054616DF5
:1010200069796120312F33350054616D6979612010
:10103000322D53686F740054616D69796100556E8B
:101040006B6E6F776E003A20004269742000476132
:10105000703A2000401F7017D007A00FA00FDC05CA
:10106000D007C40910278813983A102758026C0239
:1010700058026C0258026C0258026C0258026C0250
:1010800058026C0258026C0258026C025802B036C8
:101090006C023A026C023A026C023A026C02B036FE
:1010A000384A5C121C255C125C121C255C12BC7F49
:1010B000C7F2C07887A5B7C5A00F8813B80B401F2B
:1010C000B80BB80B7017401F556E6B6E6F776E00C4
:1010D00044657461636865642F4E41005265636FB7
:1010E000696C20536572766F0050616E2053657293
:1010F000766F00536572766F2F455343004F6E62D3
:101100006F617264204D6F746F72204472697665EE
:1011100072004F70656E2050616E7A657220536365
:101120006F75742053657269616C20455343005399
:1011300061626572746F6F74682053657269616C67
:1011400000506F6C6F6C752053657269616C005351
:101150006572766F203100536572766F20320053CE
:101160006572766F203300536572766F20340053BA
:101170006572766F203500536572766F20360053A6
:101180006572766F203700536572766F20380000E5
:10119000002100240027002A002D00300033000128
:1011A000010000040107010A0100002200250028B7
:1011B000002B002E00310034000201000005010860
:1011C000010B01000020002300260029002C002F25
:1011D00000320000010000030106010901050505B8
:1011E00005070508080808020202020A0A0808049E
:1011F00004040401010101010101010303030303CC
:10120000030303040707070C0C0C0C0C0C0C0C025A
:1012100002020206060606060606060B0B0B0B0B61
:101220000B0B0B010210202008081020401020405A
:10123000800201020108040201010204081020409A
:1012400080804020100804020180040201804020B8
:1012500010080402010804020101020408102040E1
:1012600080010204081020408000000A0B02090CD3
:101270000D0E08070304010000000000000000003C
:10128000000000000000000000000000000000005E
:10129000000000000012111000000000000000001B
:1012A00000000000000000000000000000000044FA
:1012B000726976696E672050726F66696C6520731B
:1012C000657420746F2023002500537065656420C9
:1012D0007265647563656420746F20005370656582
:1012E0006420726573746F726564005475726E2049
:1012F000456E67696E65204F6E004D616E75616C5D
:10130000207472616E736D697373696F6E202D2026
:1013100070757420696E206E65757472616C2067DB
:10132000656172206265666F7265207374617274A4
:10133000696E6720656E67696E6521005475726E0F
:1013400020456E67696E65204F666600456E676969
:101350006E65204175746F2053687574646F776E85
:1013600000456E67616765205472616E736D6973C5
:1013700073696F6E00446973656E676167652054B9
:1013800072616E736D697373696F6E00536574205B
:101390005475726E204D6F64653A20310053657448
:1013A000205475726E204D6F64653A20320053658B
:1013B00074205475726E204D6F64653A2033004579
:1013C0006E61626C65204E65757472616C20547537
:1013D000726E730044697361626C65204E6575744A
:1013E00072616C205475726E7300494F20506F7299
:1013F000742041204F7574707574202D204F6E003D
:10140000494F20506F72742041204F75747075746D
:10141000202D204F666600494F20506F7274204285
:10142000204F7574707574202D204F6E00494F2029
:10143000506F72742042204F7574707574202D2087
:101440004F6666004C56432045786974202D20561F
:101450006F6C7461676520526573746F72656400A8
:101460007629004C5643207468726573686F6C640B
:101470002072656163686564212028005265766585
:10148000727365643A2020004D61782050756C734A
:10149000653A20004D696E2050756C73653A2000E6
:1014A000456E642056616C75657300456E6420520C
:1014B00065636F696C20536572766F205365747530
:1014C0007000456E6420526F746174696F6E2053B2
:1014D0006572766F20536574757000456E642045A3
:1014E0006C65766174696F6E20536572766F2053F8
:1014F0006574757000536572766F20756E2D726518
:1015000076657273656400536572766F20726576D6
:1015100065727365640052657665727365643A201E
:1015200020004D61782050756C73653A20004D693C
:101530006E2050756C73653A20005374617274208C
:1015400056616C75657300494E56414C49442053B1
:101550004552564F2E204E4F2053455455502E0085
:101560005365747570205265636F696C20536572A2
:10157000766F0053657475702054757272657420AF
:10158000526F746174696F6E2050616E2053657282
:10159000766F005365747570205374656572696E5B
:1015A0006720536572766F20284F757470757420AC
:1015B0003229005365747570205374656572696EC5
:1015C0006720536572766F20284F7574707574208C
:1015D00034290053657475702054757272657420D7
:1015E000456C65766174696F6E20536572766F0025
:1015F000466F72776172642047656172004E65754F
:101600007472616C20476561720052657665727311
:101610006520476561720053657420416363656CA2
:101620002052616D70204C6576656C3A20005365E0
:101630007420446563656C2052616D70204C657642
:10164000656C3A2000416E616C6F6720557365725E
:101650002046756E6374696F6E2031202D20004125
:101660006E616C6F6720557365722046756E63748A
:10167000696F6E2032202D20002D00202D200020AB
:1016800000545255450046414C53450025005761D2
:101690006974696E6720666F7220726164696F2E6B
:1016A0002E2E20004952204E4F5420656E61626CF0
:1016B0006564202D206E6F2049522070726F746F08
:1016C000636F6C732073656C65637465642E00557D
:1016D0006E61626C6520746F20656E61626C65205E
:1016E000495200495220656E61626C65640049523E
:1016F0002064697361626C656400417578204F7580
:101700007470757420466C61736865640041757807
:10171000204F757470757420496E766572736520FC
:10172000466C61736865640053746F70204175780E
:10173000204F757470757420426C696E6B696E67AA
:101740000053746F70205265766F6C76696E6720F7
:10175000417578204C696768740053746F7020413C
:101760006C6C205573657220536F756E64730049FD
:101770004F20506F72742041202D2050756C73657E
:101780006400494F20506F72742041202D20537403
:1017900061727420426C696E6B696E6700494F20FC
:1017A000506F72742042202D2050756C7365640058
:1017B000494F20506F72742042202D205374617263
:1017C0007420426C696E6B696E6700557365722098
:1017D00046756E6374696F6E2031005573657220B3
:1017E00046756E6374696F6E2032004C6967687469
:1017F0002031204F6E004C696768742031204F669D
:1018000066004C696768742032204F6E004C69672F
:1018100068742032204F666600326E64204D472087
:1018200053746F7000326E64204D472053746172A0
:10183000740052756E6E696E67204C6967687473C8
:10184000204F6E0052756E6E696E67204C69676836
:101850007473204F666600417578204F75747075FB
:1018600074204F6E00417578204F75747075742028
:101870004F66660053746F70205265766F6C7669A0
:101880006E6720417578204C696768740053746FE7
:101890007020417578204F757470757420426C69A2
:1018A0006E6B696E6700417578204F757470757442
:1018B000205072657365742044696D0053746172C1
:1018C0007420417578204F757470757420426C696E
:1018D0006E6B696E670053657420766F6C756D650D
:1018E0003A2000202D205374617274205265706577
:1018F0006174696E6700202D2053746F70005573FA
:10190000657220536F756E64200041202D200042C7
:10191000202D2000536F756E642042616E6B200095
:10192000506C61792F53746F7000506C6179205244
:10193000616E646F6D00506C6179205072657669DC
:101940006F757300506C6179204E657874002028A3
:10195000776974682049522900466972652043619D
:101960006E6E6F6E004669726520526570616972B5
:10197000205369676E616C00416972736F667420F1
:101980002D204D616E75616C2054726967676572B8
:10199000004D656368616E6963616C205265636FB9
:1019A000696C202D204D616E75616C2054726967E1
:1019B00067657200536572766F205265636F696C5C
:1019C000202D204D616E75616C20547269676765CA
:1019D00072004869676820496E74656E736974792E
:1019E00020466C61736820556E6974202D204D610E
:1019F0006E75616C2054726967676572004D47208F
:101A00005374617274004D472053746F70004169C4
:101A100072736F6674202D20456E61626C65640080
:101A20004D656368616E6963616C205265636F69BF
:101A30006C202D20456E61626C6564004169727393
:101A40006F6674202D2044697361626C6564004D7B
:101A5000656368616E6963616C205265636F696C70
:101A6000202D2044697361626C656400436F6D6D65
:101A700073206368616E67656420746F20555342FC
:101A800000436F6D6D73206368616E6765642074D9
:101A90006F2053657269616C203100536D6F6B6507
:101AA0007220656E61626C656400536D6F6B657268
:101AB0002064697361626C656400537461727420A0
:101AC0005265766F6C76696E6720417578204C6937
:101AD00067687400524144494F204641494C534184
:101AE000464500526164696F205265616479202D1A
:101AF000200012AB11241FBECFEFD1E2DEBFCDBF5D
:101B000000E00CBF16E0A0E0B2E0E9EFFBE901E085
:101B10000BBF02C007900D92A233B107D9F723E1A2
:101B2000A2E3B6E001C01D92A43CB207E1F71DE0BC
:101B3000CAE7DDE000E006C021970109802FFE0121
:101B40000E9485BAC937D10780E00807A9F70E942B
:101B5000FB980C94D8BC0C9400002F923F924F92AB
:101B60005F926F927F928F929F92AF92BF92CF922D
:101B7000DF92EF92FF920F931F93CF93DF93CDB736
:101B8000DEB7E6970FB6F894DEBF0FBECDBF8091EB
:101B9000D4069091D5060E94A6560E94C1756DE9A3
:101BA00075E08091D4069091D5060E9448556CEF5F
:101BB00075E0CE0101960E9409558091D40690915E
:101BC000D506DC01ED91FC914D815E8169817A81C0
:101BD0000280F381E02D199564E076E08091D406CF
:101BE0009091D5060E946C552AE047ED51E060E0E7
:101BF00070E08091D4069091D5060E94815564E1F1
:101C000076E08091D4069091D5060E94A956CE0127
:101C100001960E94D9540E9492968091D406909188
:101C2000D506DC01ED91FC910680F781E02D199538
:101C30008091D4069091D5060E94A6560E94C17547
:101C400062E376E08091D4069091D5060E944855D3
:101C5000E091160BE4300CF0E0E08EEB95E09A8317
:101C600089838AEB95E09C838B8385EB95E09E834B
:101C70008D8380EB95E098878F83EE0FFF0B81E0DB
:101C800090E08C0F9D1FE80FF91F6081718180919A
:101C9000D4069091D5060E94B9560E94C1756CEF8A
:101CA00075E08091D4069091D5060E94B9560E94A5
:101CB000C17560EF75E08091D4069091D5060E94C1
:101CC0004855E091F810F091F91081819281883E99
:101CD000934014F40E94B175E091F810F091F9105E
:101CE000618172818091D4069091D5060E946C49E1
:101CF00084E00E943A98E091F810F091F910658123
:101D000076818091D4069091D5060E946C4985E039
:101D10000E943A98E091F810F091F9106381748173
:101D20008091D4069091D5060E946C4984E00E946F
:101D30003A98E091F810F091F91067818091D406FB
:101D40009091D5060E943F4888E00E943A98E09121
:101D5000F810F091F91080850E949D7564EE75E091
:101D60008091D4069091D5060E944855E0910211C9
:101D7000F091031181819281883E934014F40E9476
:101D8000B175E0910211F09103116181728180912E
:101D9000D4069091D5060E946C4984E00E943A983E
:101DA000E0910211F0910311658176818091D40652
:101DB0009091D5060E946C4985E00E943A98E09186
:101DC0000211F0910311638174818091D406909186
:101DD000D5060E946C4984E00E943A98E091021175
:101DE000F091031167818091D4069091D5060E94ED
:101DF0003F4888E00E943A98E0910211F091031167
:101E000080850E949D7568ED75E08091D406909163
:101E1000D5060E944855E0910C11F0910D11818179
:101E20009281883E934014F40E94B175E0910C11A8
:101E3000F0910D11618172818091D4069091D50647
:101E40000E946C4984E00E943A98E0910C11F09154
:101E50000D11658176818091D4069091D5060E94FE
:101E60006C4985E00E943A98E0910C11F0910D11B7
:101E7000638174818091D4069091D5060E946C494B
:101E800084E00E943A98E0910C11F0910D11678165
:101E90008091D4069091D5060E943F4888E00E9428
:101EA0003A98E0910C11F0910D1180850E949D757A
:101EB0006CEC75E08091D4069091D5060E9448554F
:101EC000E0911611F091171181819281883E934023
:101ED00014F40E94B175E0911611F091171161810F
:101EE00072818091D4069091D5060E946C4984E05D
:101EF0000E943A98E0911611F09117116581768150
:101F00008091D4069091D5060E946C4985E00E948C
:101F10003A98E0911611F0911711638174818091C4
:101F2000D4069091D5060E946C4984E00E943A98AC
:101F3000E0911611F091171167818091D40690916C
:101F4000D5060E943F4888E00E943A98E091161119
:101F5000F091171180850E949D758091D406909113
:101F6000D5060E94A6560E943385C82E64E676E008
:101F70008091D4069091D5060E94B9560E94C175F1
:101F800007E910E1E12CF12CD12C57012FEFA21A17
:101F9000B20AB5018091D4069091D5060E946C4991
:101FA00049E0E416F10410F48BE001C08AE00E94DD
:101FB0003A98D8012C918091D4069091D50622238D
:101FC000C9F11596ED91FC911697618172810E947D
:101FD0006C49D8011596ED91FC91169781819281FB
:101FE000883E934014F40E94B17584E00E943A98B0
:101FF000D8011596ED91FC911697638174818091BB
:10200000D4069091D5060E946C4984E00E943A98CB
:10201000D8011596ED91FC91169727818091D406F1
:102020009091D506222319F06CE576E00BC065E5AA
:1020300076E008C0EC14FD041CF46DE476E002C008
:1020400060E476E00E94B956095F1F4F7501BCE05D
:10205000AB16B10409F099CF0E94C17569E976E029
:102060008091D4069091D5060E9448550E943385F0
:10207000682F8091D4069091D5060E94284865E883
:1020800076E08091D4069091D5060E9448556091E3
:10209000130B7091140B8091D4069091D5060E9479
:1020A000A2490E9492968091D4069091D506DC01B7
:1020B000ED91FC910680F781E02D19958091D40671
:1020C0009091D5060E94A6560E94C17569E677E0F8
:1020D0008091D4069091D5060E94B9560E94C17590
:1020E00065E577E08091D4069091D5060E94485529
:1020F00080913D0F0E94584EBC018091D406909172
:10210000D5060E94485580913D0F8A30C1F463E4A2
:1021100077E08091D4069091D5060E944855609151
:10212000F10F8091D4069091D5060E943F486CE350
:1021300077E08091D4069091D5060E944855809111
:10214000D4069091D5060E94A65668E277E0809169
:10215000D4069091D5060E94485580913E0F0E946A
:10216000584EBC018091D4069091D5060E944855E6
:1021700020913E0F8091D4069091D5062B303CF4EF
:10218000293054F4283069F467E177E007C02B3038
:1021900041F463E277E002C06DE177E00E94B95656
:1021A00002C00E94A65663E077E08091D406909129
:1021B000D5060E94485580913F0F0E94584EBC01A1
:1021C0008091D4069091D5060E94485520913F0FEA
:1021D0008091D4069091D5062B303CF4293054F4EC
:1021E000283069F462EF76E007C02B3041F46EEFDF
:1021F00076E002C068EF76E00E94B95602C00E9405
:10220000A6566EED76E08091D4069091D5060E9498
:1022100048552091510F8091D4069091D5062223E4
:1022200019F066ED76E002C064EC76E00E94485555
:10223000209156128091D4069091D506222319F050
:1022400069EB76E002C06DEA76E00E944855809125
:10225000D4069091D5060E94A6560E94929680912F
:10226000D4069091D506DC01ED91FC910680F781B2
:10227000E02D199580910002823011F00C94C01964
:10228000F0906E0F0091710F10E08091D406909144
:10229000D5060E94A6560E94C17562E37AE080913D
:1022A000D4069091D5060E94B9560E94C17569E185
:1022B0007AE08091D4069091D5060E944855E0912D
:1022C0007E0FE6300CF0E0E08EEA97E09A83898397
:1022D00089EA97E09C838B838FE997E09E838D83C7
:1022E0008BE997E098878F8387E897E09A878987BB
:1022F00085E797E09C878B87EE0FFF0B81E090E0EE
:102300008C0F9D1FE80FF91F608171818091D406A9
:102310009091D5060E94B95660E07AE08091D4068B
:102320009091D5060E944855609100028091D40694
:102330009091D5060E94284867EE79E08091D406F6
:102340009091D5060E9448558F2D0E948875FF20D8
:1023500009F44AC06DED79E08091D4069091D506DC
:102360000E9448558091D4069091D506112339F0EA
:102370006091690F0E943F489091690F06C060917B
:102380006F0F0E943F4890916F0F80919A1398139E
:10239000FEC761EC79E08091D4069091D5060E9449
:1023A00048558091D4069091D506112339F060915B
:1023B0006A0F61110CC06CEB79E006C06091700F80
:1023C000611105C067EB79E00E94485505C0062EF3
:1023D000000C770B0E946C4965EB79E08091D40684
:1023E0009091D5060E9448558091D4069091D506CB
:1023F0000E94A6566CE979E08091D4069091D506AA
:102400000E944855802F0E948875002309F44AC015
:1024100062E979E08091D4069091D5060E944855F2
:102420008091D4069091D506112339F060916C0FFC
:102430000E943F4890916C0F06C06091720F0E94FD
:102440003F489091720F80919C139813BAC766E72A
:1024500079E08091D4069091D5060E9448558091EC
:10246000D4069091D506112339F060916D0F61115A
:102470000CC061E779E006C06091730F611105C07F
:102480006CE679E00E94485505C0062E000C770BDB
:102490000E946C496AE679E08091D4069091D50655
:1024A0000E9448558091D4069091D5060E94A65668
:1024B00061E579E08091D4069091D5060E94485557
:1024C0008091870F811103C00E94967535C066EB1D
:1024D00077E08091D4069091D5060E9448556EE42D
:1024E00079E08091D4069091D5060E94485560917C
:1024F000870F8091D4069091D5060E943F486EE3E5
:1025000079E08091D4069091D5060E94485540917B
:10251000880F5091890F60E070E02AE08091D40626
:102520009091D5060E94815569E379E08091D406A7
:102530009091D5060E94B95660E279E08091D40668
:102540009091D5060E94485580917F0F8436C8F43B
:1025500069E179E08091D4069091D5060E944855B2
:1025600060917F0F8091D4069091D5060E943F48DC
:1025700067E179E08091D4069091D5060E94B95622
:1025800003C080E00E9496756EEF78E08091D406DB
:102590009091D5060E9448558091800F8436C8F4EA
:1025A00067EF78E08091D4069091D5060E94485557
:1025B0006091800F8091D4069091D5060E943F488B
:1025C00065EF78E08091D4069091D5060E94B956C7
:1025D00003C080E00E9496756CED78E08091D4068F
:1025E0009091D5060E9448552091CD068091D40641
:1025F0009091D506222319F065ED78E002C06BECCE
:1026000078E00E94B95662EB78E08091D406909110
:10261000D5060E9448556091750F7091760F072E70
:10262000000C880B990B0E9426B720E030E04AE7A7
:1026300054E40E942BB9AB01BC0121E08091D40687
:102640009091D5060E94C9556DEA78E08091D40634
:102650009091D5060E94B95664E978E08091D4063D
:102660009091D5060E9448556091770F7091780F30
:10267000072E000C880B990B0E9426B720E030E053
:102680004AE754E40E942BB9AB01BC0121E08091E0
:10269000D4069091D5060E94C9556FE878E08091E4
:1026A000D4069091D5060E94B95666E778E08091ED
:1026B000D4069091D5060E9448556091790F70918B
:1026C0007A0F072E000C880B990B0E9426B720E08A
:1026D00030E04AE754E40E942BB9AB01BC0121E091
:1026E0008091D4069091D5060E94C95561E778E0A3
:1026F0008091D4069091D5060E94B95668E578E09D
:102700008091D4069091D5060E94485590917E0FF5
:10271000913011F09430F9F480917B0F0E9488750C
:1027200080917B0F882329F164E578E08091D406BD
:102730009091D5060E94485560917C0F8091D406F7
:102740009091D5060E943F4862E578E08091D406DA
:102750009091D5060CC02091D4063091D5069530C5
:1027600019F465E478E002C060E378E0C9010E94F2
:1027700048558091D4069091D5060E94A65667E1EF
:1027800078E08091D4069091D5060E9448559091AA
:102790007E0F2FEF290F8091D4069091D50622301D
:1027A00028F4609132060E94284804C062E078E074
:1027B0000E94B95669EE77E08091D4069091D506D3
:1027C0000E94485580918B0F0E94887580918B0FD5
:1027D000882341F167ED77E08091D4069091D5068A
:1027E0000E94485560918C0F8091D4069091D50637
:1027F0000E943F486FEB77E08091D4069091D50618
:102800000E94485560918D0F8091D4069091D50615
:102810000E943F486DEB77E08091D4069091D506F9
:102820000E9448558091D4069091D5060E94A656E4
:102830000E9492968091D4069091D506DC01ED918C
:10284000FC910680F781E02D19958091D406909136
:10285000D5060E94A6560E94C1756BEB7AE0809166
:10286000D4069091D5060E94B9560E94C1756AE9B6
:102870007AE08091D4069091D5060E9448558091C7
:10288000460F8436C8F463E97AE08091D4069091CB
:10289000D5060E9448556091460F8091D4069091CC
:1028A000D5060E943F4861E97AE08091D406909174
:1028B000D5060E94B95603C080E00E94967560E775
:1028C0007AE08091D4069091D5060E944855809177
:1028D000450F8436C8F469E67AE08091D406909179
:1028E000D5060E9448556091450F8091D40690917D
:1028F000D5060E943F4867E67AE08091D406909121
:10290000D5060E94B95603C080E00E94967566E421
:102910007AE08091D4069091D5060E944855609146
:10292000530F7091540F1616170614F50091D40624
:102930001091D506072E000C880B990B0E9426B724
:1029400020E030E04AE754E40E942BB9AB01BC011F
:1029500022E0C8010E94C955C8010E94A65661E440
:102960007AE08091D4069091D5060E94B95603C0B2
:1029700080E00E9496750E9492968091D406909174
:10298000D506DC01ED91FC910680F781E02D1995CB
:102990008091D4069091D5060E94A6560E94C175DA
:1029A00060E37CE08091D4069091D5060E94B956F0
:1029B0000E94C175209154068091D4069091D5064D
:1029C000222309F4C3C161E07CE00E9448550E94C3
:1029D000FF610E9496750E94FF612091D40630919C
:1029E000D506882389F06EEE7BE0C9010E94485528
:1029F000809157060E949237BC018091D406909135
:102A0000D5060E94B9564FC06BED7BE0C9010E940C
:102A10004855809154060E949237BC018091D4069B
:102A20009091D5060E944855809155068823A9F1BA
:102A300063ED7BE08091D4069091D5060E944855C5
:102A4000E0915506E4300CF0E0E08CE793E09A83E7
:102A500089838AE793E09C838B8388E793E09E8356
:102A60008D8386E793E098878F83EE0FFF0B81E0DD
:102A700090E08C0F9D1FE80FF91F6081718180919C
:102A8000D4069091D5060E94485561ED7BE0809177
:102A9000D4069091D5060E9448558091D406909115
:102AA000D5060E94A6566EEB7BE08091D4069091ED
:102AB000D5060E944855809156060091D406109183
:102AC000D506882321F00E949237BC0102C06AEB30
:102AD0007BE0C8010E94B95667EA7BE08091D4068A
:102AE0009091D5060E944855809157060091D406D2
:102AF0001091D506882321F00E949237BC0102C0B4
:102B000063EA7BE0C8010E94B95660E97BE08091EE
:102B1000D4069091D5060E94485580915906882385
:102B2000E1F06AE87BE08091D4069091D5060E949E
:102B30004855809158060E949237BC018091D40676
:102B40009091D5060E94485564E176E08091D406C4
:102B50009091D5060E94A95603C080E00E94967508
:102B600067E77BE08091D4069091D5060E94485596
:102B700080915A068823E1F061E77BE08091D406DA
:102B80009091D5060E944855809158060E94923730
:102B9000BC018091D4069091D5060E94485564E10D
:102BA00076E08091D4069091D5060E94A95603C084
:102BB00080E00E9496756EE57BE08091D40690914E
:102BC000D5060E944855E0915B06E3300CF0E3E047
:102BD00086E09BE09A8389838AEF9AE09C838B83CB
:102BE00085EF9AE09E838D838DEE9AE098878F83A0
:102BF000EE0FFF0BA1E0B0E0AC0FBD1FEA0FFB1F13
:102C0000608171818091D4069091D5060E94B95659
:102C10006BE47BE08091D4069091D5060E944855E4
:102C2000E0914D06E4300CF0E4E086EE9AE09A8301
:102C3000898380EE9AE09C838B8389ED9AE09E8362
:102C40008D8383ED9AE098878F838BEC9AE09A8747
:102C50008987EE0FFF0B81E090E08C0F9D1FE80F3E
:102C6000F91F608171818091D4069091D5060E94F0
:102C7000B95669E47BE08091D4069091D5060E9414
:102C80004855609152068091D4069091D5060E94D5
:102C90003F486AE37BE08091D4069091D5060E947C
:102CA000485580914D06811110C060915306809166
:102CB000D4069091D5060E943F486FE27BE0809158
:102CC000D4069091D5060E94485560914E067091A9
:102CD0004F06072E000C880B990B0E9426B720E0A8
:102CE00030E04AE754E40E942BB9AB01BC0121E07B
:102CF0008091D4069091D5060E94C95561E27BE08F
:102D00008091D4069091D5060E9448556091500656
:102D100070915106072E000C880B990B0E9426B764
:102D200020E030E04AE754E40E942BB9AB01BC013B
:102D300021E08091D4069091D5060E94C95562E1A8
:102D40007BE08091D4069091D50602C064E17CE0DE
:102D50000E94B9560E9492968091D4069091D50611
:102D6000DC01ED91FC910680F781E02D19958091B1
:102D7000D4069091D5060E94A6560E94C1756EEAAF
:102D80007CE08091D4069091D5060E94B9560E94AD
:102D9000C17561EA7CE08091D4069091D5060E94CD
:102DA0004855E091940FE5300CF0E5E08FE89CE0A9
:102DB0009A83898388E79CE09C838B8386E69CE0EA
:102DC0009E838D8387E59CE098878F8384E49CE0D5
:102DD0009A8789878CE39CE09C878B87EE0FFF0B9B
:102DE00081E090E08C0F9D1FE80FF91F60817181D9
:102DF0008091D4069091D5060E94B9560E94929671
:102E00008091D4069091D506DC01ED91FC9106806D
:102E1000F781E02D199583E59AE7A1E0BB278BABFD
:102E20009CABADABBEAB8091D4069091D5060E9411
:102E3000A6560E94C17563EC7EE08091D406909105
:102E4000D5060E94B9560E94C1756AEA7EE080915B
:102E5000D4069091D5060E9448552091110B80917F
:102E6000D4069091D506222319F066EA7EE002C0CE
:102E700061EA7EE00E94B9568091110B882349F1E6
:102E800068E87EE08091D4069091D5060E9448556E
:102E90006091920F7091930F072E000C880B990B85
:102EA0000E9426B720E030E04AE754E40E942BB9A4
:102EB000AB01BC0122E08091D4069091D5060E941E
:102EC000C95563E87EE08091D4069091D5060E94B2
:102ED000B95697ECE92E9EE0F92E29E2622E38E1F0
:102EE000232E3CEF332E4AE0A42EB12C54E6C52EFF
:102EF000D12CD7012C91222309F400C2F70132977B
:102F0000008111810115110509F4F8C180EB99E7E1
:102F1000A1E0BB27820F911DA11DB11DABBFFC011C
:102F2000879177247394811101C0712C2091D4066C
:102F30003091D506C8010197849790F563E67EE04D
:102F4000C9010E94485509500C3148F4E02FF0E0C7
:102F5000EE0FFF1FE25EFD4F6081718102C069EBE1
:102F60007CE08091D4069091D5060E9448550C31A2
:102F700030F4E02FF0E0EA5AFD4F808101C080E09C
:102F800090E0875A914F092E000CAA0BBB0BABBFE8
:102F9000FC0187919EE0981B892F09F051C152C115
:102FA000C801845691098438934008F03FC069E411
:102FB0007EE0C9010E944855C801B6010E945EBA70
:102FC0006130710531F06230710559F465E47EE0DD
:102FD00002C067E47EE08091D4069091D5060E94FD
:102FE00048550E94B9758090D4069090D5067720F8
:102FF000B1F0C8010E947D91811107C061E47EE0BB
:10300000C4010E94485587E01BC1813009F01AC1F4
:103010006EE37EE0C4010E94485588E011C165E37B
:103020007EE0C4010E94485582E00AC1C801885E62
:1030300093408035964408F05AC0C80168EE73E0AA
:103040000E945EBA4B0168E27EE0C9010E944855C9
:10305000FAE08F16910410F40E94B175B4018091CA
:10306000D4069091D5060E946C490E94B975409093
:10307000D4065090D5067720A1F1C8010E947D9119
:10308000782E63E27EE0C2010E944855672D809150
:10309000D4069091D5060E943F486DE17EE0809174
:1030A000D4069091D5060E944855829CC001839C0D
:1030B000900D929C900D1124800F911FB5010E94DC
:1030C00072BA77278091D4069091D5060E946C49F8
:1030D0006BE17EE08091D4069091D5060E94485520
:1030E000B1C062E17EE0C2010E94485561C0F801B2
:1030F000E853FA44E83E43E0F40708F046C0EC30F9
:10310000F10508F09FC08827EE58FF4F8F4F0C94B1
:1031100085BA63E07EE019C068EF7DE0C9010E94D6
:10312000485583E18DC066EE7DE027C066ED7DE009
:1031300016C069EC7DE055C06DEB7DE0C9010E94D1
:10314000485582E17DC06EEA7DE0C9010E94485584
:103150008FE076C06FE97DE0F8CF6FE87DE0C901D0
:103160000E9448558EE06CC06CE77DE0C9010E946A
:1031700048558BE065C06AE67DE0C9010E9448556C
:103180008CE05EC06DE57DE02CC0C80180529E449D
:10319000883E934078F4005266E47DE0C9010E94C5
:1031A00048550A3010F40E94B175802F0E9479753D
:1031B00084E046C0C80188509245883E934020F480
:1031C00008506FE27DE0EACF013FE5E51E0719F404
:1031D0006EE17DE01CC0023FF5E51F0739F461E1B7
:1031E0007DE0C9010E94485581E12AC0033F45E5C1
:1031F000140739F463E07DE0C9010E94485580E17D
:103200001FC0043F85E5180739F462EF7CE0C9016F
:103210000E9448558DE014C0053F95E5190739F423
:103220006AED7CE0C9010E94485586E009C0063F6E
:10323000154541F461EC7CE0C9010E94485585E0E8
:103240000E943A986EE77EE08091D4069091D50670
:103250000E94485563E77EE08091D4069091D506A0
:103260000E944855F701608170E08091D4069091EA
:10327000D5060E946C49D7018C918A3020F482E0F7
:103280000E943A9804C0843610F40E94B1750E94DE
:10329000B975F7014081649EA0011124052E000C30
:1032A000660B770B8BA99CA9ADA9BEA9480F591F26
:1032B0006A1F7B1FDE0111968A019B010F5F1F4F62
:1032C0002F4F3F4F6BBFFA0187918D93B901A80132
:1032D0008111F2CFBE016F5F7F4F8091D406909134
:1032E000D5060E94A9568091D4069091D506DC019E
:1032F000ED91FC910680F781E02D1995B3E0EB0E7E
:10330000F11CEFE3EE16EFE0FE0609F0F2CD0E94AD
:1033100092968091D4069091D506DC01ED91FC91B6
:103320000680F781E02D19958091D4069091D506FD
:103330000E94A6560E94C17564E27FE08091D40687
:103340009091D5060E94B9560E94C17561E17FE057
:103350008091D4069091D5060E9448550E94178FFF
:1033600020E030E040E050E40E9420B72091D406F5
:103370003091D50687FF3EC06EE07FE0C90158C09E
:10338000F090680F00916B0F11E00C9445116EECFA
:1033900079E08091D4069091D5060E9448556091BD
:1033A0009A138091D4069091D5060E943F486CEC08
:1033B00079E08091D4069091D5060E9448550C94EE
:1033C000C91163E879E08091D4069091D5060E94F6
:1033D000485560919C138091D4069091D5060E9427
:1033E0003F4861E879E08091D4069091D5060E942B
:1033F00048552DC86AE07FE0C9010E94B95667EFC1
:103400007EE08091D4069091D5060E9448550E9496
:10341000178FAB01BC0122E08091D4069091D506B4
:103420000E94C95565EF7EE08091D4069091D50643
:103430000E94B95662EE7EE08091D4069091D50646
:103440000E9448558091DE0F0E9488752091DE0F02
:103450008091D4069091D506222379F06FED7EE01D
:103460000E9448550E94799865ED7EE08091D406CF
:103470009091D5060E94B95602C00E94A6560E949D
:1034800092968091D4069091D506DC01ED91FC9145
:103490000680F781E02D19958091D4069091D5068C
:1034A0000E94A6560E94C1756CE77FE08091D40609
:1034B0009091D5060E94B9560E94C17568E67FE0DA
:1034C0008091D4069091D5060E9448554091CE0F28
:1034D0005091CF0F6091D00F7091D10F8091D40691
:1034E0009091D5060E94594964E57FE08091D40609
:1034F0009091D5060E9448554091D60F5091D70F14
:103500006091D80F7091D90F8091D4069091D50613
:103510000E94594960E47FE08091D4069091D506DD
:103520000E9448554091D20F5091D30F6091D40F13
:103530007091D50F8091D4069091D5060E9459497B
:103540006CE27FE08091D4069091D5060E944855A8
:103550004091DA0F5091DB0F6091DC0F7091DD0F1D
:103560008091D4069091D5060E9459490E94929666
:103570008091D4069091D506DC01ED91FC910680F6
:10358000F781E02D19958091D4069091D5060E947F
:10359000A6560E94C175E6960FB6F894DEBF0FBE20
:1035A000CDBFDF91CF911F910F91FF90EF90DF90F2
:1035B000CF90BF90AF909F908F907F906F905F90D3
:1035C0004F903F902F9008952F923F924F925F928D
:1035D0006F927F928F929F92AF92BF92CF92DF9223
:1035E000EF92FF920F931F93CF93DF93CDB7DEB788
:1035F000AB970FB6F894DEBF0FBECDBF83ED91E061
:103600000E9451B86338714F8105910519F00E94ED
:10361000CF3808C047ED51E060E070E080E29EE006
:103620000E9439B840E052EC61E070E089EF98E028
:103630000E9464724091D20F5091D30F6091D40FC9
:103640007091D50F8CE598E00E9464724091D60F7E
:103650005091D70F6091D80F7091D90F8FEB97E0F1
:103660000E9464724091DA0F5091DB0F6091DC0F81
:103670007091DD0F82E297E00E9464728BEC9DE016
:103680009093200780931F078CE89BE090931E0780
:1036900080931D0789EF98E09093BA138093B91334
:1036A0001092DA111092D00D1092CD0D1092CF0D14
:1036B0001092CE0D11E01093AB120E946D95809187
:1036C000F20F8093D7061092D6061092800082E007
:1036D000809381008FE286BB10926F00109285006C
:1036E000109284009BE29093A00099E09093A10037
:1036F00089BB109272001092A5001092A400109243
:10370000A9001092A8001092AB001092AA0010928B
:10371000AD001092AC0099EA909320011093210122
:103720008ABB10927300109225011092240110920E
:1037300029011092280110922B0110922A01109257
:103740002D0110922C018091BD0E9091BE0E8093A0
:10375000680690936906813001F58FE38093340BFE
:103760001092350B61E00E94EF588AE29BE00E94C4
:10377000CB3C1092360B1092390B1092380B809183
:103780006906882329F08AE29BE00E94239811C0F1
:103790008AE29BE00E94753E0CC0809169068823F6
:1037A00011F062E001C060E08FE30E94EF580E94D8
:1037B00091668091BF0E9091C00E80936E0690939B
:1037C0006F06813001F58EE38093650B1092660BD6
:1037D00061E00E94EF588BE59BE00E94CB3C109289
:1037E000670B10926A0B1092690B80916F06882309
:1037F00029F08BE59BE00E94239811C08BE59BE0AC
:103800000E94753E0CC080916F06882311F062E023
:1038100001C060E08EE30E94EF580E945E6660E0A7
:1038200085E40E94EF5862E08CE30E94EF5862E06A
:103830008BE30E94EF5862E080E40E94EF5862E060
:1038400081E40E94EF5862E082E40E94EF5862E057
:1038500081E20E94EF5862E084E40E94EF5861E048
:1038600089E30E94EF5861E08AE30E94EF580E94CA
:10387000D08D0E94058E61E085E30E94EF5861E0E3
:1038800085E00E94EF5861E070E085E00E942B59CE
:1038900061E084E00E94EF5861E087E00E94EF5809
:1038A00061E089E20E94C05861E089E20E94EF581D
:1038B000519A60E085E30E94C05860E085E00E9474
:1038C000C05860E084E00E94C05860E087E00E9439
:1038D000C058599861E088E00E94EF5880E090E07D
:1038E0009C01205E314FF901E955FF4F40814F3671
:1038F00029F4329720813181232B31F403968837C4
:10390000910571F760E001C061E088E00E94C05855
:1039100061E08BE20E94EF5860E08BE20E94C058A9
:103920000E94058E0E94EA4880911A0B813009F0AE
:103930006CC080911D0B90911E0BA0911F0BB0913C
:10394000200B4091210B5091220B6091230B709121
:10395000240B841B950BA60BB70B84379E40A10547
:10396000B10500F30E94CF388091D4069091D5061E
:103970000E94A6568091D4069091D5060E94A65624
:103980000E94C1756AE87FE08091D4069091D506C7
:103990000E94485501E010E00E94D48D0E94058EDF
:1039A0006EEE72E080E090E00E941E8967E87FE0A2
:1039B0008091D4069091D5060E9448550E94D08DE2
:1039C0000E94018E0530110531F064EF71E080E056
:1039D00090E00E941E890F5F1F4F06301105E1F62F
:1039E0008091D4069091D5060E94A6560E94C1757A
:1039F0008091D4069091D5060E94A6568091D40657
:103A00009091D5060E94A65602C081118BCF80915D
:103A10006F00826080936F00809184009091850098
:103A20008056904F90938900809388000E943D2992
:103A30008DE89BE0909302128093011210918D0FFC
:103A400020918C0F80917B0F90917D0F30917E0F94
:103A500030932107909332068093330630E0AFEF26
:103A6000B0E00E94B7B824E630E040E050E00E94A9
:103A700069B82093A313612F70E080E090E00E946A
:103A800024B723EC34E64AEA5AE30E9485B72AE9D0
:103A900039E949E55FE30E94C7B860939D137093CD
:103AA0009E1380939F139093A013109295001092F1
:103AB0009400109290008CE08093910084EF90E04D
:103AC000909399008093980011E018BB82E0809356
:103AD0007100809100020E94BD698091D40690918E
:103AE000D5062091D7064091770F5091780F5093CB
:103AF000DD0D4093DC0D20935C1290935B1280935C
:103B00005A12109234061093DE0D8091940F853076
:103B100040F01092940F60E070E084E791E00E9422
:103B20007B481091940F123009F444C008F511231A
:103B300009F466C0113009F05BC08CE090E00E948F
:103B400099BA26E433E0DC0111963C932E932FEBD7
:103B500037E01B963C932E931A979093D10680934F
:103B6000D00610939112109394121093971267C07D
:103B7000133009F45EC01430D9F586E090E00E945D
:103B800099BA8C012EEA33E0DC012D933D93CD01EF
:103B900041E06DE87BE00E94AF4186E792E0F801EA
:103BA000918380831093D1060093D00681E08093A7
:103BB000911241C086E090E00E9499BA2EED32E069
:103BC000FC01318320839093D1068093D0068FB778
:103BD000F8942CED35E030931A11209319111092BE
:103BE0001F118FBF81E0809391128093941225C0A2
:103BF0001092940F60E070E084E791E00E947B48AF
:103C000086E090E00E9499BA8C012EEA33E0DC0154
:103C10002D933D93CD0140E06DE87BE00E94AF41E4
:103C200086E792E0F801918380831093D106009398
:103C3000D0061092911210929412109297128091C5
:103C4000D0069091D106DC01ED91FC910190F081BC
:103C5000E02D19958091851281111FC080918812E5
:103C600081111BC080918B12811117C080918E121F
:103C7000811113C08091911281110FC08091941213
:103C800081110BC080919712811107C081E00E94C1
:103C90001E6A882309F418C310C3A12CB12C812CEF
:103CA000912C1DA2412C512C612C712C04EF15E09C
:103CB000EE24EA94A3E0FA2ECC24CA94DD24D39413
:103CC00088EE282E85E0382EC501805E914FFC01DC
:103CD000E955FF4FE081EE2309F4E6C2DC01AB5564
:103CE000BF4F8D919C91892B09F4DEC28E2F90E0FD
:103CF000FC01F797EB32F10508F0D6C28827E258AD
:103D0000FF4F8F4F0C9485BA80918512882309F458
:103D1000CBC27110C9C289E190E00E9499BA9C019E
:103D2000FC011183008387E090E0938382831582F6
:103D30001482F782E682D186C086108EC9012AA736
:103D40003BA70E940B832AA53BA5EAE3F4E0D90137
:103D5000ED93FC933093761220937512C9010E9463
:103D6000C17C7DC180918812882309F49DC26110B5
:103D70009BC289E190E00E9499BA9C01DC011196F6
:103D80001C930E93E6E0F0E01396FC93EE931297EB
:103D900015961C921E9214971796FC92EE92169707
:103DA0001996DC92CE92189758961C922AA73BA798
:103DB0000E940B832AA53BA5EAE3F4E0D901ED9329
:103DC000FC933093781220937712C9010E94C17C32
:103DD00074C180918B12882309F466C2511064C2A9
:103DE00089E190E00E9499BA9C01DC0111961C9334
:103DF0000E93E5E0F0E01396FC93EE931297159680
:103E00001C921E9214971796FC92EE921697199692
:103E1000DC92CE92189758961C922AA73BA70E9434
:103E20000B832AA53BA5EAE3F4E0D901ED93FC93CB
:103E300030937A1220937912C9010E94C17C6BC120
:103E400080918E12882309F42FC241102DC289E17E
:103E500090E00E9499BA9C01DC0111961C930E938C
:103E6000E4E0F0E01396FC93EE93129715961C9203
:103E70001E9214971796FC92EE9216971996DC9262
:103E8000CE92189758961C922AA73BA70E940B83A4
:103E90002AA53BA5EAE3F4E0D901ED93FC93309326
:103EA0007C1220937B12C9010E94C17C62C1809167
:103EB0009112882309F4F8C12DA12111F5C189E1DE
:103EC00090E00E9499BA9C01DC0111961C930E931C
:103ED000E2E0F0E01396FC93EE93129715961C9295
:103EE0001E9214971796FC92EE9216971996DC92F2
:103EF000CE92189758961C922AA73BA70E940B8334
:103F00002AA53BA5EAE3F4E0D901ED93FC933093B5
:103F10007E1220937D12C9010E94C17C62C18091F2
:103F20009412882309F4C0C19110BEC189E190E0C8
:103F30000E9499BA9C01DC0111961C930E93E1E05A
:103F4000F0E01396FC93EE93129715961C921E9236
:103F500014971796FC92EE9216971996DC92CE92D1
:103F6000189758961C922AA73BA70E940B832AA554
:103F70003BA5EAE3F4E0D901ED93FC933093801282
:103F800020937F12C9010E94C17C62C18091971267
:103F9000882309F489C1811087C189E190E00E94DA
:103FA00099BA9C01DC0111961C930E9313961C92F6
:103FB0001E92129715961C921E9214971796FC92B9
:103FC000EE9216971996DC92CE92189758961C92FC
:103FD0002AA73BA70E940B832AA53BA58AE394E06E
:103FE000F901918380833093821220938112C90159
:103FF0000E94C17C57C180918512882309F454C165
:10400000711052C18CE190E00E9499BA9C01DC01D0
:1040100011961C930E93E7E0F0E01396FC93EE9359
:10402000129715961C921E9214971796FC92EE9278
:1040300016971996DC92CE92189758961C922AA73A
:104040003BA70E940B832AA53BA5D9012D923C9248
:104050003093841220938312C9010E94807D7724BB
:10406000739422C180918812882309F41DC16110C4
:104070001BC18CE190E00E9499BA9C01FC01118364
:10408000008386E090E09383828315821482F78216
:10409000E682D186C086108EC9012AA73BA70E945E
:1040A0000B832AA53BA5D9012D923C923093871210
:1040B00020938612C9010E94807D66246394F4C017
:1040C00080918B12882309F4EFC05110EDC08CE170
:1040D00090E00E9499BA9C01FC011183008385E065
:1040E00090E09383828315821482F782E682D186E0
:1040F000C086108EC9012AA73BA70E940B832AA560
:104100003BA5D9012D923C9230938A1220938912BB
:10411000C9010E94807D55245394C6C080918E129F
:10412000882309F4C1C04110BFC08CE190E00E9417
:1041300099BA9C01FC011183008384E090E0938391
:10414000828315821482F782E682D186C086108E21
:10415000C9012AA73BA70E940B832AA53BA5D90129
:104160002D923C9230938D1220938C12C9010E94A3
:10417000807D4424439498C080919112882309F44F
:1041800093C02DA1211190C08CE190E00E9499BABA
:104190009C01DC0111961C930E93E2E0F0E0139673
:1041A000FC93EE93129715961C921E9214971796F5
:1041B000FC92EE9216971996DC92CE92189758962A
:1041C0001C922AA73BA70E940B832AA53BA5D901D5
:1041D0002D923C923093901220938F12C9010E942D
:1041E000807D21E02DA360C080919412882309F482
:1041F0005BC0911059C08CE190E00E9499BA9C017B
:10420000DC0111961C930E93E1E0F0E01396FC9311
:10421000EE93129715961C921E9214971796FC9285
:10422000EE9216971996DC92CE92189758961C9299
:104230002AA73BA70E940B832AA53BA5D9012D9253
:104240003C923093931220939212C9010E94807D78
:104250009924939429C080919712882329F1811081
:1042600023C08CE190E00E9499BA9C01FC0111836B
:1042700000831382128215821482F782E682D1862D
:10428000C086108E2AA73BA70E940B832AA53BA5B8
:10429000D9012D923C923093961220939512C90128
:1042A0000E94807D88248394B3E0AB0EB11CE8E7C4
:1042B000AE16B10409F008CDE9CC82E00E941E6A76
:1042C000882311F01FA216C081E00E941E6A882375
:1042D00029F082E00E94026A81118AC78CE30E9461
:1042E0009858892B09F075C78CE30E949858892B40
:1042F00009F075C786E0E4ECFFE0DE01549601901A
:104300000D928A95E1F78091BD0F9091CD0FB090FD
:10431000BE0F0091BF0F1091C00F7091C10F60913F
:10432000C20F5091C30F4091CA0F2091CB0F309113
:10433000CC0FA091D006B091D106BEA3ADA3E09161
:104340008E13F0918F13F9A7E8A79090F00F60906B
:10435000EB0FE090E40FF090E50F8090EE0F70907F
:10436000ED0FC090530FD090540F5090560F4090C7
:10437000510F3090520FFFA1FB8B8A8F9B8FBC8E09
:104380000D8F1E8F7F8F68A359A34AA33CA32BA335
:10439000F2E1AF2EFE017396DE01119601900D92AF
:1043A000AA94E1F7EDE8FBE0F0933D06E0933C06CC
:1043B000AFA1A98388879987BA860B871C877D87D9
:1043C0006E875F87488B3A8B298B22E1FE013196FD
:1043D000ADE4B6E001900D922A95E1F7992321F022
:1043E000863011F0109255063092561240925712B4
:1043F00050925412D0924D12C0924C12609290136F
:104400007092511280925012F0924F12E0924E121E
:104410009092551288A599A59093531280935212A9
:104420008DA19EA190933F0680933E0687E08093E6
:104430001A0A10921B0A61E00E94EF5880E19AE08C
:104440000E94CB3C10921C0A10921F0A10921E0A66
:1044500080915806811102C010925906909154061D
:10446000911105C0811103C01092010B98C0809179
:10447000FC0A9091FD0A0E943C5281E08093010B5E
:1044800080914D06882359F1813071F08330C1F459
:1044900088E293E290934F0680934E0689E08093E2
:1044A000520680E197E217C088EB9BE090934F069D
:1044B00080934E0683E08093520688E99AE30BC00E
:1044C00088E893E190934F0680934E0686E08093B0
:1044D000520680EE9EE290935106809350068091A2
:1044E00054068823E9F1809158066091520670E0E5
:1044F0008823C9F080915A068823A9F080E090E0D3
:104500000E9424B79B01AC0160E070E088EC92E46B
:104510000E942BB960934006709341068093420637
:104520009093430625C080E090E00E9424B79B0151
:10453000AC0160E070E088EC92E40E942BB96093DB
:104540004006709341068093420690934306109272
:104550003706109238061092390610923A061FC09C
:1045600010924006109241061092420610924306A5
:104570006091530670E080E090E00E9424B79B01B8
:10458000AC0160E070E088EC92E40E942BB960938B
:104590003706709338068093390690933A06109246
:1045A0004A061092440610923B061092450610925D
:1045B000460610924706109248060E94518650986F
:1045C000589AE898809169008C7F80936900809167
:1045D0005712882321F080916900826003C0809186
:1045E0006900836080936900E8980E942F6180E0F1
:1045F00090E040E09C01205E314FF901E955FF4F0A
:104600005081552331F0329720813181232B09F0DD
:104610004F5F03968837910569F740936106A0E7DD
:10462000B6E020E030E080EB282E88E7382E9DE6CB
:10463000492E95E6592E42E4642E45E6742E55E542
:10464000852E55E6952E63EBA62E68E7B62E46EF2F
:1046500053E705EB18E772ECE72E78E7F72EE0E07A
:10466000CE2EE3E7DE2EC901805E914FFC01E955B5
:10467000FF4F6081662309F49EC38B559F4FFC0159
:1046800080819181892B09F496C370E0FB013197F9
:10469000E23AF10508F08FC38827E755FF4F8F4FA7
:1046A0000C9485BA8BE291E911969C938E9383C307
:1046B00089E291E911969C938E937DC387E291E9FB
:1046C00011969C938E9377C380E291E911969C9307
:1046D0008E9371C38EE191E911969C938E936BC377
:1046E0008CE890E911969C938E9365C386E990E9D6
:1046F00011969C938E935FC38FE690E911969C93DD
:104700008E9359C38BE590E911969C938E9353C376
:104710008CE490E911969C938E934DC380EF9FE8B3
:1047200011969C938E9347C387EA9FE811969C93BA
:104730008E9341C38FEB9BE711969C938E933BC363
:104740008AE49BE711969C938E9335C384EB9BE799
:1047500011969C938E932FC38DEB9BE711969C93A0
:104760008E9329C386EB9BE711969C938E9323C36C
:104770008DE79BE711969C938E931DC385EA9BE77B
:1047800011969C938E9317C38EE99BE711969C9389
:104790008E9311C38DE69BE711969C938E930BC36A
:1047A0008BE69BE711969C938E9305C389E69BE766
:1047B00011969C938E93FFC289E59BE711969C937B
:1047C0008E93F9C287E59BE711969C938E93F3C273
:1047D00088E49BE711969C938E93EDC288E39BE758
:1047E00011969C938E93E7C286E39BE711969C9368
:1047F0008E93E1C284E39BE711969C938E93DBC278
:1048000084E998E711969C938E93D5C282E998E744
:1048100011969C938E93CFC280E998E711969C9352
:104820008E93C9C280E99CE811969C938E93C3C273
:1048300082E39BE711969C938E93BDC282E29BE735
:1048400011969C938E93B7C28CEA99E711969C932C
:104850008E93B1C28DE899E711969C938E93ABC26B
:1048600080E29BE711969C938E93A5C281EF9AE715
:1048700011969C938E939FC28AEE9AE711969C9311
:104880008E9399C289EB9AE711969C938E9393C26B
:1048900084E391E911969C938E938DC287EB9AE7FE
:1048A00011969C938E9387C285EB9AE711969C9301
:1048B0008E9381C282EB9AE711969C938E937BC272
:1048C0008EE89AE711969C938E9375C28AE69AE7D2
:1048D00011969C938E936FC28FEA9AE711969C93E0
:1048E0008E9369C28BE89AE711969C938E9363C26C
:1048F00087E69AE711969C938E935DC28CEA9AE7BD
:1049000011969C938E9357C288E89AE711969C93D0
:104910008E9351C284E69AE711969C938E934BC274
:1049200089EA9AE711969C938E9345C285E89AE7A7
:1049300011969C938E933FC281E69AE711969C93C1
:104940008E9339C286EA9AE711969C938E9333C26E
:1049500082E89AE711969C938E932DC28EE59AE792
:1049600011969C938E9327C283EA9AE711969C93A3
:104970008E9321C28FE79AE711969C938E931BC268
:104980008BE59AE711969C938E9315C280EA9AE77D
:1049900011969C938E930FC28CE79AE711969C9385
:1049A0008E9309C288E59AE711969C938E9303C271
:1049B0008DE99AE711969C938E93FDC189E79AE75A
:1049C00011969C938E93F7C185E59AE711969C9377
:1049D0008E93F1C18AE99AE711969C938E93EBC16D
:1049E00086E79AE711969C938E93E5C182E59AE754
:1049F00011969C938E93DFC187E99AE711969C9359
:104A00008E93D9C183E79AE711969C938E93D3C175
:104A10008FE49AE711969C938E93CDC184E99AE72F
:104A200011969C938E93C7C180E79AE711969C9349
:104A30008E93C1C18CE49AE711969C938E93BBC16F
:104A400081E99AE711969C938E93B5C18DE69AE71A
:104A500011969C938E93AFC189E49AE711969C932B
:104A60008E93A9C18FEC98E711969C938E93A3C166
:104A700085E49AE711969C938E939DC181E49AE711
:104A800011969C938E9397C18DE39AE711969C9310
:104A90008E9391C189E39AE711969C938E938BC173
:104AA00085E39AE711969C938E9385C181E39AE7FB
:104AB00011969C938E937FC18DE29AE711969C93F9
:104AC0008E9379C189E29AE711969C938E9373C174
:104AD00080E29AE711969C938E936DC18EE898E7D9
:104AE00011969C938E9367C18CE898E711969C93DE
:104AF0008E9361C181EF99E711969C938E935BC170
:104B000089EE98E711969C938E9355C187E19AE7B9
:104B100011969C938E934FC18AE898E711969C93C7
:104B20008E9349C188E898E711969C938E9343C170
:104B30008BEC99E711969C938E933DC18BE399E79B
:104B400011969C938E9337C181EE94E711969C93B6
:104B50008E9331C186E994E711969C938E932BC175
:104B60008FE995E611969C938E9325C18BE895E687
:104B700011969C938E931FC187E795E611969C939F
:104B80008E9319C18FE79FE811969C938E9313C162
:104B900083ED93E711969C938E930DC181EC93E77F
:104BA00011969C938E9307C185EA93E711969C9387
:104BB0008E9301C18EEE92E711969C938E93FBC06B
:104BC00084EA92E711969C938E93F5C086EC92E767
:104BD00011969C938E93EFC086EB92E711969C936F
:104BE0008E93E9C088ED92E711969C938E93E3C073
:104BF0008CE792E711969C938E93DDC08CE692E74A
:104C000011969C938E93D7C08EE892E711969C9351
:104C10008E93D1C08AE894E711969C938E93CBC073
:104C20008EE794E711969C938E93C5C082E794E734
:104C300011969C938E93BFC086E694E711969C9341
:104C40008E93B9C08AE594E711969C938E93B3C076
:104C50008EE494E711969C938E93ADC082E494E722
:104C600011969C938E93A7C08CE693E711969C9324
:104C70008E93A1C08AE593E711969C938E939BC077
:104C800088E493E711969C938E9395C086E393E70F
:104C900011969C938E938FC084E293E711969C9318
:104CA0008E9389C082E193E711969C938E9383C083
:104CB0001196DC92CE927FC01196FC92EE927BC050
:104CC00011961C930E9377C08CE194E711969C93F8
:104CD0008E9371C011965C934E936DC01196BC92E9
:104CE000AE9269C011969C928E9265C011967C928C
:104CF0006E9261C011965C924E925DC011963C928C
:104D00002E9259C0EDEAF8E71196FC93EE9353C04A
:104D100084EA98E711969C938E934DC0E6E7F5E7F9
:104D20001196FC93EE9347C083E795E711969C9309
:104D30008E9341C0E0E7F5E71196FC93EE933BC0FC
:104D40008DE695E711969C938E9335C0E2E6F5E7E4
:104D50001196FC93EE932FC08BE695E711969C93EA
:104D60008E9329C0E4E6F5E71196FC93EE9323C0F9
:104D700088E993E711969C938E931DC0EBE8F3E7C7
:104D80001196FC93EE9317C08EE793E711969C93D0
:104D90008E9311C0E0E5F5E71196FC93EE930BC0FE
:104DA0008EE395E711969C938E9305C0ECE2F5E7B0
:104DB0001196FC93EE932D5F3F4F129628373105E5
:104DC00009F051CC1092640680916806811114C0DC
:104DD00080E090E0FC01EB53F14F208131812456BB
:104DE00031092436310528F003968837910591F76B
:104DF00003C081E08093640610926A0680916E067B
:104E0000811114C080E090E0FC01EB53F14F208150
:104E10003181285C31092436310528F00396883722
:104E2000910591F703C081E080936A068091D006D6
:104E30009091D106DC01ED91FC91E05BFF4F209158
:104E4000970F3091980F4091950F5091960F0190C8
:104E5000F081E02D61E019958091D0069091D10606
:104E6000DC01ED91FC91E05BFF4F20919B0F3091B5
:104E70009C0F4091990F50919A0F0190F081E02D75
:104E800062E019958091D0069091D106DC01ED91F8
:104E9000FC91E05BFF4F20919F0F3091A00F40915C
:104EA0009D0F50919E0F0190F081E02D63E01995C8
:104EB0008091D0069091D106DC01ED91FC91E05BF0
:104EC000FF4F2091AA0F3091AB0F4091A80F509146
:104ED000A90F0190F081E02D64E019958091D00632
:104EE0009091D106DC01ED91FC91E05BFF4F2091A8
:104EF000AE0F3091AF0F4091AC0F5091AD0F0190BC
:104F0000F081E02D65E019958091D0069091D10651
:104F1000DC01ED91FC91E05BFF4F2091B20F3091ED
:104F2000B30F4091B00F5091B10F0190F081E02D7F
:104F300066E019958091D0069091D106DC01ED9143
:104F4000FC91EE5AFF4F0190F081E02D4091A10FAE
:104F500061E019958091D0069091D106DC01ED9128
:104F6000FC91EE5AFF4F0190F081E02D4091A20F8D
:104F700062E019958091D0069091D106DC01ED9107
:104F8000FC91EE5AFF4F0190F081E02D4091A30F6C
:104F900063E019958091D0069091D106DC01ED91E6
:104FA000FC91EE5AFF4F0190F081E02D4091B40F3B
:104FB00064E019958091D0069091D106DC01ED91C5
:104FC000FC91EE5AFF4F0190F081E02D4091B50F1A
:104FD00065E019958091D0069091D106DC01ED91A4
:104FE000FC91EE5AFF4F0190F081E02D4091B60FF9
:104FF00066E019958091D0069091D106DC01ED9183
:10500000FC9100ACF1ADE02D6091A50F1995809158
:10501000D0069091D106DC01ED91FC9104ACF5AD88
:10502000E02D6091BA0F19958091D0069091D1062C
:10503000DC01ED91FC9106A4F7A5E02D6091A60F8F
:1050400019958091D0069091D106DC01ED91FC91EB
:1050500004A8F5A9E02D6091A70F19958091D006BD
:105060009091D106DC01ED91FC91E85BFF4F01903E
:10507000F081E02D4091BB0F60E019958091D00642
:105080009091D106DC01ED91FC91E85BFF4F01901E
:10509000F081E02D4091BC0F61E0199580E090E037
:1050A0009C01205E314FF901E955FF4F40814237A5
:1050B00031F4329720813181232B09F09FC0039670
:1050C0008837910569F70E9476928091D006909179
:1050D000D106DC01ED91FC91EE59FF4F0190F0817A
:1050E000E02D40E06091B70F19958091D006909126
:1050F000D106DC01ED91FC91EE59FF4F0190F0815A
:10510000E02D41E06091B90F19958091D006909102
:10511000D106DC01ED91FC91EE59FF4F0190F08139
:10512000E02D42E06091B80F19952091E20F30E038
:10513000AFEFB0E00E94B7B824E630E040E050E0C6
:105140000E9469B8209376138091E10F81110E942B
:105150005C8E0E94E3980E9456896B017C0110E0EE
:1051600011110FC08091D706882359F025EE33E73F
:1051700040ED57E060E070E08DE89BE00E94B643B0
:1051800011E00E94F77F882351F00E947B8D0E94DE
:1051900006680E94058E0E94857F0E94978D0E945E
:1051A0005E85029711F00E943C5A0E9492960E94DE
:1051B0005E850297A9F60E945689DC01CB018C1905
:1051C0009D09AE09BF098C3B9240A105B10540F293
:1051D00018C082E00E941E6A81110DC085C882E05D
:1051E0000E94026A882309F485C883E08FA382C8DD
:1051F000F1E0FFA37FC822E02FA37CC80E946A923F
:1052000064CF0E9490980E94058E8091150B8111A9
:1052100002C00E94F1490E94338586E30E94F25940
:10522000BC01990F880B990B6115710581059105DA
:1052300011F00E94ABB627E632E748EE53E060E09B
:1052400070E08DE89BE0AB960FB6F894DEBF0FBE22
:10525000CDBFDF91CF911F910F91FF90EF90DF9025
:10526000CF90BF90AF909F908F907F906F905F9006
:105270004F903F902F900C94B6437F928F929F92C5
:10528000AF92BF92CF92DF92EF92FF920F931F9354
:10529000CF93DF9381E0809385128093881280936F
:1052A0008B1280938E1280939A1280939D1290910C
:1052B0007E0F9150953040F080937E0F61E070E05A
:1052C0008EE591E00E947B4890917E0F2DEF290F93
:1052D00080913D0F233008F006C28A3079F03CF40B
:1052E000883009F461C0893009F4B7C1ADC18B3091
:1052F00009F4A0C08C3009F4E1C0A6C184E290E0BA
:105300000E9499BAFC018091F10F28E030E03383CC
:1053100022838824839499249A9495828482AA244F
:10532000AA94B12CB782A68211861086108E33E81B
:10533000D32ED18E4FEBE42E47E0F42EF38EE28E87
:105340000AE614E011830083C6EDDFE0D1A3C0A319
:1053500012A283A3F093C606E093C506CF010E9474
:10536000F17784E290E00E9499BAFC018091F10FFC
:1053700029E030E03383228395828482B782A6823B
:1053800011861086108ED18EF38EE28E11830083EB
:10539000D1A3C0A312A283A3F093C406E093C306D3
:1053A000CF010E94F177FEC280E290E00E9499BA9C
:1053B000FC0188E090E093838283AA24A394BB2419
:1053C000BA94B582A482CC24CA94D12CD782C68246
:1053D00011861086108E0AE0F02EF18E0FEB17E08A
:1053E000138F028FC2E5D4E0D183C083F093C60649
:1053F000E093C506CF010E947A7680E290E00E9499
:1054000099BAFC0189E090E093838283B582A482FB
:10541000D782C68211861086108EF18E138F028F6E
:10542000D183C083F093C406E093C306CF010E94EA
:105430007A76B8C289E190E00E9499BAFC0188E0CE
:1054400090E093838283EE24E394FF24FA94F58220
:10545000E4820FEF10E01783068311861086108E0A
:10546000C6E4D4E0D183C083F093C606E093C506BA
:10547000CF010E94247E10929A1280917E0F843078
:1054800009F090C289E190E00E9499BAFC0189E09C
:1054900090E093838283F582E482178306831186EA
:1054A0001086108ED183C083F093C406E093C306A8
:1054B000CF010E94247E10929D1274C2943009F094
:1054C00049C089E190E00E9499BAEC01F4EFAF2E57
:1054D000F5E0BF2EB982A88287E090E09B838A83A3
:1054E000CC24C394DD24DA94DD82CC82EE24EA94C9
:1054F000F12CFF82EE8219861886188ECE010E944A
:105500000B830AE314E019830883D093C606C09383
:10551000C506CE010E94C17C1092851289E190E0FF
:105520000E9499BAEC01B982A88286E090E09B8340
:105530008A83DD82CC82FF82EE8219861886188EDD
:10554000CE010E940B8319830883D093C406C093B5
:10555000C3064BC0953009F04EC089E190E00E942F
:1055600099BAEC0164EFA62E65E0B62EB982A88246
:1055700087E090E09B838A83CC24C394DD24DA9473
:10558000DD82CC82EE24EA94F12CFF82EE82198631
:105590001886188ECE010E940B830AE314E019834B
:1055A0000883D093C406C093C306CE010E94C17C79
:1055B0001092851289E190E00E9499BAEC01B982BB
:1055C000A88286E090E09B838A83DD82CC82FF8282
:1055D000EE8219861886188ECE010E940B831983DD
:1055E0000883D093C606C093C506CE010E94C17C35
:1055F00010928812D7C189E190E00E9499BAEC011B
:1056000084EF95E09983888387E090E09B838A8389
:1056100081E09FEF9D838C838FEF90E09F838E834B
:1056200019861886188ECE010E940B838AE394E0B7
:1056300099838883D093C606C093C506CE010E9485
:10564000C17C10928512AEC189E080933D0F69E064
:1056500070E08DE191E00E947B4880E290E00E9442
:1056600099BAFC0188E090E093838283AA24A394F2
:10567000BB24BA94B582A482CC24CA94D12CD782FC
:10568000C68211861086108E50E8F52EF18E0FEB33
:1056900017E0138F028FCEE5D4E0D183C083F0935F
:1056A000C606E093C506CF010E942C7780E290E009
:1056B0000E9499BAFC0189E090E093838283B582CD
:1056C000A482D782C68211861086108EF18E138F27
:1056D000028FD183C083F093C406E093C306CF0149
:1056E0000E942C775FC18A3009F456C03CF48830A0
:1056F00009F4A0C0893009F400C1F6C08B3009F468
:10570000BAC08C3009F0F0C089E190E00E9499BAEB
:10571000EC0174EFA72E75E0B72EB982A88287E05E
:1057200090E09B838A83CC24C394DD24DA94DD82C9
:10573000CC82EE24EA94F12CFF82EE821986188640
:10574000188ECE010E940B830AE314E019830883AC
:10575000D093C806C093C70689E190E00E9499BA29
:10576000EC01B982A88286E090E09B838A83DD8287
:10577000CC82FF82EE8219861886188ECE010E9496
:105780000B8319830883D093CA06C093C90610926D
:10579000851210928812F0C084E290E00E9499BABB
:1057A000FC01C091F10FD0918A0F88E090E09383C3
:1057B00082838824839499249A9495828482AA244B
:1057C000AA94B12CB782A68211861086108E83E827
:1057D000782E718E9FEBC92E97E0D92ED38EC28E74
:1057E0002AE6E22E24E0F22EF182E08206ED1FE0AE
:1057F00011A300A3D2A3C3A3F093C806E093C706E6
:1058000084E290E00E9499BAFC0189E090E09383E1
:10581000828395828482B782A68211861086108E3A
:10582000718ED38EC28EF182E08211A300A3D2A327
:10583000C3A39EC080E290E00E9499BAFC0188E078
:1058400090E093838283AA24A394BB24BA94B58264
:10585000A482CC24CA94D12CD782C6821186108609
:10586000108EDAE0FD2EF18E0FEB17E0138F028F12
:10587000C2E5D4E062C089E190E00E9499BAFC01DF
:1058800088E090E093838283EE24E394FF24FA94EB
:10589000F582E4820FEF10E01783068311861086ED
:1058A000108EC6E4D4E0D183C083F093C806E093A1
:1058B000C70689E190E00E9499BAFC0189E090E076
:1058C00093838283F582E482178306831186108690
:1058D000108ED183C083F093CA06E093C90610925C
:1058E0009A1210929D1248C089E080933D0F69E0A2
:1058F00070E08DE191E00E947B4880E290E00E94A0
:1059000099BAFC0188E090E093838283AA24A3944F
:10591000BB24BA94B582A482CC24CA94D12CD78259
:10592000C68211861086108E60E8F62EF18E0FEB7F
:1059300017E0138F028FCEE5D4E0D183C083F093BC
:10594000C806E093C70680E290E00E9499BAFC0185
:1059500089E090E093838283B582A482D782C68255
:1059600011861086108EF18E138F028FD183C08323
:10597000F093CA06E093C9068091C9069091CA06C1
:10598000DC01ED91FC910280F381E02D199580916D
:10599000C7069091C806DC01ED91FC910280F3816D
:1059A000E02D199580917E0F833039F0823009F017
:1059B0006CC080913D0F8C3051F189E190E00E94E4
:1059C00099BAEC0184EF95E09983888386E090E0B2
:1059D0009B838A8381E09FEF9D838C838FEF90E090
:1059E0009F838E8319861886188ECE010E940B83A2
:1059F0008AE394E099838883D093C106C093C0065C
:105A0000CE010E94C17C10928812C6E029C089E1B3
:105A100090E00E9499BAEC0184EF95E09983888325
:105A200084E090E09B838A8381E09FEF9D838C8359
:105A30008FEF90E09F838E8319861886188ECE0193
:105A40000E940B838AE394E099838883D093C106F4
:105A5000C093C006CE010E94C17C10928E12C4E099
:105A600060914C0F70914D0F8C2F0E942582609198
:105A70004E0F70914F0F8C2F0E9421828091500FFA
:105A8000E091C006F091C106808FE0913E0F8E2F0D
:105A9000EE0F990BAA0BBB0BFC013897E830F10510
:105AA00008F0BBC08827E55BFE4F8F4F0C9485BA8A
:105AB00084E290E00E9499BAFC018091F10F28E005
:105AC00030E03383228321E03FEF358324832FEFBF
:105AD00030E03783268311861086108E94E8918FEC
:105AE0002FEB37E0338F228F2AE634E03183208397
:105AF00026ED3FE031A320A312A283A31EC080E2C3
:105B000090E00E9499BAFC0188E090E09383828340
:105B100081E09FEF958384838FEF90E09783868366
:105B200011861086108E87E8818F8FEB97E0938F18
:105B3000828F8EE594E091838083F093CF06E0938B
:105B4000CE0699C080E290E00E9499BAFC0188E0FC
:105B500090E09383828381E09FEF958384838FEF2E
:105B600090E09783868311861086108E8DE0818F5A
:105B70008FEB97E0938F828F82E594E0DCCF89E111
:105B800090E00E9499BAFC0188E090E093838283C0
:105B900081E09FEF958384838FEF90E097838683E6
:105BA00011861086108E86E494E091838083F093B2
:105BB000CF06E093CE0610929A125DC08CE190E081
:105BC0000E9499BAEC0184EF95E09983888385E07F
:105BD00090E09B838A8381E09FEF9D838C838FEF8E
:105BE00090E09F838E8319861886188ECE010E94BE
:105BF0000B8388EE95E037C089E190E00E9499BA66
:105C0000FC01138212821582148217821682118679
:105C10001086108E86E194E08ECF8CE080933E0F4C
:105C20006CE070E08EE191E00E947B4889E190E0B9
:105C30000E9499BAEC0184EF95E09983888385E00E
:105C400090E09B838A8381E09FEF9D838C838FEF1D
:105C500090E09F838E8319861886188ECE010E944D
:105C60000B838AE394E099838883D093CF06C09313
:105C7000CE0610928B128091CE069091CF06DC0159
:105C8000ED91FC910280F381E02D19958091460FF2
:105C9000843658F4853608F084E664E6681B809103
:105CA000CE069091CF060E942C4E80913E0F8C50D4
:105CB0008230A8F46091470F7091480F85E00E94F0
:105CC00058816091490F70914A0F85E00E943D8193
:105CD00080914B0FE091CE06F091CF06808F2091FE
:105CE0003F0F822F022E000C990BAA0BBB0BFC015D
:105CF0003897E830F10508F089C08827ED5AFE4F43
:105D00008F4F0C9485BA84E290E00E9499BAFC010E
:105D10008091F10F29E030E03383228321E03FEFCF
:105D2000358324832FEF30E0378326831186108656
:105D3000108E94E8918F2FEB37E0338F228F2AE675
:105D400034E03183208326ED3FE031A320A312A26B
:105D500083A357C080E290E00E9499BAFC0189E0D9
:105D600090E09383828381E09FEF958384838FEF1C
:105D700090E09783868311861086108E87E8818F46
:105D80008FEB97E0938F828F8EE594E038C080E2AE
:105D900090E00E9499BAFC0189E090E093838283AD
:105DA00081E09FEF958384838FEF90E097838683D4
:105DB00011861086108E8DE0818F8FEB97E0938F88
:105DC000828F82E594E01BC080917E0F823009F0C3
:105DD000BBC180913D0F8C3009F0B6C11FC089E175
:105DE00090E00E9499BAFC011382128215821482FB
:105DF0001782168211861086108E86E194E09183B8
:105E00008083F093D306E093D2065EC080917E0F2C
:105E1000823061F580913D0F8C3041F58BE08093AD
:105E20003F0F6BE070E08FE191E00E947B4889E1D9
:105E300090E00E9499BAFC0189E090E0938382830C
:105E400081E09FEF958384838FEF90E09783868333
:105E500011861086108E86E494E091838083F093FF
:105E6000D306E093D20610929D122EC08CE0809350
:105E70003F0F6CE070E08FE191E00E947B4889E188
:105E800090E00E9499BAEC0184EF95E099838883B1
:105E900084E090E09B838A8381E09FEF9D838C83E5
:105EA0008FEF90E09F838E8319861886188ECE011F
:105EB0000E940B838AE394E099838883D093D3066E
:105EC000C093D20610928E128091D2069091D30682
:105ED000DC01ED91FC910280F381E02D1995809118
:105EE000450F843658F4853608F084E664E6681B6E
:105EF0008091D2069091D3060E942C4E80913F0F44
:105F00008C50823000F56091400F7091410F84E019
:105F10000E9458816091420F7091430F84E00E946B
:105F20003D818091440FE091D206F091D306808F9D
:105F300080913F0F8D3039F48091440FE0917312BE
:105F4000F0917412808F8EE190E00E9499BAEC017A
:105F5000F090550FC090590FD0905A0FA090570F46
:105F6000B090580F84EF95E09983888383E090E0A8
:105F70009B838A8381E09FEF9D838C830FEF10E0EA
:105F80001F830E8319861886188ECE010E940B83FC
:105F90008EE294E099838883BA8EA98EDC8ECB8EB4
:105FA000FD8ED0938F13C0938E1360915B0F709111
:105FB0005C0F83E00E94588160915D0F70915E0FCD
:105FC00083E00E943D818091550FE0918E13F09106
:105FD0008F13808F8091550F0E94464880918E13B9
:105FE00090918F13DC01ED91FC910280F381E02D03
:105FF000199580915F0F882339F185E290E00E9426
:1060000099BAFC018091640F9091650F2091620F05
:106010003091630F4091600F5091610F68E070E024
:106020007383628315821482178306831186108618
:10603000108E62E274E071836083528F418F348FDF
:10604000238F968F858F22C085E290E00E9499BAB7
:10605000FC018091620F9091630F2091600F30914D
:10606000610F48E050E05383428315821482178306
:10607000068311861086108E42E254E051834083DD
:10608000328F218F948F838F168F058FF0934C065C
:10609000E0934B0680914B0690914C060E94027E45
:1060A00080919A128823F9F089E190E00E9499BAD0
:1060B000FC0188E090E093838283158214828FEF45
:1060C00093E0978386838FEF91E091878087108E8E
:1060D00086E494E091838083F0939912E093981280
:1060E000CF010E94247E80919D12882309F474C000
:1060F00089E190E00E9499BAFC0189E090E09383E5
:106100008283158214828FEF93E0978386838FEFCB
:1061100091E091878087108E86E494E0918380835C
:10612000F0939C12E0939B12CF01DF91CF911F91CE
:106130000F91FF90EF90DF90CF90BF90AF909F9026
:106140008F907F900C94247E2C3009F498CE8CE1B3
:1061500090E00E9499BAEC0184EF882E85E0982E99
:106160009982888294E0A92EB12CBB82AA82CC2489
:10617000C394DD24DA94DD82CC82EE24EA94F12CFF
:10618000FF82EE8219861886188ECE010E940B833C
:1061900008EE15E019830883D093D306C093D20686
:1061A0008CE190E00E9499BAEC0199828882BB82CE
:1061B000AA82DD82CC82FF82EE8219861886188E32
:1061C0000E940B8319830883D0937412C0937312B7
:1061D000CE010E94807D76CEDF91CF911F910F91ED
:1061E000FF90EF90DF90CF90BF90AF909F908F90F7
:1061F0007F9008952F923F924F925F926F927F927D
:106200008F929F92AF92BF92CF92DF92EF92FF92C6
:106210000F931F93CF93DF93CDB7DEB7C65AD10943
:106220000FB6F894DEBF0FBECDBFCDB6DEB6CC55EF
:10623000DF4F1882C45AD040CD55DF4F1882C35A61
:10624000D0408091D10D8A3709F447C0C0F4873718
:1062500009F4D9C238F48F3109F433C5863709F40B
:10626000E2C1F5C5883709F4DDC2893709F0EFC509
:106270000E941C850E9456892B013C0129C08E3743
:1062800009F42DC338F48B3709F4CAC18C3709F4EB
:10629000D8C2DDC5813809F405C5823809F4EBC4DC
:1062A000803809F0D4C563C40E945689DC01CB0153
:1062B00084199509A609B70980329340A105B10553
:1062C00008F00AC50E943C5A0E941C850E94D060BA
:1062D0000E945E85029741F7FFC40E945E85029787
:1062E00029F060E084E80E9490978BC18091160BA2
:1062F000823031F0833039F482E08093DF1103C0C3
:1063000081E08093341381E08093DB0D8E010C5586
:106310001F4F2BE0AE0144575F4F68E871E90E94C0
:106320000A970E943385893058F0015011092BE0FB
:10633000AE014F575F4F68E872E981E00E940A970B
:106340001092DA0D772473940E944985882309F40A
:106350003DC1198222961FAE22971091DA0D1111BC
:106360000EC0BE0164577F4FCE018F5B9F4F0E94CE
:10637000B7BCCC55DF4F0881C45AD04011C0113092
:1063800071F4BE016F577F4FCE018F5B9F4F0E940C
:10639000B7BCCD55DF4F0881C35AD04001C000E0E3
:1063A000ADB6BEB68091120BEDB7FEB722E0829F6C
:1063B000E019F10911240FB6F894FEBF0FBEEDBF2E
:1063C0008DB79EB701967C016CE276E0CE018356D4
:1063D0009F4F0E9409558091160B823089F08330BF
:1063E00061F1813009F0A1C04091120B50E0B7017A
:1063F00080910D1390910E130E94055D10E039C03D
:106400002091120B30E05FB7F89440E0842F90E0C9
:106410008217930774F4880F991FF701E80FF91F8B
:10642000DC01AD5EBC4E8D919C91918380834F5F6A
:10643000EDCF5FBF109233131CC02091120B30E0E0
:106440005FB7F89440E0842F90E08217930774F4CC
:10645000880F991FF701E80FF91FDC01AB51BE4E01
:106460008D919C91918380834F5FEDCF5FBF1092A0
:106470000A136DE270E0CE0183569F4F0E9438549C
:106480002091120B293048F0112321F0113021F412
:1064900018E004C028E001C020E010E0121758F511
:1064A000F701E10FF11DE10FF11D608171814AE0FB
:1064B000CE0189569F4FCB55DF4F2883C55AD04018
:1064C0000E94DE54BE0169567F4FCE0183569F4F16
:1064D0000E945F54CE0189569F4F0E94D954CE012D
:1064E00083569F4F0E94A04B1F5FCB55DF4F2881E3
:1064F000C55AD040D3CF40E450E0BE016F5F7F4F1C
:10650000CE0183569F4F0E94984BCF55DF4F188185
:10651000C15AD040CE0183569F4F0E94D9540FB626
:10652000F894BEBE0FBEADBE0BC0CE0183569F4FCA
:106530000E94D9540FB6F894BEBE0FBEADBE10E097
:10654000BE016F5F7F4FCE018F5B9F4F0E94B7BC34
:10655000010F10E0E1E4F0E0EC0FFD1FE00FF11F90
:106560001082BE016F5B7F4F8091B9139091BA1377
:106570000E946C55B801CE018F5B9F4F0E94ED6069
:10658000BC018091B9139091BA130E946C496AE0E2
:106590008091B9139091BA130E9441558091B9131B
:1065A0009091BA13DC01ED91FC910680F781E02D0A
:1065B00019950E943385893048F08091DA0D811158
:1065C00003C07092DA0D02C01092DA0D0E941C8591
:1065D0000E94D0600E94867E81110CDE8091D00DD9
:1065E00081110FC08091DB0D882359F08091DA1161
:1065F000811107C08091CE0D9091CF0D0A970CF4B8
:10660000A3CE8091160B823039F0833009F01FC47D
:1066100081E08093DF111BC481E08093341317C4A1
:106620001092DB0D4BC31091D40D8FEF810F85308D
:1066300028F060E089E80E94909709C4133079F04F
:1066400018F41230F9F004C0143079F0153099F0D4
:1066500040E6442E49E0542E612C712C19C0412C87
:106660003BE4532E612C712C13C0412C26E9522E91
:10667000612C712C0DC0412C92EC592E6624639430
:10668000712C06C080E8482E85E2582E612C712CB2
:1066900000E0E12EF12C5701BFE8AB0EB11C150153
:1066A000E89427F83324E6E9EE0EF11CE894E7F8C5
:1066B000FF24023091F018F4013051F004C003308F
:1066C00089F00430A1F040E659E060E070E013C0CA
:1066D00040E855E260E070E00EC040E05BE460E05E
:1066E00070E009C040E056E960E070E004C040E0BE
:1066F00052EC61E070E08FEB97E00E9464728FEBE8
:1067000097E00E945D530E9456894B015C01F2E3C1
:106710008F0E911CA11CB11C0E9490600E94568992
:10672000681579058A059B05B8F360E870E08FEB82
:1067300097E00E9476806FE070E08FEB97E00E9418
:106740007680612F8FEB97E00E941753B1018FEB9A
:1067500097E00E9476800E9456894B015C012AE0F6
:10676000820E911CA11CB11C0E9490600E9456894F
:10677000681579058A059B05B8F367E870E08FEB2B
:1067800097E00E9476806FE070E08FEB97E00E94C8
:106790007680612F8FEB97E00E941753B7018FEB44
:1067A00097E00E9476808FEB97E00E945D530E94F5
:1067B00056894B015C013EE5830E31E0931EA11C1E
:1067C000B11C0E9490600E945689681579058A055F
:1067D0009B05B8F30F5F053009F06BCFB301A20141
:1067E0008FEB97E00E9464724092D60F5092D70FC1
:1067F0006092D80F7092D90FB301A20186EB91E09D
:106800000E94D34B5BC283E090E00E9499BA2AE0D9
:10681000DC012C932FEB37E012963C932E931197CB
:106820006AE00CC083E090E00E9499BA2DE0FC0180
:1068300020832FEB37E0328321836DE00E94615C7F
:106840003DC24091D40D5091D50D0091D60D1091BF
:10685000D70D6091D20D7091D30DCE010196CB551D
:10686000DF4F4883C55AD040CA55DF4F5883C65AB8
:10687000D04025D7CB55DF4F4881C55AD040CA55A7
:10688000DF4F5881C65AD040892BE9F08D8187307F
:1068900050F4853080F48130B0F0642F8B819C817E
:1068A0000E94D7490DC0893070F4B8018B819C815A
:1068B0000E94D34B05C0BA018B819C810E947B480A
:1068C0000E940C9804C061E085E80E949097809136
:1068D000CD0D8111BCC281E08093CD0DB8C2B090C6
:1068E000D20DE090D30DC956DF4F1882C759D04062
:1068F0006CE276E0CE018F579F4F0E9409556B2DB9
:106900007E2DCE0184579F4FDAD6892B09F4C9C05A
:10691000C057DF4FE881C059D0404E2F50E0FA01F8
:106920003197E830F10508F0BCC08827E55AFE4FE2
:106930008F4F0C9485BAC257DF4F88819981CE580A
:10694000D0400E9449B823961FAE1EAE23972596CD
:106950001FAE1EAE259727961FAE1EAE27974AE0A4
:10696000BE016F5F7F4F90E03EC0C257DF4F88810E
:106970009981CE58D0400E9449B8682F880F770B74
:106980004AE00AC0C257DF4F88819981CE58D04073
:106990000E9456B84AE0BC01CE0101960E94DE5426
:1069A000BE016F5F7F4FCE018F579F4F0E94FF53F5
:1069B000CE01019663C0C257DF4F88819981CE58BE
:1069C000D0400E9456B823961FAE1EAE2397259640
:1069D0001FAE1EAE259727961FAE1EAE27974AE024
:1069E000BE016F5F7F4F0E94F7B635C0C257DF4FC1
:1069F00088819981CE58D0400E9451B823961FAE0D
:106A00001EAE239725961FAE1EAE259727961FAE66
:106A10001EAE27972AE0AE014F5F5F4F0E94C8B6B7
:106A20001AC0C257DF4F88819981CE58D0400E944A
:106A300051B823961FAE1EAE239725961FAE1EAEED
:106A4000259727961FAE1EAE27972AE0AE014F5F0F
:106A50005F4F0E94D6B6BE016F5F7F4FCE018F5B46
:106A60009F4F0E94B954BE016F5B7F4FCE018F577D
:106A70009F4F0E94FF53CE018F5B9F4F0E94D954BE
:106A80004BE050E0BE016F5B7F4FCE018F579F4FB1
:106A90000E94984BCB57DF4FF880C558D04011E08B
:106AA00002C0F12C10E0CE018F579F4F0E94D954A5
:106AB000112309F4BECD8E0109561F4F20E4AE010B
:106AC0004F5F5F4F68E87B2D8E2D0E940A97BE01B5
:106AD0006F5B7F4FCE0101960E94B7BCC956DF4F56
:106AE0008881C759D040F80E81E08F0DC956DF4F1D
:106AF0008883C759D040E1E0F0E0EC0FFD1FEF0DB7
:106B0000F11D9CE79083E1E0F0E0EC0FFD1FE80F42
:106B1000F11D1082BE016F5F7F4F8091B91390917C
:106B2000BA130E946C55C956DF4F6881C759D040CF
:106B300070E0CE0101960E94ED60BC018091B91316
:106B40009091BA130E946C496AE08091B9139091B8
:106B5000BA130E9441558091B9139091BA13DC0188
:106B6000ED91FC910680F781E02D199570C180911F
:106B7000D20D9091D30D8038910509F068C18E0136
:106B800004571F4F20E4AE014F5F5F4F68E870E885
:106B900080E00E940A976CEF75E0CE018F579F4FFF
:106BA0000E940955CE018F579F4F0E94A04BC4579A
:106BB000DF4F2881CC58D040CB57DF4F8881998157
:106BC000C558D040820F911DC457DF4F8883CC58E1
:106BD000D04022961FAE22974BE050E0BE016F5B83
:106BE0007F4FCE018F579F4F0E94754BBE016F5B49
:106BF0007F4FCE0101960E94B7BCC457DF4F8881FA
:106C0000CC58D040E1E0F0E0EC0FFD1FE80FF11DA3
:106C10001082BE016F5F7F4F8091B9139091BA13BC
:106C20000E946C55C457DF4F6881CC58D04070E04B
:106C3000CE0101960E94ED60BC018091B913909144
:106C4000BA130E946C496AE08091B9139091BA130B
:106C50000E9441558091B9139091BA13DC01ED91D6
:106C6000FC910680F781E02D1995CE018F579F4F3B
:106C70000E94D954ECC08091D20D9091D30D8238EE
:106C8000910509F0E4C08E0104571F4F20E4AE01C6
:106C90004F5F5F4F68E872E880E00E940A9766E104
:106CA00076E07BCF8091D20D9091D30D8138910504
:106CB00009F0CDC08091DB0D8111C9C00E940C98F4
:106CC000C6C08091D20D9091D30D4F9709F0BFC0EF
:106CD00081E08093D00DBBC00E945E85029719F0C1
:106CE00060E084E8A8CC8091150B811102C00E945D
:106CF000F1490E943385F82E6CE276E0CE0184578C
:106D00009F4F0E940955C956DF4F1882C759D0407E
:106D10008E0109561F4F20E4AE014F5F5F4F68E8B8
:106D200079E780E00E940A97CF57DF4F19821882D7
:106D3000C158D040CD57DF4F19821882C358D04078
:106D4000CB57DF4F19821882C558D0406F2D70E0A5
:106D500080E090E02AE0AE014F5B5F4F0E94C8B632
:106D6000BE016F5B7F4FCE018F579F4F0E94B9547A
:106D7000BE016F577F4FCE0184579F4F0E94FF5334
:106D8000CE018F579F4F0E94D9544BE050E0BE0177
:106D90006F5B7F4FCE0184579F4F0E94754BC0574A
:106DA000DF4F1881C059D040BE016F5B7F4FCE01CD
:106DB00001960E94B7BCC956DF4F8881C759D040A1
:106DC000810F91E0980FC956DF4F9883C759D04083
:106DD000E1E0F0E0EC0FFD1FE80FF11D8CE7808390
:106DE000E1E0F0E0EC0FFD1FE90FF11D1082BE01A4
:106DF0006F5F7F4F8091B9139091BA130E946C55C9
:106E0000C956DF4F6881C759D04070E0CE01019666
:106E10000E94ED60BC018091B9139091BA130E9459
:106E20006C496AE08091B9139091BA130E94415560
:106E30008091B9139091BA13DC01ED91FC91068019
:106E4000F781E02D1995CE0184579F4F11CF0FB6D2
:106E5000F894DEBE0FBECDBECA55DF4F0FB6F89414
:106E6000DEBF0FBECDBFDF91CF911F910F91FF907D
:106E7000EF90DF90CF90BF90AF909F908F907F90DA
:106E80006F905F904F903F902F900895FC01128279
:106E9000138214821582168217821286089580E06A
:106EA00008950F931F93CF938C016EE470E189EFE7
:106EB00098E00E944855D8011896ED91FC911997D9
:106EC0006081718189EF98E00E948445C1E0D8011A
:106ED0001A968C91C81710F569E470E189EF98E073
:106EE0000E9448556C2F89EF98E00E943F4866E465
:106EF00070E189EF98E00E944855F80190858185FE
:106F0000E92FF82FEC0FF11DEC0FF11D608171815D
:106F100089EF98E00E948445CF5FD9CFCF911F9130
:106F20000F910895CF93DF93CDB7DEB7A0970FB63B
:106F3000F894DEBF0FBECDBF80310CF080E02EE3B1
:106F400030E13A83298327E330E13C832B8329E234
:106F500030E13E832D832DE130E138872F8323E11B
:106F600030E13A87298729E030E13C872B8725E00B
:106F700030E13E872D872EEF3FE0388B2F8723EFC0
:106F80003FE03A8B298B26EE3FE03C8B2B8B2BEDA1
:106F90003FE03E8B2D8B2FEC3FE0388F2F8B2DEB7E
:106FA0003FE03A8F298F2CEA3FE03C8F2B8F27EA76
:106FB0003FE03E8F2D8F2AE93FE038A32F8FE82F47
:106FC000EE0FFF0BEC0FFD1F81819281A0960FB693
:106FD000F894DEBF0FBECDBFDF91CF910895AF9281
:106FE000BF92CF92DF92EF92FF920F931F93CF93B6
:106FF000DF9385EE9DE07EE1D72ED80ECC24C3949E
:1070000002E010E0C3E0D0E0E2E0BE2EEE24E39424
:10701000F12C8091E3119091E411DC01ED91FC9150
:107020000084F185E02D1995892B09F4ADC0A0905D
:1070300030018091E3119091E411DC01ED91FC911C
:107040000284F385E02D199596B3B39A20918400BC
:1070500030918500285A344E30938D0020938C0057
:107060002A2D2C7119F01092E0114BC093FB992737
:1070700090F9E091E011E11116C0992351F28032AC
:1070800041F6C092E0118093E50D80910813909134
:107090000913892B09F0BDCFF0920913E092081370
:1070A0001092E211B6CF9111DECFE13041F480347D
:1070B00009F0AFCFB092E0118093E60DE6CF91E0FA
:1070C0009E0F9093E011F0E0EB51F24F80839032ED
:1070D00009F09FCF1092E011E5EEFDE02FEF3FEFBA
:1070E0008191281B3109DE12FBCF4091030E809164
:1070F000040E90E0982F8827840F911D28173907D8
:1071000029F0D0930913C093081383CF80910813FB
:1071100090910913019739F48091E2118F5F809368
:10712000E211843020F0109309130093081380912A
:10713000E1118F5F8093E1119091DF11981708F5AD
:10714000C0920A1320E030E0F901EB51F24F428186
:10715000838190E0982F8827840F911DAC014F5EAA
:1071600052404B3D554028F4F901EB51FE4E9183BE
:1071700080832E5F3F4F2C31310531F71092E111A2
:1071800048CF10920A1345CFDF91CF911F910F91F5
:10719000FF90EF90DF90CF90BF90AF900895EF9267
:1071A000FF920F931F93CF93DF931092200E82E0F4
:1071B0008093210E68EE73E07093230E6093220E8D
:1071C00040ED57E05093250E4093240E2CED35E012
:1071D0003093270E2093260E8FE08093280E109276
:1071E000290E94E090932A0E70932C0E60932B0E30
:1071F00050932E0E40932D0E3093300E20932F0E71
:107200008093310E1092320E93E09093330E709370
:10721000350E6093340E5093370E4093360E3093F4
:10722000390E2093380E80933A0E10923B0E91E067
:1072300090933C0E70933E0E60933D0E5093400E23
:1072400040933F0E3093420E2093410E8093430EA5
:107250001092440EE5E4FEE0AEE4BEE080E008EE0D
:1072600013E060ED77E04CED55E031E022E095E091
:10727000980F9083128301837483638356834583BD
:10728000ED01229791E03883219628831C928F5F2D
:107290003A961A968C3059F71092BD0E9093BE0E06
:1072A0001092BF0E9093C00E8AE892E09093C20EA7
:1072B0008093C10E9093C40E8093C30E80E090E043
:1072C0009C01205E314FF901EB55FF4F1182108276
:1072D0003296108203968837910591F784E290E008
:1072E0009093C60E8093C50E81E08093C70E2CE06C
:1072F00030E03093C90E2093C80E94E09093CA0EEC
:1073000021E230E03093CC0E2093CB0E27E0209387
:10731000CD0E29E030E03093CF0E2093CE0E20E149
:107320002093D00E7AE070933D0F2BE020933E0F18
:1073300020933F0F48EE53E05093410F4093400F8E
:1073400020ED37E03093430F2093420F1092440F0B
:1073500064E66093450F6093460F5093480F409347
:10736000470F30934A0F2093490F10924B0F5093C1
:107370004D0F40934C0F30934F0F20934E0F1092B0
:10738000500F1092510F8093520F1092540F109281
:10739000530F8093550F8093560FE8ECF0E0F09375
:1073A000580FE093570FE0E2F3E0F0935A0FE093A9
:1073B000590F50935C0F40935B0F30935E0F2093F7
:1073C0005D0F80935F0FE9E5F0E0F093610FE093CC
:1073D000600FE0E8F0E0F093630FE093620FEFEFEF
:1073E000F0E0F093650FE093640FF093670FE09384
:1073F000660F8093680F9093690F10926A0F8093C5
:107400006B0F90936C0F10926D0F10926E0F809314
:107410006F0F1092700F1092710F8093720F109275
:10742000730F98E29093740F5093760F4093750FFB
:107430005093780F4093770F30937A0F2093790F02
:1074400080937B0F92E390937C0FE2E0E0937D0FBB
:1074500080937E0F60937F0FE6E4E093800F90931C
:10746000810F1092820F1092830F1092840F10924E
:10747000850F1092860F1092870FEAEFF0E0F093DD
:10748000890FE093880F10928A0F10928B0F6093F0
:107490008C0F61E460938D0F10928E0F90938F0F7D
:1074A0001092900F9093910FEEE5F1E0F093930F0F
:1074B000E093920F1092940FACEDB5E0B093960F5D
:1074C000A093950F00EA1FE01093980F0093970F79
:1074D00030939A0F2093990FC8E8D3E1D0939C0F73
:1074E000C0939B0F68EBE62E6BE0F62EF0929E0F9A
:1074F000E0929D0FE0E4FFE1F093A00FE0939F0F77
:107500001092A10F1092A20F1092A30F69E1609345
:10751000A40F8093A50F8093A60F8093A70F50937D
:10752000A90F4093A80F3093AB0F2093AA0FF092AE
:10753000AD0FE092AC0F1093AF0F0093AE0FD0934E
:10754000B10FC093B00F20E737E13093B30F209312
:10755000B20F1092B40F1092B50F1092B60F909315
:10756000B70F9093B80F9093B90F1092BA0F109273
:10757000BB0F1092BC0F8093BD0F1092CD0F1092D5
:10758000BE0F99E09093BF0F1092C00F1092C10FE1
:107590001092C20F1092C30FB093C50FA093C40FE7
:1075A000F093C70FE093C60F8093C80F7093C90F75
:1075B0001092CA0F21E030E03093CC0F2093CB0F14
:1075C00040E052EC61E070E04093CE0F5093CF0F5B
:1075D0006093D00F7093D10F4093D20F5093D30F7D
:1075E0006093D40F7093D50F40E056E960E070E0EF
:1075F0004093D60F5093D70F6093D80F7093D90F45
:107600004093DA0F5093DB0F6093DC0F7093DD0F24
:107610001092DE0F20E039E13093E00F2093DF0F6E
:107620001092E10F9EE19093E20F1092E30F2EE192
:1076300030E03093E50F2093E40F3093E70F209371
:10764000E60F3093E90F2093E80F9093EA0F9093A1
:10765000EB0F8093EC0F8093ED0F1092EE0F909351
:10766000EF0F8093F00F9CE09093F10F8093F20F57
:1076700083E891EFA0E0B0E08093F30F9093F40FD4
:10768000A093F50FB093F60F00E21EE0C0E0D0E04B
:10769000CE010E9449B8F80161918F01861719F057
:1076A000CE010E945BB82196C73DF1E0DF0781F76C
:1076B000DF91CF911F910F91FF90EF9008954F921E
:1076C0005F926F927F928F929F92AF92BF92CF9272
:1076D000DF92EF92FF92CF93DF93EB01A091E30D46
:1076E000B091E40D9D012F5F3F4F45E0429F200187
:1076F000439F500C1124052C000C66087708812C40
:10770000912C54012434E1E03E07ECF44EE654E9B8
:1077100061E0772775016401C40CD51CE61CF71CD9
:107720004C0D5D1D6E1D7F1D6BBFFA01479156917B
:1077300065E0860E911CA11CB11CC417D50729F168
:107740002F5F3F4FDFCF25E0822E912CA12CB12C53
:1077500021E030E0A217B30708F44CC04EE654E92C
:1077600061E07727480D591D6A1D7B1D6BBFFA012B
:1077700047915691F5E08F0E911CA11CB11CC417C6
:10778000D50719F02F5F3F4FE5CF4EE654E961E092
:107790007727E5E0E29F6001E39FD00C11240D2CD8
:1077A000000CEE08FF084E5F5F4F6F4F7F4F4C0D90
:1077B0005D1D6E1D7F1D6BBFFA0147915691FC0147
:1077C000538342834EE654E961E077274C5F5F4F75
:1077D0006F4F7F4FC40ED51EE61EF71EEBBEF6019F
:1077E000C790FC01C4823093E40D2093E30DC901DE
:1077F000019606C01092E40D1092E30D80E090E037
:10780000DF91CF91FF90EF90DF90CF90BF90AF903E
:107810009F908F907F906F905F904F9008950F93FF
:107820001F938091DE0D81111EC00E945689009128
:10783000DF0D1091E00D2091E10D3091E20DAB01D3
:10784000BC01401B510B620B730B8091DC0D9091BE
:10785000DD0DA0E0B0E084179507A607B70718F480
:1078600081E08093DE0D1F910F9108958091DC0DD2
:107870009091DD0D892B89F08091DE0D882381F0B8
:107880000E9456896093DF0D7093E00D8093E10DA7
:107890009093E20D1092DE0D089581E08093DE0D4D
:1078A00008951F920F920FB60F9211242F938F936A
:1078B0009F93109295001092940080910A0B8F5F15
:1078C00080930A0B90919613891784F010920A0BFB
:1078D00020910C0B8091A1139091A213820F911D06
:1078E00027FD9A959093A2138093A1138091090B81
:1078F0008F5F8093090B9091A613891784F01092E3
:10790000090B20910B0B8091A4139091A513820F6A
:10791000911D27FD9A959093A5138093A4139F9191
:107920008F912F910F900FBE0F901F9018958091FF
:10793000080B811104C08091070B882321F08091EE
:107940007100826003C0809171008D7F809371000F
:107950000895CF93DF93EC01198618861F861E8643
:10796000198A188A1B8A1A8A0E94C2441EA61D867A
:10797000DF91CF910895CF93DF93EC011F861E8690
:10798000198A188A1B8A1A8AFDD7198618861C86B6
:10799000DF91CF910895FC018385882311F061E088
:1079A00001C060E082850C94C058FC018385882367
:1079B00011F060E001C061E082850C94C0580F9323
:1079C0001F93CF93DF93CDB7DEB78C01D4DFF801DF
:1079D000148A85E1FE013896D801559601900D92E2
:1079E0008A95E1F7F80185899689938B828B8D8D35
:1079F0008B3008F08AE090E0F801918B808BC80111
:107A0000D4DFC801BFD781E0F8018487DF91CF912F
:107A10001F910F910895CF92DF92EF92FF920F93F3
:107A20001F93CF93DF93CDB7DEB765970FB6F8946A
:107A3000DEBF0FBECDBF8C01FC0185858823E1F040
:107A400082899389892B09F441C10E945689F801E2
:107A5000C080D180E280F380AB01BC014C195D098C
:107A60006E097F0982899389A0E0B0E084179507A9
:107A7000A607B70718F12AC1F80180859185892BDF
:107A800009F48FC00E945689F801C480D580E68031
:107A9000F780AB01BC014C195D096E097F09808537
:107AA0009185A0E0B0E084179507A607B70708F016
:107AB00078C0C80170DFC8015EDFB4C0F8018685F8
:107AC00097850196978786876089718986179707BA
:107AD00068F580E090E00E9424B79B01AC016BED5B
:107AE0007FE089E490E40E942BB9F80122A533A538
:107AF00044A555A50E94C7B8F80162A773A784A73B
:107B000095A70E94C8B920E030E04FEF52E40E94F0
:107B100085B720E030E04FEF52E40E94C7B80E94E2
:107B200093B9F80182850E942B596CC0F8018585B4
:107B3000823019F4C8012FDF75C0F80186A58823AB
:107B400009F470C0C80105DF82E390E09A8389835D
:107B500088E290E09C838B838EE690E09E838D8309
:107B600084EF91E098878F831D8A84E08F938DB78F
:107B70009EB745970FB6F8949EBF0FBE8DBFADB7A9
:107B8000BEB7119685E1FE01319601900D928A955E
:107B9000E1F7C80114DF0FB6F894DEBF0FBECDBF0A
:107BA00095C0F80182899389892B09F48FC00E94BE
:107BB0005689F801C080D180E280F380AB01BC011E
:107BC0004C195D096E097F0982899389A0E0B0E0B4
:107BD00084179507A607B70708F078C0F8018685CF
:107BE0009785019697878687208931898217930721
:107BF00008F04DC080FF26C0C801CDDEF8018489A1
:107C0000882319F1C80165960FB6F894DEBF0FBE40
:107C1000CDBFDF91CF911F910F91FF90EF90DF903B
:107C2000CF90B0C6C80165960FB6F894DEBF0FBE00
:107C3000CDBFDF91CF911F910F91FF90EF90DF901B
:107C4000CF9087CEC801B1DED9CF868597858B309E
:107C5000910590F0C8019FDEC80165960FB6F894B3
:107C6000DEBF0FBECDBFDF91CF911F910F91FF906F
:107C7000EF90DF90CF907FCE880F991FF801E80F2B
:107C8000F91F85899689F801938B828BBBCFF80108
:107C900081A5882349F085899689938B828B1786E5
:107CA0001686C80182DEAECFF80186A5882391F240
:107CB00016A682E08587C8015EDE84E690E0F801C2
:107CC000918B808B87A590A9938B828B65960FB63D
:107CD000F894DEBF0FBECDBFDF91CF911F910F9102
:107CE000FF90EF90DF90CF900895CF93DF93EC015A
:107CF0008C85882321F0CE014EDECE013CDE8D85C1
:107D0000882311F0CE0125DECE01DF91CF9143CE45
:107D10008091110E9091120E91609093120E8093AB
:107D2000110E08958091110E9091120E806890931B
:107D3000120E8093110E08958091110E9091120EE3
:107D400080619093120E8093110E0895FC01828140
:107D5000882371F08381882359F013828091110E5A
:107D60009091120E24E082279093120E8093110EB0
:107D70000895FC018281882371F0838181110BC0F9
:107D800081E083838091110E9091120E8460909314
:107D9000120E8093110E0895FC018481882371F0E6
:107DA0008581882359F015828091110E9091120ED1
:107DB00028E082279093120E8093110E0895FC0103
:107DC0008481882371F0858181110BC081E08583D6
:107DD0008091110E9091120E88609093120E8093F4
:107DE000110E08958091110E9091120E20E28227BB
:107DF0009093120E8093110E08958091110E909120
:107E0000120E80629093120E8093110E0895DC0181
:107E1000ED91FC910680F781E02D60E070E019940F
:107E200077FF03C07195619571096F3F710519F076
:107E300014F06FEF70E08091110E9091120E8C7B18
:107E400091709093120E8093110E8091110E90916B
:107E5000120E6F30710514F480641FC06733710512
:107E600014F481641AC06F3571051CF4816490614B
:107E700014C0673871051CF4816490630EC06F3ABA
:107E800071051CF48164906408C0673D71051CF4A1
:107E90008164906502C0816490669093120E809315
:107EA000110E089580E094E09093120E8093110ECD
:107EB00008958091110E9091120E92609093120E7F
:107EC0008093110E8091110E9091120E8064909308
:107ED000120E8093110E089508950895089508953F
:107EE00008950895089508950895089580E00895E7
:107EF000089508950895089508950895089508959A
:107F00000895089508950895089508950895089589
:107F1000089508950895089580E0089508950895B6
:107F2000FC0164830895FC0162830895FC011382BF
:107F3000148215821682178210861186089508957C
:107F400008950895FC0183810895FC0165830895D7
:107F5000FC0164830895FC0160870895FC01668339
:107F60000895FC018281089581E08093090E6CEDF3
:107F700075E00C9473816CED75E080E00C94738176
:107F8000FC01128213821482158261E086E10E9454
:107F9000EF5861E086E10E94C058E2E7F0E080819E
:107FA000816080831092120E1092110E0895FF923C
:107FB0000F931F93CF93DF938C01C62FF42ED22FF4
:107FC0006AED70E0DC011A968D919C911B970E94DE
:107FD0007680F80182859385DC01ED91FC9101901A
:107FE000F081E02D6C2F1995F80182859385DC01D5
:107FF000ED91FC910190F081E02D6F2D1995F80124
:1080000082859385DC01ED91FC910190F081E02D5A
:108010006D2F1995EC2FF0E0BF0166527F4F6F0D69
:10802000711D6D0F711D6F777727F801828593851C
:10803000DF91CF911F910F91FF900C94768020E0FB
:1080400040E0B5CF65E4FBCF68E4F9CFCF93DF9391
:10805000FC012381222321F0EC0161E4F0DF1B828B
:10806000DF91CF910895CF93DF93FC0123812111FC
:1080700005C0EC0160E4E3DF81E08B83DF91CF9109
:10808000089563E5DCCFFC012581222311F060E532
:10809000D6CF0895FC012481222311F06CE3CFCFC9
:1080A0000895FC012085222331F02185222319F037
:1080B00011866BE3C4CF0895FC012085222339F09B
:1080C0002185211104C021E021876AE3B8CF0895FA
:1080D000FC012681222331F02781222319F0178207
:1080E00069E3ADCF0895FC012681222339F0278171
:1080F000211104C021E0278368E3A1CF089567E33D
:108100009ECF6AE49CCF69E49ACF66E398CF65E39B
:1081100096CF6EE494CF64E392CF63E390CF62E3B3
:108120008ECF61E38CCF60E38ACF6FE288CF6DE2C0
:1081300086CF6CE284CF242F462F6CE438CF77FFB4
:1081400003C071956195710920E0462F6EE22FCF33
:10815000462F20E067E42BCF462F20E066E427CFB0
:10816000262F64E424CFCF92DF92FF920F931F93C8
:10817000CF93DF938C01F62E443F81E0580738F00F
:10818000413187E2580728F040E157E202C044EF4E
:1081900051E0243F81E0380738F0E90121313742CE
:1081A00028F0C0E1D7E202C0C4EFD1E0CA01845F89
:1081B000914022E3C22ED12CB6010E945EBA462F16
:1081C0002F2D62E4C801F3DECE01845F9140B60139
:1081D0000E945EBA462F2F2D63E4C801DF91CF9134
:1081E0001F910F91FF90DF90CF90E1CE242F462F6B
:1081F00062E5DDCE242F462F61E5D9CE262F40E063
:108200006FE3D5CE262F40E06EE3D1CE262F40E09F
:108210006DE3CDCE462F20E06FE4C9CE462F20E09F
:108220006DE4C5CEFC016283611104C020E040E032
:108230006BE4BDCE089577FF03C071956195710918
:1082400020E0462F6BE4B3CE4F925F926F927F9205
:108250008F929F92AF92BF92CF92DF92EF92FF9256
:108260000F931F93CF93DF936C01A4ECCA1AADEF69
:10827000DA0AD601ED91FC917E970CF05DC0FC010D
:10828000E858FF4F812C912CA191B191AB2B21F497
:108290002115310549F450C0BFEF8B1A9B0AAEE19E
:1082A0008A16910489F748C0EC015401AA0CBB1C42
:1082B000AA0CBB1CAC0EBD1EF501EC54FF4F408355
:1082C0005183628373837401EE0CFF1CEC0EFD1E60
:1082D000F701E858FF4F31832083EC54FF4F11839F
:1082E0000083BE01680D791DFB01EC55FE4F81E056
:1082F00080830E945689F501608371838283938312
:10830000C65CDD4F88819981F701E250FE4F918371
:108310008083D6012D913C9111972F5F3F4F2D9374
:108320003C939C012F5F3F4F1216130614F021E07F
:1083300030E03983288302C08FEF9FEFDF91CF9128
:108340001F910F91FF90EF90DF90CF90BF90AF9073
:108350009F908F907F906F905F904F9008950F93B4
:108360001F93CF93DF93EC017093451260934412F7
:1083700040934B1281E090E00E9499BA8C010E94D8
:108380000B831093140E0093130E91E09093090E3B
:1083900090932C121092080E1092070E10922F122A
:1083A00010922E121092301210922D121092060E70
:1083B00024EF31E0309337122093361228EB3BE064
:1083C000309339122093381220E233E030933E127A
:1083D00020933D122CEA3DE03093401220933F124F
:1083E00028E037E0309347122093461224E931E128
:1083F0003093491220934812109233121092321285
:108400001092311210923A121092411210924A12A6
:108410001092050E109235121092341210923C12E6
:1084200010923B1210924312109242129883998339
:108430009A83DF91CF911F910F9108951F920F9210
:108440000FB60F9211240BB60F922F933F934F93B9
:108450005F936F937F938F939F93AF93BF93EF93AC
:10846000FF938091100E8F5F8093100E90910F0EEE
:10847000891708F401C11092100E80910E0E90E041
:108480008730910508F0F8C0FC018827ED59FE4FB0
:108490008F4F0C9485BA60E086E10E94C05880E45A
:1084A00080930F0E81E048C061E086E10E94C058D1
:1084B00088E080930F0E36C060E086E10E94C058CD
:1084C00080910C0E90910D0E97FF05C088E180936E
:1084D0000F0E84E031C088E080930F0E83E02CC043
:1084E00061E086E10E94C05888E180930F0E809180
:1084F0000B0E8F5F80930B0E803150F010920B0E9D
:1085000085E01AC061E086E10E94C05888E0EDCFA6
:1085100080910C0E90910D0E880F991F90930D0E67
:1085200080930C0E82E008C060E086E10E94C05893
:1085300088E080930F0E86E080930E0E9DC061E070
:1085400086E10E94C05880EC80930F0E8091110E3E
:108550009091120E90930D0E80930C0E8091110E3F
:108560009091120E91FF1DC080910A0E8823B1F0E8
:108570008091110E9091120E22E092279093120E8C
:108580008093110E8091110E9091120E8064909341
:10859000120E8093110E10920A0E03C081E0809398
:1085A0000A0E8091110E9091120E92FF0EC08091D2
:1085B0000A0E882339F01092120E1092110E1092AA
:1085C0000A0E03C081E080930A0E8091110E9091F3
:1085D000120E84FF14C080910A0E882369F08091E6
:1085E000110E9091120E20E182279093120E80932B
:1085F000110E10920A0E03C081E080930A0E809142
:10860000110E9091120E87FF13C080910A0E8823DD
:1086100061F08091110E9091120E80589093120E7D
:108620008093110E10920A0E03C081E080930A0E0F
:108630008091110E9091120E90FF14C080910A0E3D
:10864000882369F08091110E9091120E21E09227FB
:108650009093120E8093110E10920A0E03C081E0C7
:1086600080930A0E8091110E9091120E90930D0E30
:1086700080930C0E10920E0EFF91EF91BF91AF916F
:108680009F918F917F916F915F914F913F912F912A
:108690000F900BBE0F900FBE0F901F901895DC012E
:1086A000A250BE4F20E030E04D915D914617570734
:1086B00039F4280F391FF901EC55FE4F80810895D8
:1086C0002F5F3F4F2E31310579F780E00895CF932A
:1086D000DF93EC01C45CDD4FA881B981109709F4E8
:1086E00042C0FC01E250FE4F20E030E04191519148
:1086F0004617570799F5A901440F551F480F591FF1
:10870000FA01E858FF4F60817181672B61F1118296
:108710001082FC01E20FF31FEC55FE4F1082FA01AC
:10872000EE53FE4F11821082235D3F4F220F331F05
:10873000220F331FFC01E20FF31F108211821282FD
:108740001382FA01E859FE4F11821082EA56FF4F58
:10875000118210821197B983A88305C02F5F3F4F04
:108760002E31310519F6DF91CF9108950F931F93A4
:1087700001E010E069DD1F910F9108951092090E3C
:1087800024EB3FE344EF51E060E070E0809144125D
:1087900090914512EBDF9093080E8093070E089599
:1087A00080914B1281110AC08091090E882331F00B
:1087B00060ED77E081E00E947381E0CF08950F9330
:1087C0001F9300E010E040DD1F910F9108952F925C
:1087D0003F924F925F926F927F928F929F92AF9251
:1087E000BF92CF92DF92EF92FF920F931F93CF939E
:1087F000DF9300D000D0CDB7DEB78C010E94568940
:1088000098012E533E4F3C832B831E830D83D8014A
:10881000AC55BE4FBA83A9831801B2E02B1ABEEF44
:108820003B0AF901AA24A394B12C32E0832E912CA7
:10883000118210829F012A543140D9012D913C911F
:10884000232B09F44DC0AD81BE812D913D914D91F9
:108850005C9113977D01B4EBEB0EF11CD701CD9029
:10886000DD90ED90FC902B013C01421A530A640A02
:10887000750A4C145D046E047F0490F1C20ED31E81
:10888000E41EF51EAD81BE81CD92DD92ED92FC928B
:108890001397A981BA812C91222311F19F012659A6
:1088A0003109D9012D913C912115310519F4B1827D
:1088B000A08216C07F01BAE5EB1AF108D7014D91ED
:1088C0005C911197421753075CF4B182A0824F5F0D
:1088D0005F4F4D935C934217530714F0918280824F
:1088E00032962D813E812C5F3F4F3E832D83A9819F
:1088F000BA811196BA83A983E215F30509F098CFDE
:10890000EB81FC8181919191FC83EB838130910516
:1089100099F00297C9F4EB81FC81EC54F14001908D
:10892000F081E02D1995AB81BC81DA966D917C9137
:10893000DB97C801CCDE08C0EB81FC81EC54F14030
:108940000190F081E02D19952B813C812215330592
:10895000B9F626960FB6F894DEBF0FBECDBFDF91F5
:10896000CF911F910F91FF90EF90DF90CF90BF902C
:10897000AF909F908F907F906F905F904F903F90BF
:108980002F900895CF93DF93EC010E94568968835E
:1089900079838A839B83CE01DF91CF910895EF92F3
:1089A000FF921F93CF93DF93CDB7DEB765970FB6D6
:1089B000F894DEBF0FBECDBF182F7B0180E19AE097
:1089C0000E94A93C81E080933E0A84E690E0909367
:1089D000210A8093200A84E6E816F10418F484E65C
:1089E000E82EF12CC70164E670E00E945EBA709335
:1089F000400A60933F0A7093230A6093220A1093FF
:108A00001D0A8FEF810F823010F41230D1F080E117
:108A10009AE00E94CB3C80911B0A882329F083ECCA
:108A200095EFA8ECBFE304C084EB98ECA6E9B0E4B2
:108A300080933A0A90933B0AA0933C0AB0933D0A74
:108A400055C080911B0A882329F084EB98ECA6E995
:108A5000B0E404C083EC95EFA8ECBFE380933A0A3E
:108A600090933B0AA0933C0AB0933D0A80E19AE0C0
:108A70000E94D53C80913E0A8823C1F110921D0AC4
:108A80008EE690E09A83898388E290E09C838B83D2
:108A90008CE390E09E838D831D8A83E08F938DB756
:108AA0009EB745970FB6F8949EBF0FBE8DBFADB76A
:108AB000BEB7119685E1FE01319601900D928A951F
:108AC000E1F780E19AE00E94DF3C0FB6F894DEBF48
:108AD0000FBECDBF65960FB6F894DEBF0FBECDBFFB
:108AE000DF91CF911F91FF90EF90089580E19AE080
:108AF00065960FB6F894DEBF0FBECDBFDF91CF9164
:108B00001F91FF90EF903ECF0F931F93CF93DF9372
:108B1000EC01AB0160E070E02AE00E9481558C011D
:108B2000CE010E94A656800F911FDF91CF911F9119
:108B30000F9108958F929F92AF92BF92CF92DF9242
:108B4000EF92FF920F931F93CF93DF931F921F9289
:108B5000CDB7DEB7082E000C990BAA0BBB0BFC019E
:108B60003197EF30F10508F064C28827E659FE4FCF
:108B70008F4F0C9485BA84E08093FF098AE080933C
:108B8000000A86E28093020A81E08093050A8093BE
:108B9000060A8093040A40EC50E120E030E0809126
:108BA000FF0990E0281739070CF08CC1FA01859174
:108BB0009491A0E0B0E0880F991FAA1FBB1FF90194
:108BC000EE0FFF1FEE0FFF1FEA56F64F80839183D3
:108BD000A283B3832F5F3F4F4E5F5F4FE0CF84E0B0
:108BE0008093FF098AE08093000A86E28093020A5C
:108BF00081E08093050A8093060A82E08093040A4C
:108C000048EB50E120E030E08091FF0990E0281728
:108C100039070CF057C1FA0185919491A0E0B0E0BA
:108C2000880F991FAA1FBB1FF901EE0FFF1FEE0F40
:108C3000FF1FEA56F64F80839183A283B3832F5F91
:108C40003F4F4E5F5F4FE0CF84E08093000A85E2A4
:108C50008093020A81E08093050A88E08093060AE7
:108C600083E08093040A80E090E0FC01E055FF4E31
:108C7000E491DC01A95FB54FEC9301968830910532
:108C8000A1F70E94464F1EC188E08093FF0986E04D
:108C90008093000A86E28093020A81E08093050AAD
:108CA0008093060A84E08093040A40EA50E120E0C1
:108CB00030E08091FF0990E0281739070CF002C1DD
:108CC000FA0185919491A0E0B0E0880F991FAA1F46
:108CD000BB1FF901EE0FFF1FEE0FFF1FEA56F64F05
:108CE00080839183A283B3832F5F3F4F4E5F5F4F9B
:108CF000E0CF88E08093FF0981E08093000A97E24B
:108D00009093020A8093050A8093060A85E0809377
:108D1000040A40E950E120E030E08091FF0990E052
:108D2000281739070CF0CEC0FA0185919491A0E084
:108D3000B0E0880F991FAA1FBB1FF901EE0FFF1F9C
:108D4000EE0FFF1FEA56F64F80839183A283B38311
:108D50002F5F3F4F4E5F5F4FE0CF82E18093FF096F
:108D600081E08093000A97E29093020A8093050ABB
:108D70008093060A8FE08093040A4CE650E120E0DD
:108D800030E08091FF0990E0281739070CF09AC075
:108D9000FA0185919491A0E0B0E0880F991FAA1F75
:108DA000BB1FF901EE0FFF1FEE0FFF1FEA56F64F34
:108DB00080839183A283B3832F5F3F4F4E5F5F4FCA
:108DC000E0CFE0916A0AF0916B0A749780819181FB
:108DD00040E550E060E070E08659954F0E949D505C
:108DE00028C182E18093FF0985E08093000A82E236
:108DF0008093020A81E08093050A8093060A87E047
:108E00008093040A80E993E3A0E0B0E080939609A0
:108E100090939709A0939809B0939909F2E08F2E47
:108E2000912C01E010E080E090E0A0E0BBE54CE494
:108E300054E060E070E024EEC22E2CE0D22EE12C53
:108E4000F12C9801220F331F220F331F5401AA0C5B
:108E5000BB1CAA0CBB1C2A56364FF901B7FF0DC02C
:108E6000C082D182E282F38295012A56364FF901FF
:108E700040835183628373830CC040835183628338
:108E8000738395012A56364FF901C082D182E2825E
:108E9000F382880F991FAA1FBB1F0E5F1F4FF2E0BE
:108EA0008F0E911C22E18216910459F688E79FEFFC
:108EB000A0E0B0E08093DA099093DB09A093DC098D
:108EC000B093DD090E94B54FB4C0CE010196CAD758
:108ED00023E040E150E060E070E071C084E0809306
:108EE000FF0982E38093000A86E28093020A81E010
:108EF0008093050A8093060A8AE08093040A44E678
:108F000050E120E030E08091FF0990E02817390718
:108F1000CCF6FA0185919491A0E0B0E0880F991FFA
:108F2000AA1FBB1FF901EE0FFF1FEE0FFF1FEA562E
:108F3000F64F80839183A283B3832F5F3F4F4E5FB1
:108F40005F4FE1CF84E08093FF0980E28093000AC5
:108F500086E28093020A81E08093050A8093060AE4
:108F60008BE08093040A4CE550E120E030E08091F2
:108F7000FF0990E0281739070CF0A4CFFA0185917A
:108F80009491A0E0B0E0880F991FAA1FBB1FF901C0
:108F9000EE0FFF1FEE0FFF1FEA56F64F80839183FF
:108FA000A283B3832F5F3F4F4E5F5F4FE0CFCE0171
:108FB000019658D721E040E154E060E070E0CE0136
:108FC00001960E94115035C084E08093FF0983E030
:108FD0008093000A86E28093020A81E08093050A6A
:108FE0008093060A8DE08093040A44E550E120E076
:108FF00030E08091FF0990E0281739070CF062CF2C
:10900000FA0185919491A0E0B0E0880F991FAA1F02
:10901000BB1FF901EE0FFF1FEE0FFF1FEA56F64FC1
:1090200080839183A283B3832F5F3F4F4E5F5F4F57
:10903000E0CF0F900F90DF91CF911F910F91FF9094
:10904000EF90DF90CF90BF90AF909F908F9008955A
:109050000F931F93CF93DF93EC01462F50E060E016
:1090600070E02AE00E9481558C01CE010E94A65634
:10907000800F911FDF91CF911F910F910895462F7F
:1090800050E060E070E02AE00C9481552FB7F8942E
:10909000882381F080915A1190915B11909369110E
:1090A0008093681180916A1190916B1118161906BE
:1090B000ACF00FC080915C1190915D11909369119B
:1090C0008093681180916A1190916B11181619069E
:1090D0002CF480916A1190916B1107C080916A11F4
:1090E00090916B1191958195910990936B1180935B
:1090F0006A112FBF0895AF92BF92CF92DF92EF9285
:10910000FF920F931F93CF93DF931F921F92CDB7C0
:10911000DEB78C017A836983CE0101966C01580118
:1091200092E0A90EB11CE12CF12CC8010E9449B8B3
:10913000F60161916F01861731F0C8010E945BB89A
:10914000FFEFEF1AFF0A0F5F1F4F0A151B0569F7A4
:1091500081E0EF2809F480E00F900F90DF91CF912C
:109160001F910F91FF90EF90DF90CF90BF90AF9045
:109170000895EF92FF920F931F93CF93DF931F9267
:109180001F92CDB7DEB78C017B018AEA8A8341E06A
:1091900050E0BE016E5F7F4FC8010E94F45BD701B3
:1091A000ED91FC910680F781E02DC701199582E8C9
:1091B000898341E050E0BE016F5F7F4FC8010E948C
:1091C000F45B0F900F90DF91CF911F910F91FF9063
:1091D000EF900895CF92DF92EF92FF920F931F933B
:1091E0000E9456896B017C016093D6117093D71150
:1091F0008093D8119093D9118091170B0E949858A1
:109200008093D5119091190B992329F091E0811148
:1092100090E09093D5118091210B9091220BA09119
:10922000230BB091240B97018601081B190B2A0B05
:109230003B0B4091250B5091260B6091270B7091B1
:10924000280B90911A0B041715072607370760F4AF
:10925000C0921D0BD0921E0BE0921F0BF092200BC0
:1092600010921C0B892F1EC090931B0B8091D5115F
:1092700080931A0BC0921D0BD0921E0BE0921F0B15
:10928000F092200B891761F0C092210BD092220B33
:10929000E092230BF092240B91E090931C0B02C000
:1092A00010921C0B1F910F91FF90EF90DF90CF90C9
:1092B00008950F931F93CF93DF93EC012AE00E9450
:1092C00081558C01CE010E94A656800F911FDF911F
:1092D000CF911F910F910895CF92DF92EF92FF925D
:1092E0000F931F93CF93DF936B01770FEE08FF0867
:1092F000F7FE1BC0EC016DE20E9441558C01442732
:109300005527BA014C195D096E097F092AE0CE0183
:109310000E948155800F911FDF91CF911F910F9176
:10932000FF90EF90DF90CF9008952AE0B701A6015B
:10933000DF91CF911F910F91FF90EF90DF90CF9031
:109340000C948155CF92DF92EF92FF920F931F936F
:10935000CF93DF938C016B01770FEE08FF08F7FEC8
:1093600012C06DE20E944155EC0144275527BA0115
:109370004C195D096E097F092AE0C8010E948155D8
:10938000C80FD91F06C02AE0B701A6010E94815567
:10939000EC01C8010E94A6568C0F9D1FDF91CF9152
:1093A0001F910F91FF90EF90DF90CF9008950F9352
:1093B0001F93CF93DF931F92CDB7DEB78C016983E4
:1093C0000E9449B86981861729F0C8010E945BB8DC
:1093D00081E001C080E00F90DF91CF911F910F914C
:1093E0000895CF930E94338584E090E09093140B0E
:1093F0008093130B81E29EE09093F9108093F81014
:109400001092F3108091120B9091210E891718F091
:1094100091E09093F0102AE23EE030930311209304
:1094200002111092FD1090912A0E891718F091E008
:109430009093FA1023E33EE030930D1120930C112A
:10944000109207119091330E891718F091E09093C4
:1094500004112CE33EE03093171120931611109263
:10946000111190913C0E891718F091E090930E1114
:109470001092110B20E030E0F901EB53F14F4081E5
:109480005181415051094432510520F491E09093AB
:10949000110B05C02D5F3F4F2837310569F79091BB
:1094A000110B992341F12091340E3091350E2D5D31
:1094B0003F4F3093350E2093340E2091360E30916D
:1094C000370E235231093093370E2093360E2091F8
:1094D0003D0E30913E0E2D5D3F4F30933E0E20935A
:1094E0003D0E20913F0E3091400E235231093093B2
:1094F000400E20933F0E90913E0F9F3049F4909183
:109500003F0F9F3029F41092EF101092EE1008C018
:109510002091920F3091930F3093EF102093EE1023
:1095200022E130E03093EC102093EB102091130BEC
:109530003091140BA5E4BEE0E7E9F0E141E0B68329
:10954000A5839C91992329F0891718F040832F5FF8
:109550003F4F1A96379690E1EB3EF90781F730932B
:10956000140B2093130B2131310534F080E190E08E
:109570009093140B8093130B0E941E8584EF90E14F
:109580009093FA0F8093F90F8091F8109091F91051
:109590009093F80F8093F70F81EF90E19093FC0F79
:1095A0008093FB0F82EF90E19093FE0F8093FD0F6D
:1095B00080EF90E1909300108093FF0F8EEF90E189
:1095C00090930410809303108091021190910311E5
:1095D00090930210809301108BEF90E1909306100E
:1095E000809305108CEF90E1909308108093071002
:1095F0008AEF90E190930A108093091088E091E13E
:1096000090930E1080930D1080910C1190910D117C
:1096100090930C1080930B1085E091E190931010C3
:1096200080930F1086E091E19093121080931110B7
:1096300084E091E1909314108093131082E191E102
:109640009093181080931710809116119091171114
:1096500090931610809315108FE091E190931A105B
:109660008093191080E191E190931C1080931B105E
:109670008EE091E190931E1080931D102091130BAA
:109680003091140B2450310960E07AE0C7E0462F96
:1096900050E04217530724F5CA010496789FF00161
:1096A000799FF00D1124E950F04FC49FC001C59F70
:1096B000900D1124AC0147565F4E53834283DC0169
:1096C000A956BF4E15964D915C91169751834083D4
:1096D00088569F4E95838483B187A0876F5FD7CFCD
:1096E00081E08093150BCF9108950F931F93CF9333
:1096F000DF93FC01248135812115310519F4FB012B
:10970000108211C0EA0121972C173D0708F4E901E6
:109710008B01FC0160817181AE01C8010E94C9BC4E
:10972000C00FD11F1882DF91CF911F910F91089523
:109730004115510521F06115710509F0D6CF089545
:10974000EF92FF920F931F93CF93DF931F921F927D
:10975000CDB7DEB78C018CE789831A82F801E480EB
:10976000F580FFEFEF1AFF0AB701C8010E943854D5
:10977000882381F0F8012081318184819581BE01A7
:109780006F5F7F4F820F931F0E94C2BCF801F5826A
:10979000E48281E00F900F90DF91CF911F910F91A4
:1097A000FF90EF900895AF92BF92CF92DF92EF9229
:1097B000FF920F931F93CF93DF9300D01F92CDB7EB
:1097C000DEB78C0149835A836B837C83CE0101967B
:1097D0006C01580194E0A90EB11CE12CF12CC801D8
:1097E0000E9449B8F60161916F01861731F0C801F6
:1097F0000E945BB8FFEFEF1AFF0A0F5F1F4F0A15B9
:109800001B0569F781E0EF2809F480E00F900F90C5
:109810000F900F90DF91CF911F910F91FF90EF90DC
:10982000DF90CF90BF90AF900895CF92DF92EF92EC
:10983000FF920F931F93CF93DF93EC010091150ECE
:10984000E0E0F0E020E030E0A90110E0CE17DF0713
:109850001CF1309711F40D32E1F0DF01AB5EB14F36
:10986000FC9080ED8F0D8A30A8F4AAE0B0E00E9451
:1098700085B82F2DFF0C330B205331096901330FAD
:10988000EE08FF089B01AC012C0D3D1D4E1D5F1D18
:1098900001C011E03196DACFCA01B901112339F0C4
:1098A00090958095709561957F4F8F4F9F4FDF9179
:1098B000CF911F910F91FF90EF90DF90CF9008957F
:1098C00080911A0B811105C081E090911C0B9111C0
:1098D00001C080E00895CF93DF932091410A309139
:1098E000420AE9012697A881B981AF5BB54F12966C
:1098F0001C92082E000C990BAA0BBB0BFC01319794
:10990000EF30F10508F06EC18827E758FE4F8F4F02
:109910000C9485BAF9013A97808191818F5B954FBC
:109920000E94C5AE882309F462C1E091410AF0911A
:10993000420A36970190F081E02DEF5BF54F81E010
:10994000EDC0F9013C97808191818F5B954F0E941A
:10995000F4AD882309F44BC1E091410AF091420A29
:1099600036970190F081E02DEF5BF54F82E0D6C095
:10997000F9013E97808191818F5B954F0E94A2B53E
:10998000882309F434C1E091410AF091420A3697E4
:109990000190F081E02DEF5BF54F83E0BFC0F9014E
:1099A0007097808191818F5B954F0E9428B58823A5
:1099B00009F41DC1E091410AF091420A36970190E5
:1099C000F081E02DEF5BF54F84E0A8C0F9017297BC
:1099D000808191818F5B954F0E94E3B4882309F4C5
:1099E00006C1E091410AF091420A36970190F08158
:1099F000E02DEF5BF54F85E091C0F9017497808110
:109A000091818F5B954F0E949EB4882309F4EFC02B
:109A1000E091410AF091420A36970190F081E02DE1
:109A2000EF5BF54F8FE07AC0F901769780819181E5
:109A30008F5B954F0E9425B4882309F4D8C0E0912C
:109A4000410AF091420A36970190F081E02DEF5BD8
:109A5000F54F86E063C0F9017897808191818F5B33
:109A6000954F0E949FB3882309F4C1C0E091410A39
:109A7000F091420A36970190F081E02DEF5BF54FAF
:109A800087E04CC0F9017A97808191818F5B954F77
:109A90000E9491B3882309F4AAC0E091410AF09191
:109AA000420A36970190F081E02DEF5BF54F88E098
:109AB00035C0F901B297808191818F5B954F0E94EB
:109AC000CEB0882309F493C0E091410AF091420A94
:109AD00036970190F081E02DEF5BF54F8381948103
:109AE000A581B6814097A105B10509F080C08FC05E
:109AF000F9017C97808191818F5B954F0E94CEB256
:109B0000882309F474C0E091410AF091420A369723
:109B10000190F081E02DEF5BF54F8AE0828367C012
:109B2000F9017E97808191818F5B954F0E940BB2E6
:109B3000882309F45CC0E091410AF091420A36970B
:109B40000190F081E02DEF5BF54F8BE0E7CFF9015D
:109B5000B297808191818F5B954F0E94CEB0882310
:109B600009F445C0E091410AF091420A369701900C
:109B7000F081E02DEF5BF54F83819481A581B68163
:109B800080319440A105B10591F543C0F901B0972A
:109B9000808191818F5B954F0E9447B1882339F175
:109BA000E091410AF091420A36970190F081E02D50
:109BB000EF5BF54F8DE0B2CFF901B29780819181D3
:109BC0008F5B954F0E94CEB0882389F0E091410AC7
:109BD000F091420A36970190F081E02DEF5BF54F4E
:109BE0008EE09CCFE881F981EF5BF54F1282E09126
:109BF000410AF091420A36970190F081E02DEF5B27
:109C0000F54F81E09281911106C080E004C089E0A7
:109C100085CF8CE083CFDF91CF910895089508958B
:109C2000089508951092FA0A08950C947D80CF93B8
:109C3000DF93CCE8DAE081E090E09A8389831092A8
:109C4000FA0A0E94F9886C837D838E839F83E49A4D
:109C5000EC9ADF91CF910895EF92FF920F931F93AB
:109C6000CF93DF93EC016623E1F0262F653608F0F1
:109C700024E60A891B89E888F988D801AE19BF094A
:109C800030E00E9493BA28EC30E040E050E00E94BF
:109C900095B8E20EF31EFB86EA86021B130B1D87A6
:109CA0000C87DF91CF911F910F91FF90EF90089556
:109CB000CF93DF93CDB7DEB7A2970FB6F894DEBF90
:109CC0000FBECDBF80310CF080E127E831E13A834F
:109CD00029832FE731E13C832B8327E731E13E8362
:109CE0002D832FE631E138872F8327E631E13A874C
:109CF00029872FE531E13C872B8727E531E13E8736
:109D00002D872FE431E1388B2F8721E431E13A8B25
:109D1000298B2FE231E13C8B2B8B22E131E13E8B11
:109D20002D8B2DEF30E1388F2F8B23EF30E13A8FE1
:109D3000298F29EE30E13C8F2B8F2CED30E13E8FC7
:109D40002D8F20ED30E138A32F8F28EC30E13AA39E
:109D500029A3E82FEE0FFF0BEC0FFD1F81819281ED
:109D6000A2960FB6F894DEBF0FBECDBFDF91CF91A4
:109D700008958F929F92AF92BF92CF92DF92EF920F
:109D8000FF920F931F93DC0118968D919C91199768
:109D90001E96CD90DC901F976817790709F456C07E
:109DA0005896FC9058974C01092E000CAA08BB0845
:109DB0008B01072E000C220B330B861797073CF400
:109DC0001696ED91FC911797FF2039F015C0149667
:109DD000ED91FC911597FF2079F00D2C000CEE0809
:109DE000FF08A9019801281939094A095B091C963D
:109DF0006D917C911D970EC00D2C000CEE08FF0894
:109E0000A9019801281939094A095B091A966D9127
:109E10007C911B97CB01770FAA0BBB0BBC01CD012B
:109E20006C197D098E099F090E944FBA8F01FF0F9F
:109E3000220B330BA9019801281939094A095B093A
:109E40000E9469B8C20ED31EE41EF51EC6011F9102
:109E50000F91FF90EF90DF90CF90BF90AF909F90C9
:109E60008F900895CF93DF93EC0161E089E00E9429
:109E7000EF5860E089E00E94C0581092030A86E320
:109E800095E099838883DF91CF910895CF92DF92F7
:109E9000EF92FF928091040A833009F061C08091B3
:109EA000050A8130D1F488EE93E0A0E0B0E0809321
:109EB000960990939709A0939809B093990980E720
:109EC00097E1A0E0B0E080939A0990939B09A0935A
:109ED0009C09B0939D0932E001C030E0E091050A91
:109EE000F0E0EA5FF54F2081A0E1A30F48EE53E0D8
:109EF00060E070E088EBC82E8BE0D82EE12CF12CCE
:109F0000832F90E0FC01EE0FFF1FEE0FFF1FEA56BC
:109F1000F64F27FF10C0C082D182E282F382880F01
:109F2000991F880F991FFC01E656F64F4083518315
:109F3000628373830FC04083518362837383880F6E
:109F4000991F880F991FFC01E656F64FC082D182F7
:109F5000E282F3823E5F220F3A13D2CF3093FF09A1
:109F6000FF90EF90DF90CF900895CF93DF93809193
:109F7000030A811153C01092010A1092FE09C1E038
:109F8000C093030AD091020A61E089E00E94EF5871
:109F900060E089E00E94C0582D2F30E040E050E0A2
:109FA00060E47FE180E090E00E9469B8C093B00077
:109FB00089E08093B1002093B3008BEA289F212D84
:109FC000112426952093B40080916F008B7F80939D
:109FD0006F008091B00080628093B0002091840077
:109FE00030918500E091FE0981E08E0F8093FE099B
:109FF00084E0E89FF0011124EA56F64F80819181B8
:10A00000A281B381820F931F90938B0080938A006B
:10A01000B29A80916F00846080936F00DF91CF913E
:10A0200008954F925F926F927F928F929F92AF921C
:10A03000BF92CF92DF92EF92FF928AE18093FF0965
:10A040002093000A88E28093020A81E08093050A47
:10A050008093060A8EE08093040A80EC92E1A0E0EF
:10A06000B0E08093960990939709A0939809B093D4
:10A07000990980EB94E0A0E0B0E080939A09909376
:10A080009B09A0939C09B0939D09A4E1440F551F1F
:10A09000661F771FAA95D1F722E030E0B0EBCB2EF8
:10A0A000B4E0DB2EE12CF12C80E6482E89E0582E1E
:10A0B000612C712C90E4892E9CE9992EA12CB12C55
:10A0C000C901880F991F880F991FFC01EA56F64FA6
:10A0D00077FF05C0408251826282738204C0C082D1
:10A0E000D182E282F382C9010196880F991F880FFD
:10A0F000991FFC01EA56F64F283129F0C082D1821F
:10A10000E282F38204C080829182A282B382440FF1
:10A11000551F661F771F2E5F3F4F2A31310581F68D
:10A12000FF90EF90DF90CF90BF90AF909F908F9077
:10A130007F906F905F904F9018CF8F929F92AF92C9
:10A14000BF92CF92DF92EF92FF9282E18093FF095C
:10A1500086E08093000A96E29093020A91E0909341
:10A16000050A9093060A8093040A88ED90E4A0E023
:10A17000B0E08093960990939709A0939809B093C3
:10A1800099098CE19CE0A0E0B0E080939A0990935B
:10A190009B09A0939C09B0939D09742F66275527AE
:10A1A000442722E030E0ACE1CA2EACE0DA2EE12C0C
:10A1B000F12CB8E38B2EB8E19B2EA12CB12CC90158
:10A1C000880F991F880F991FFC01EA56F64F77FFF9
:10A1D00005C080829182A282B38204C0C082D182F3
:10A1E000E282F382F901EE0FFF1FEE0FFF1FE6562A
:10A1F000F64FC082D182E282F382440F551F661F60
:10A20000771F2E5F3F4F22313105C9F68CE199E867
:10A21000A0E0B0E08093DA099093DB09A093DC0919
:10A22000B093DD09FF90EF90DF90CF90BF90AF909B
:10A230009F908F909ACE1F920F920FB60F9211247B
:10A240000BB60F922F933F934F935F936F937F9330
:10A250008F939F93AF93BF93EF93FF939091FE09DA
:10A260008091FF09981316C01092FE098091050A8B
:10A270008F5F8093050A9091050A8091060A8917DD
:10A2800040F481E08093050A8091010A8F5F8093FA
:10A29000010AFCDD9091010A8091000A98130DC01B
:10A2A0008091B0008F7D8093B00080916F008B7F94
:10A2B00080936F001092030A27C08091B00085FF41
:10A2C00004C08091B0008F7D03C08091B000806297
:10A2D0008093B0002091840030918500E091FE09C8
:10A2E00081E08E0F8093FE0984E0E89FF001112445
:10A2F000EA56F64F80819181A281B381820F931F2C
:10A3000090938B0080938A00FF91EF91BF91AF9162
:10A310009F918F917F916F915F914F913F912F917D
:10A320000F900BBE0F900FBE0F901F9018951F92AD
:10A330000F920FB60F9211240BB60F921F932F930B
:10A340003F934F935F936F937F938F939F93AF93BD
:10A35000BF93EF93FF93CF93DF9300D01F92CDB7BE
:10A36000DEB780918C0AE4D611E0892B09F010E069
:10A370000E94F98869837A838B839C8389819A817F
:10A38000AB81BC814091900A5091910A6091920AF0
:10A390007091930A841B950BA60BB70B20918D0A25
:10A3A00030918E0A2430310509F44CC02530310536
:10A3B00021F021303105E9F414C020918F0A2223C5
:10A3C00039F02091FA0A20FF02C0289A01C028988B
:10A3D000112379F0813E2EE29207A105B10548F0E4
:10A3E0002BC0112379F125E030E030938E0A2093C1
:10A3F0008D0A20918D0A30918E0A2530310511F594
:10A40000E091FA0AF0E0EE0FFF1FEC56F54F918352
:10A41000808389819A81AB81BC818093900A9093DB
:10A42000910AA093920AB093930A8091FA0A8F5FDF
:10A430008093FA0A833330F084E090E090938E0AA0
:10A4400080938D0A0F900F900F900F90DF91CF9116
:10A45000FF91EF91BF91AF919F918F917F916F91FC
:10A460005F914F913F912F911F910F900BBE0F90D5
:10A470000FBE0F901F901895CF93DF93EC01809142
:10A480008C0A62E0ACD6E881F9810190F081E02D80
:10A49000CE01DF91CF9119940895CF92DF92EF9280
:10A4A000FF920F931F93CF93DF936C017A018B017F
:10A4B000C0E0D0E0CE15DF0589F0D8016D918D01A7
:10A4C000D601ED91FC910190F081E02DC601199526
:10A4D000892B11F47E0102C02196ECCFC701DF91D8
:10A4E000CF911F910F91FF90EF90DF90CF90089543
:10A4F000FC01A089B1898C91A689B78982FD0FC022
:10A500009C91818D8F5F8F73228D821749F0218DF1
:10A51000DF01A20FB11D5D969C93818F08958C91F0
:10A520000895089580E090E00895FC01538D448DD6
:10A53000252F30E0842F90E0821B930B541710F0EE
:10A54000CF96089501970895FC01918D828D9817FB
:10A5500061F0828DDF01A80FB11D5D968C91928D07
:10A560009F5F9F73928F90E008958FEF9FEF089504
:10A57000FC01918D828D981731F0828DE80FF11DCD
:10A58000858D90E008958FEF9FEF0895FC01918DE8
:10A59000228D892F90E0805C9F4F821B91098F73E1
:10A5A0009927089582E297E0F1DF21E0892B09F4F1
:10A5B00020E0822F08958FEB97E0E8DF21E0892BE0
:10A5C00009F420E0822F08958CE598E0DFDF21E098
:10A5D000892B09F420E0822F089589EF98E0D6DFD7
:10A5E00021E0892B09F420E0822F0895FC01848D5D
:10A5F000DF01A80FB11DA35ABF4F2C91848D90E0AD
:10A6000001968F739927848FA689B7892C93A08987
:10A61000B1898C9180648C93938D848D981306C03E
:10A620000288F389E02D80818F7D80830895EF92E9
:10A63000FF920F931F93CF93DF93EC0181E0888FFC
:10A640009B8D8C8D981305C0E889F989808185FDE3
:10A6500023C0F62E0B8D10E00F5F1F4F0F731127D5
:10A66000E02E8C8DE8120BC00FB607FCFACFE889FC
:10A67000F989808185FFF5CFCE01B8DFF2CF8B8DD0
:10A68000FE01E80FF11DE35AFF4FF0820B8FEA89BC
:10A69000FB898081806207C0EE89FF896083E88939
:10A6A000F98980818064808381E090E0DF91CF919F
:10A6B0001F910F91FF90EF900895CF93DF93EC01DE
:10A6C000888D8823C1F0EA89FB89808185FD05C0DA
:10A6D000A889B9898C9186FD0EC00FB607FCF5CF0D
:10A6E000808185FFF2CFA889B9898C9185FFEDCF54
:10A6F000CE017CDFE8CFDF91CF91089580E090E03C
:10A70000892B19F06ADF811116C080E090E0892B57
:10A7100019F05ADF811112C080E090E0892B19F006
:10A720004ADF81110EC080E090E0892B79F03ADF9A
:10A7300081110AC008950E940000E7CF0E94000026
:10A74000EBCF0E940000EFCF0C940000089590E042
:10A75000FC013197E231F10508F04EC08827E85737
:10A76000FE4F8F4F0C9485BA809180008F7703C085
:10A77000809180008F7D809380000895809180007B
:10A78000877FF9CF84B58F7702C084B58F7D84BD74
:10A7900008958091B0008F7703C08091B0008F7DC5
:10A7A0008093B0000895809190008F7707C08091CA
:10A7B00090008F7D03C080919000877F80939000F0
:10A7C00008958091A0008F7707C08091A0008F7DB1
:10A7D00003C08091A000877F8093A000089580919E
:10A7E00020018F7707C0809120018F7D03C0809169
:10A7F0002001877F8093200108950E94AABC0F93B7
:10A800001F93CF93DF938C01EB01FC018081918139
:10A810000097B1F0688179816115710579F0428105
:10A8200053812C813D814217530740F00E94C2BCE6
:10A830008C819D81F8019583848313C00E942EBB77
:10A8400088819981F801918380838A819B81938398
:10A8500082838C819D8195838483198218821B82D7
:10A860001A821D821C82DF91CF911F910F91089552
:10A870000F931F93CF93DF93EC0188819981009709
:10A8800029F02A813B812617370788F48B016F5FF7
:10A890007F4F0E94C6BB009761F0998388831B831A
:10A8A0000A832C813D81232B11F4FC01108281E06D
:10A8B00001C080E0DF91CF911F910F910895EF9239
:10A8C000FF920F931F93CF93DF93FB012481358178
:10A8D000E080F180FC0104811581E114F10411F4A0
:10A8E00080E016C02115310591F0EC01020F131F15
:10A8F000B801BEDF8823A1F3288139818C819D8135
:10A90000B701820F931F0E94C2BC1D830C8381E09C
:10A91000DF91CF911F910F91FF90EF900895EF92EB
:10A92000FF920F931F93CF93DF93EC017B018A017A
:10A93000BA019EDF2881398181110DC021153105B1
:10A9400019F0C9010E942EBB198218821D821C8237
:10A950001B821A8206C01D830C83B701C9010E94A5
:10A96000C2BCCE01DF91CF911F910F91FF90EF906C
:10A970000895CF93DF93EC016115710551F0FB0150
:10A9800001900020E9F73197AF01461B570BC7DF55
:10A990000CC088819981009711F00E942EBB19820A
:10A9A00018821D821C821B821A82CE01DF91CF91F8
:10A9B0000895FC01808191810C942EBB0F931F930D
:10A9C000CF93DF93CDB7DEB762970FB6F894DEBFB3
:10A9D0000FBECDBF8C01CB01F80111821082138212
:10A9E00012821582148250E0BE016F5F7F4F0E9479
:10A9F000B4B6BE016F5F7F4FC801BBDF62960FB672
:10AA0000F894DEBF0FBECDBFDF91CF911F910F91A4
:10AA10000895FC0111821082138212821582148221
:10AA20006115710549F0FB0101900020E9F73197AC
:10AA3000AF01461B570B73CF0895CF93DF9300D020
:10AA40001F92CDB7DEB7611571058105910579F0CB
:10AA50009B01AC0169833A834B835C830E94A8B657
:10AA600029813A814B815C810E9469B803C060E012
:10AA700070E0CB010F900F900F900F90DF91CF916E
:10AA80000895DC01ED91FC910190F081E02D199485
:10AA9000EF92FF920F931F93CF93DF938C017B0173
:10AAA000C0E0D0E0F701EC0FFD1F6491662361F078
:10AAB000D801ED91FC910190F081E02DC80119952C
:10AAC000892B11F02196EECFCE01DF91CF911F910E
:10AAD0000F91FF90EF9008956115710579F0FB01DA
:10AAE00001900020E9F73197AF01461B570BDC01BD
:10AAF000ED91FC910280F381E02D199480E090E0CB
:10AB000008954F925F926F927F92EF92FF920F9310
:10AB10001F93CF93DF93CDB7DEB7A1970FB6F8940D
:10AB2000DEBF0FBECDBF7C01FA01CB0119A22230DE
:10AB300008F42AE08E010F5D1F4F422E512C612C2C
:10AB4000712CBF01A30192010E9495B8F901CA01BD
:10AB5000015011096A3014F4605D01C0695CD801CC
:10AB60006C93232B242B252B61F7B801C701B4DF8D
:10AB7000A1960FB6F894DEBF0FBECDBFDF91CF9187
:10AB80001F910F91FF90EF907F906F905F904F908B
:10AB900008954F925F926F927F928F929F92AF92A1
:10ABA000BF92CF92DF92EF92FF92CF93DF93EC01AF
:10ABB0006A017B01B22E9A01AB01C701B6010E9466
:10ABC000CEB9882319F06EE176E027C0260137015F
:10ABD000E89477F82FEF3FEF4FE75FE7C301B2014B
:10ABE0000E94CEB981110DC02FEF3FEF4FE75FE715
:10ABF000C301B2010E9420B718161CF462E276E08D
:10AC00000CC02FEF3FEF4FE75FE4C701B6010E9492
:10AC1000C4B9181694F466E276E0CE01DF91CF91C4
:10AC2000FF90EF90DF90CF90BF90AF909F908F906C
:10AC30007F906F905F904F904FCF2FEF3FEF4FE798
:10AC40005FECC701B6010E9420B787FDE4CF20E08A
:10AC500030E0A901C701B6010E9420B787FF09C0F3
:10AC60006DE2CE010EDF4C01F7FAF094F7F8F094A4
:10AC700002C0812C912CA12C60E070E080E09FE369
:10AC8000AB1441F020E030E040E251E40E942BB9E7
:10AC9000A394F6CF9B01AC01C701B6010E94C7B8CF
:10ACA0002B013C010E9498B96B017C010E9424B7E2
:10ACB0009B01AC01C301B2010E94C6B82B013C014B
:10ACC0002AE0B701A601CE011CDF7C01E80CF91CCB
:10ACD000BB2029F06EE2CE01D4DEE80EF91EDB2C9B
:10ACE000DD2021F120E030E040E251E4C301B20177
:10ACF0000E9485B72B013C010E9498B94B01A12C01
:10AD0000B12C2AE0B501A401CE01FBDEE80EF91E4C
:10AD1000C501B4010E9424B79B01AC01C301B2017B
:10AD20000E94C6B82B013C01DA94DACFC701DF914B
:10AD3000CF91FF90EF90DF90CF90BF90AF909F901A
:10AD40008F907F906F905F904F9008956AE276E0C9
:10AD5000C3CE0F931F93CF93DF93EC01BDDE8C0125
:10AD6000CE01F4DF800F911FDF91CF911F910F91E2
:10AD700008950F931F93CF93DF93EC0189DE8C012D
:10AD8000CE01E4DF800F911FDF91CF911F910F91D2
:10AD900008951F920F920FB60F9211240BB60F92C7
:10ADA0002F933F934F935F936F937F938F939F93D3
:10ADB000AF93BF93EF93FF9382E297E017DCFF918D
:10ADC000EF91BF91AF919F918F917F916F915F9123
:10ADD0004F913F912F910F900BBE0F900FBE0F9090
:10ADE0001F9018951F920F920FB60F9211240BB659
:10ADF0000F922F933F934F935F936F937F938F9314
:10AE00009F93AF93BF93EF93FF9382E297E070DB42
:10AE1000FF91EF91BF91AF919F918F917F916F9132
:10AE20005F914F913F912F910F900BBE0F900FBEEE
:10AE30000F901F9018951F920F920FB60F9211242A
:10AE40000BB60F922F933F934F935F936F937F9324
:10AE50008F939F93AF93BF93EF93FF938FEB97E005
:10AE6000C5DBFF91EF91BF91AF919F918F917F9142
:10AE70006F915F914F913F912F910F900BBE0F906B
:10AE80000FBE0F901F9018951F920F920FB60F9242
:10AE900011240BB60F922F933F934F935F936F93B1
:10AEA0007F938F939F93AF93BF93EF93FF938FEB1A
:10AEB00097E01EDBFF91EF91BF91AF919F918F9132
:10AEC0007F916F915F914F913F912F910F900BBEAA
:10AED0000F900FBE0F901F9018951F920F920FB6F4
:10AEE0000F9211240BB60F922F933F934F935F93C2
:10AEF0006F937F938F939F93AF93BF93EF93FF9342
:10AF00008CE598E073DBFF91EF91BF91AF919F913A
:10AF10008F917F916F915F914F913F912F910F9002
:10AF20000BBE0F900FBE0F901F9018951F920F929F
:10AF30000FB60F9211240BB60F922F933F934F939E
:10AF40005F936F937F938F939F93AF93BF93EF9391
:10AF5000FF938CE598E0CCDAFF91EF91BF91AF9130
:10AF60009F918F917F916F915F914F913F912F9121
:10AF70000F900BBE0F900FBE0F901F9018951F9251
:10AF80000F920FB60F9211240BB60F922F933F938F
:10AF90004F935F936F937F938F939F93AF93BF93E1
:10AFA000EF93FF9389EF98E021DBFF91EF91BF9141
:10AFB000AF919F918F917F916F915F914F913F9151
:10AFC0002F910F900BBE0F900FBE0F901F901895F2
:10AFD0001F920F920FB60F9211240BB60F922F9360
:10AFE0003F934F935F936F937F938F939F93AF9311
:10AFF000BF93EF93FF9389EF98E07ADAFF91EF9197
:10B00000BF91AF919F918F917F916F915F914F9180
:10B010003F912F910F900BBE0F900FBE0F901F907E
:10B020001895CF93DF93EC01E881F9810680F781D1
:10B03000E02D1995EA89FB8980818F7E8083EA89DA
:10B04000FB898081877F8083EA89FB8980818F7774
:10B050008083EA89FB8980818F7D80838A8D898FB7
:10B06000DF91CF910895CF92DF92EF92FF921F93DD
:10B07000CF93DF93EC016A017B01122FE889F989F4
:10B0800082E080834115514E61057105B1F060E0A9
:10B0900079E08DE390E0A70196010E9495B8DA016E
:10B0A000C9010197A109B109B695A795979587950B
:10B0B000AC01411580E15807A8F0E889F9891082B0
:10B0C00060E874E88EE190E0A70196010E9495B8CF
:10B0D000BA01A90141505109610971097695679535
:10B0E00057954795EC85FD855083EE85FF85408318
:10B0F000188EEC89FD891083EA89FB898081806143
:10B100008083EA89FB89808188608083EA89FB8962
:10B11000808180688083EA89FB8980818F7D80833C
:10B12000DF91CF911F91FF90EF90DF90CF90089526
:10B13000CF93DF93282F30E0F901E759FD4E84913A
:10B14000F901ED5DFD4ED491F901E352FE4EC4913B
:10B15000CC2389F08111FBDAEC2FF0E0EE0FFF1F1A
:10B16000ED53FE4EA591B491EC91ED2381E090E07A
:10B1700021F480E002C080E090E0DF91CF9108955B
:10B180001F93CF93DF93282F30E0F901E759FD4E4D
:10B190008491F901ED5DFD4ED491F901E352FE4E2B
:10B1A000C491CC23C1F0162F8111D1DAEC2FF0E03D
:10B1B000EE0FFF1FE755FE4EA591B4918FB7F8949F
:10B1C000111105C09C91ED2FE095E92302C0EC918F
:10B1D000ED2BEC938FBFDF91CF911F910895CF930B
:10B1E000DF9390E0FC01ED5DFD4E2491FC01E35204
:10B1F000FE4E8491882361F190E0880F991FFC0135
:10B20000E157FE4EC591D491FC01E755FE4EA59144
:10B21000B491611109C09FB7F89488812095822369
:10B220008883EC912E230BC0623061F49FB7F894B1
:10B230003881822F809583238883EC912E2B2C9349
:10B240009FBF06C08FB7F894E8812E2B28838FBF4D
:10B25000DF91CF9108951F93CF93DF93182FEB01C8
:10B2600061E0BDDF209711F460E004C0CF3FD1055D
:10B2700031F461E0812FDF91CF911F9181CFE12FD8
:10B28000F0E0E759FD4EE4914E2F50E0FA0131977E
:10B29000E231F10508F09DC08827E656FE4F8F4F3A
:10B2A0000C9485BA84B5806884BDC7BD97C084B549
:10B2B000806284BDC8BD92C0809180008068809308
:10B2C0008000D0938900C093880088C0809180005E
:10B2D000806280938000D0938B00C0938A007EC0F0
:10B2E00080918000886080938000D0938D00C0930F
:10B2F0008C0074C08091B00080688093B000C093CF
:10B30000B3006CC08091B00080628093B000C093A5
:10B31000B40064C080919000806880939000D093C6
:10B320009900C09398005AC08091900080628093E9
:10B330009000D0939B00C0939A0050C080919000E1
:10B34000886080939000D0939D00C0939C0046C07D
:10B350008091A00080688093A0008091A0008F7BE6
:10B360008093A000D093A900C093A80037C080911B
:10B37000A00080628093A000D093AB00C093AA008D
:10B380002DC08091A00088608093A000D093AD0074
:10B39000C093AC0023C0809120018068809320017D
:10B3A000D0932901C093280119C0809120018062A7
:10B3B00080932001D0932B01C0932A010FC080916C
:10B3C0002001886080932001D0932D01C0932C012F
:10B3D00005C0C038D1050CF04CCF46CFDF91CF91DE
:10B3E0001F910895863308F0865390917B00282F93
:10B3F0002870977F922B90937B0087708064809356
:10B400007C0080917A00806480937A0080917A0039
:10B4100086FDFCCF809178002091790090E0922BFE
:10B42000089581E080930D0B089581E080930E0BC9
:10B43000089581E080930F0B0895CF93DF93C0911F
:10B440000112D091021260912A1270912B12CE013A
:10B450000E944F4381110DC02BED30E844EF51E0C5
:10B4600060E070E0CE010E94B64390932B1280936F
:10B470002A12DF91CF910895CF9380912512C09128
:10B480000A028111FEC0C23009F44FC0C33009F472
:10B490009BC0C13009F025C180910F0B811121C1E2
:10B4A00081E090E00E9499BA90930E1380930D135F
:10B4B00062E083E094DE109224121092071310923F
:10B4C000061310920B1380E090E0FC01EE0FFF1FBB
:10B4D000EE5EFD4E11821082019688309105A9F72B
:10B4E000109223121092221280916A008C60809335
:10B4F0006A00ED9A8FB7F89420918400309185000E
:10B5000030931112209310128FBF29E13AE54AEFD0
:10B5100050E060E070E080910112909102120E9470
:10B52000B64381E080932512DCC080910E0B81111F
:10B53000D8C081E090E00E9499BA90931013809354
:10B540000F13809104018E7F809304018091050187
:10B5500081608093050182E297E090933A13809393
:10B5600039132EE240EA56E861E070E07CDD80911C
:10B5700065008B7F809365001092350189E0809390
:10B5800034018EE2809332018CEF8093300180E9A8
:10B5900080933101109238131092371310923613A2
:10B5A0001092351310923313E3E1F3E18CED95E043
:10B5B0008193919323E1E333F207D1F7C1E0C09384
:10B5C000341325E13AE550C080910D0B811189C0FB
:10B5D00081E090E00E9499BA909312138093111326
:10B5E000809104018E7F8093040180910501816028
:10B5F0008093050182E297E09093E4118093E31138
:10B6000026E040E052EC61E070E02DDD80916500C5
:10B610008B7F809365001092350180E18093340127
:10B6200086E0809332018EEF8093300180E9809331
:10B63000310110920913109208131092E211109226
:10B64000E11110920A13E5EEF1E18CED95E08193A2
:10B65000919322E1E130F207D1F71092E011C1E0BD
:10B66000C093DF1121E13AE54AEF50E060E070E07D
:10B6700080910112909102120E94B643C09325124C
:10B6800030C0C23069F0C330D1F0C13051F5809183
:10B690000F0B811126C080910613909107131DC0D6
:10B6A00080910E0B81111DC080910F13909110138A
:10B6B0000E94018480913713909138130EC08091BD
:10B6C0000D0B81110EC080911113909112130E94E5
:10B6D000EF378091081390910913029711F4C093EA
:10B6E000160B80910A028230A1F1833009F453C015
:10B6F000813009F072C080910F0B882309F46DC06E
:10B70000ED98E59A1092241210920C1310920713E0
:10B710001092061310920B1380E090E0FC01EE0FE4
:10B72000FF1FEE5EFD4E118210820196883091055A
:10B73000A9F7109223121092221280910D1390916A
:10B740000E130E942EBB1092251210920E0B82E057
:10B7500042C080910E0B882309F43FC080913913B9
:10B7600090913A135EDC809131018F7780933101A3
:10B77000809131018F7E8093310110923001809150
:10B780000F13909110130E942EBB1092251210924D
:10B790000D0B83E020C080910D0B8823F1F0809188
:10B7A000E3119091E4113DDC809131018F7780931A
:10B7B0003101809131018F7E8093310110923001EF
:10B7C00080911113909112130E942EBB109225129A
:10B7D00010920F0B81E080930A02809101129091E8
:10B7E0000212CF910C94E743AF92BF92CF92DF92B7
:10B7F000EF92FF920F931F93CF93DF937C016B0126
:10B800005A01D0E0C0E08D2F90E0F701A181B28114
:10B810008A159B05D0F4F601E80FF91F608102EC50
:10B820001AE921E03327C6270C0F111D211D311DF8
:10B830002BBFF801C791ED91FC9111970190F08118
:10B84000E02DCD011995DF5FDECFED91FC911197D1
:10B850000190F081E02D6C2FCD01DF91CF911F91F0
:10B860000F91FF90EF90DF90CF90BF90AF90199421
:10B87000CF93DF9300D01F921F92CDB7DEB7FE01AA
:10B88000319625E0DF011D922A95E9F724E8298306
:10B8900025E52C832AE22D836A834B8345E050E023
:10B8A000BF01A2DF65E070E080E090E00E941E89A9
:10B8B00080E00F900F900F900F900F90DF91CF913D
:10B8C0000895EF92FF921F93CF93DF931F92CDB70E
:10B8D000DEB77C01162FFC01618172810E94B9489C
:10B8E00065E070E080E090E00E941E8942E462E43E
:10B8F000C701BEDF412F60E0C701BADF811163C01D
:10B9000040E061E0C701B4DF81115DC040E062E06A
:10B91000C701AEDF811157C046E062E0C701A8DF72
:10B92000811151C040E063E0C701A2DF81114BC02B
:10B9300040E064E0C7019CDF11E0811110E040E0CD
:10B9400065E0C70195DF811101C01F5F40E066E03F
:10B95000C7018EDF811101C01F5F40E067E0C701B2
:10B9600087DF811101C01F5F40E068E0C70180DF11
:10B97000811101C01F5F40E069E0C70179DF8111DB
:10B9800001C01F5F44E06AE0C70172DF811101C09E
:10B990001F5F44E06AE0C7016BDF811101C01F5FD8
:10B9A00062E370E080E090E00E941E8982E8898373
:10B9B00041E050E0BE016F5F7F4FC70115DF81E0BE
:10B9C000183011F0111180E00F90DF91CF911F918D
:10B9D000FF90EF900895CF93DF9300D01F92CDB7E3
:10B9E000DEB72AEA2983FC0120812A836B834C83FA
:10B9F00044E050E0BE016F5F7F4FF6DE0F900F9086
:10BA00000F900F90DF91CF9108953FB7F89420E009
:10BA1000822F90E0841795079CF4FC01EE0FFF1F26
:10BA2000EC5EFD4EA081B181880F991FFB01E80FEC
:10BA3000F91FCD0196958795918380832F5FE8CF7D
:10BA40003FBF10920B1308952F923F925F926F9217
:10BA50007F928F929F92AF92CF92DF92EF92FF925E
:10BA60000F931F93CF93DF931F921F92CDB7DEB733
:10BA70006DB67EB60E9412850E9407850E945E8583
:10BA8000029709F023C20E944985882309F419C24C
:10BA9000C0902A12D0902B12E0900112F090021266
:10BAA000B601C7010E944F438823F1F0F701E2502D
:10BAB000FE4F00E010E0819191918C159D0571F48D
:10BAC0000E945689000F111F000F111FF701E00F90
:10BAD000F11F608371838283938307C00F5F1F4FC1
:10BAE0000E31110541F701C0A8DC1092100BEDB624
:10BAF000FEB64091130B5091140BCA01880F991F89
:10BB00002DB73EB7281B390B0FB6F8943EBF0FBEBA
:10BB10002DBF0DB71EB70F5F1F4F8091160B8230E0
:10BB200061F0833021F1813009F070C0B80180915B
:10BB30000D1390910E1369DF33C03FB7F89420E0E6
:10BB4000822F90E08417950774F4880F991FF801ED
:10BB5000E80FF91FDC01AD5EBC4E8D919C91918385
:10BB600080832F5FEDCF3FBF1092331319C03FB7D3
:10BB7000F89420E0822F90E08417950774F4880FE2
:10BB8000991FF801E80FF91FDC01AB51BE4E8D91F2
:10BB90009C91918380832F5FEDCF3FBF10920A135A
:10BBA00020E06AE071E0822F90E04091130B509109
:10BBB000140B8417950754F5689FF001699FF00DE9
:10BBC0001124E950F04FA085B1858C918823E1F0D4
:10BBD000A081B1813C91C801830F911D830F911DFC
:10BBE000DC0112978D919C91A281B3814D915C9162
:10BBF00011970480F581E02D4817590711F4108240
:10BC000003C070838D939C932F5FCDCF0FB6F894B4
:10BC1000FEBE0FBEEDBE8091F110882321F080EFB3
:10BC200090E10E947A858091FB10882321F08AEFB1
:10BC300090E10E947A8580910511882321F084E0AB
:10BC400091E10E947A8580910F11882321F08EE086
:10BC500091E10E947A858091110B882309F465C0D7
:10BC600080910511811105C080910F11882309F47D
:10BC700050C08091081190910911E0910C11F09140
:10BC80000D11238134812817390724F4808581110F
:10BC900009C00EC0218132818217930734F4808558
:10BCA000811106C088E090E005C080E190E002C00C
:10BCB00080E290E02091121130911311E091161161
:10BCC000F0911711438154814217530724F42085C2
:10BCD000222349F00AC041815281241735073CF4E0
:10BCE0002085222311F0816003C0846001C082603E
:10BCF0002091EB103091EC102817390719F41092AD
:10BD0000ED1007C09093EC108093EB1081E08093CE
:10BD1000ED108091EB109091EC10429709F4DAC08D
:10BD200081E08093111180930711E8E9F0E18BE93C
:10BD300090E19A83898398EE892E93E0992E552479
:10BD40005394CF010197DC018C91882309F4ACC096
:10BD5000E480F580D70117968C911797882309F412
:10BD6000A3C08081882309F49FC041815281189625
:10BD70006C918401041B150B101611061CF08A012E
:10BD8000085E134020E030E022242394312C8FE021
:10BD900097E2A12CC62ED12C2C143D04ACF56430B6
:10BDA000A9F040F4623071F0633019F5C901865290
:10BDB0009A4F13C0653071F06630D9F4C9018454CC
:10BDC0009A4F0BC0C90180529A4F07C0C9018E52C9
:10BDD0009A4F03C0C90188539A4FDC0112968D9186
:10BDE0009C911397841B950B97FF03C091958195A8
:10BDF00091098017910714F4A22C8C01BFEF2B1A24
:10BE00003B0A2E5F3F4FC8CF81E08A0DD7011996BC
:10BE10009C919923F1F1643099F028F4623041F05B
:10BE2000633049F036C06530A1F06630D9F031C0DA
:10BE3000813021F52DC0813049F1833051F51EC08C
:10BE4000813011F1823011F1833011F1843009F524
:10BE500015C08130B9F08230B9F08430C9F0853036
:10BE6000C1F40CC0813061F0823061F0833061F048
:10BE7000843061F0853061F0863059F481E009C08A
:10BE800086E007C085E005C084E003C083E001C010
:10BE900082E0A981BA819C91981302C0108204C0EB
:10BEA0005082A981BA818C93379629813A81295F82
:10BEB0003F4F3A83298330E1EC3EF30709F041CF4D
:10BEC00003C00E941E85B9DA81E066C00E941E850B
:10BED00080E062C0E090EE10F090EF101E141F049E
:10BEE0000CF055C0809106110091011210910212C0
:10BEF00060912812709129128823B1F081E080931B
:10BF00000711C8010E944F43811115C0A701FF0C02
:10BF1000660B770B2AE331E8C8010E94B643909381
:10BF200029128093281207C0C8010E944F43811133
:10BF300002C010920711809110110091011210910E
:10BF4000021260912612709127128823D1F081E0AD
:10BF500080931111C8010E944F438111E6CE409198
:10BF6000EE105091EF10052E000C660B770B27E3B7
:10BF700031E8C8010E94B64390932712809326129D
:10BF8000D4CEC8010E944F438111CFCE02C010927F
:10BF9000071110921111C9CE0FB6F8947EBE0FBED4
:10BFA0006DBE0F900F90DF91CF911F910F91FF9079
:10BFB000EF90DF90CF90AF909F908F907F906F9099
:10BFC0005F903F902F9008951F920F920FB60F929F
:10BFD00011240BB60F922F933F934F938F939F9300
:10BFE000EF93FF938091840090918500209110122F
:10BFF00030911112821B930B2091840030918500A7
:10C000003093111220931012803727E1920770F1BC
:10C01000909313128093121280910613909107133C
:10C02000029751F49091241280910C1398133CC004
:10C0300081E080930B133EC080910613909107130B
:10C04000892B49F481E090E09093071380930613C5
:10C0500010920F122FC08091061390910713019731
:10C0600061F5809124128430D8F527C020912412E4
:10C07000283008F047C09C012C5D3540293B3B40EF
:10C0800068F4E0912412EF5FE0932412F0E0EE0FE9
:10C09000FF1FEE5EFD4E9183808334C080910613B6
:10C0A00090910713029771F583E090E09093071346
:10C0B000809306131092241225C08091061390914C
:10C0C00007130397B9F79091241280910C139813DA
:10C0D000F1CF80910C13843068F382E090E0E6CFDA
:10C0E00080910F128F5F80930F12863018F382E0D9
:10C0F00090E090930713809306138091241280930D
:10C100000C13D8CFFF91EF919F918F914F913F9159
:10C110002F910F900BBE0F900FBE0F901F90189590
:10C120000F931F938091071281110DC00E945689B1
:10C130006093031270930412809305129093061279
:10C1400081E0809307120E9456890091031210919A
:10C1500004122091051230910612DC01CB01801BE4
:10C16000910BA20BB30B893E9340A105B105A8F03A
:10C170008AE30E949858892B11F060E001C061E0C9
:10C180008AE30E94C0580E945689609303127093FC
:10C19000041280930512909306121F910F91089537
:10C1A0000F931F930E9456890091DB111091DC11AF
:10C1B0002091DD113091DE11DC01CB01801B910B50
:10C1C000A20BB30B85339142A105B10518F081E0B4
:10C1D0008093DA111F910F91A3CFFC0180E090E0D2
:10C1E0006150710977FD18C02191022E000C330BAC
:10C1F000322F22278227932728E0AC01440F551FB6
:10C2000097FF06C0CA0131E2832730E1932701C0BE
:10C21000CA01215091F7E4CF089580910B02882341
:10C2200011F0599801C0599A90910B0281E0892729
:10C2300080930B02089561E089E20C94C05810923B
:10C24000020B40914E0650914F0660E070E024E6EC
:10C2500031E680913C0690913D060C94B6430F93D5
:10C260001F93CF93DF9360E08BE20E94C058009150
:10C27000581210915912C0913C06D0913D06B80158
:10C28000CE010E944F43882341F0B801CE01DF91D7
:10C29000CF911F910F910C946743DF91CF911F9124
:10C2A0000F91089580915906882369F08091010BC0
:10C2B000882349F081E08093FE0A809158060E940D
:10C2C0009A450C9451860895CF93DF93CDB7DEB78E
:10C2D00065970FB6F894DEBF0FBECDBF81E08093A7
:10C2E000020B80915512882371F182E390E09A83CA
:10C2F000898388E290E09C838B838EE690E09E8326
:10C300008D8384EF91E098878F831D8A84E08F93DB
:10C310008DB79EB745970FB6F8949EBF0FBE8DBFE1
:10C32000ADB7BEB7119685E1FE01319601900D9231
:10C330008A95E1F780E19AE00E94DF3C0FB6F8941D
:10C34000DEBF0FBECDBF65960FB6F894DEBF0FBE41
:10C35000CDBFDF91CF91089580914B12811112C012
:10C3600082EC9BE9A1E0BB27ABBFFC016791769112
:10C3700082E00E94738181E080932C12109230122F
:10C3800010922D12089560E089E20E94C0582BE1BE
:10C3900031E642E350E060E070E080913C0690912D
:10C3A0003D060C94B64361E08BE20E94C058E89AC7
:10C3B0002FE231E648E853E160E070E080913C060E
:10C3C00090913D060E94B643909359128093581263
:10C3D000089561E08BE20E94C058E89A2FE231E6AE
:10C3E00048E853E160E070E080913C0690913D06A2
:10C3F0000E94B6439093591280935812089581E297
:10C400000E94985821E0892B09F420E0822F08959A
:10C4100080915406882309F44CC08091010B882335
:10C4200009F447C081E08093FE0AE9DF882329F000
:10C43000809157068823D9F106C080915506811155
:10C4400005C0809154060E949A4531C090915406CF
:10C45000963069F5823081F08330D1F0813039F542
:10C46000E0916A0AF0916B0A74978081918145E5A9
:10C4700050E060E070E017C0E0916A0AF0916B0A4A
:10C480007497808191814AE550E060E070E00BC0D4
:10C49000E0916A0AF0916B0A7497808191814FE56F
:10C4A00050E060E070E08659954F0E949D500C94DA
:10C4B0005186089580915712882339F08091561241
:10C4C000882319F081E08093FB0A80913E069091C9
:10C4D0003F06DC01ED91FC910688F789E02D199566
:10C4E0008091511281114FDF80915012882391F079
:10C4F00061E088E00E94C05840914E1250914F1266
:10C5000060E070E025EF38E880913C0690913D06B0
:10C510000E94B64380915712882321F080915612D1
:10C52000811101C075DF80915612882379F08091C6
:10C530005712882359F080915412882339F0E091E2
:10C540005212F091531282810E94C18178CE1F92C3
:10C550000F920FB60F9211240BB60F922F933F93A9
:10C560004F935F936F937F938F939F93AF93BF93FB
:10C57000EF93FF93809157128823A9F0489917C031
:10C58000E8982FE231E64CE251E060E070E0809103
:10C590003C0690913D060E94B64380915612882336
:10C5A00031F088DF04C0489B02C0E89858DEFF9154
:10C5B000EF91BF91AF919F918F917F916F915F911B
:10C5C0004F913F912F910F900BBE0F900FBE0F9088
:10C5D0001F9018958091000B811156C010DF8823A1
:10C5E000F1F081E08093000B80913E0690913F0630
:10C5F000DC01ED91FC910288F389E02D19950E94F0
:10C60000118725E337E848E95AE360E070E080915C
:10C610003C0690913D060E94B64311DE09C0809110
:10C620005612882329F180915712882311F0D1DE08
:10C63000EFCEB9DE80915412882339F0E091521286
:10C64000F091531282810E94C18140914C1250910D
:10C650004D1214161506BCF4052E000C660B770B54
:10C660002AE532E680913C0690913D060C94B64353
:10C6700080915412882339F0E0915212F0915312B4
:10C6800082810E94C18116CF08950F931F9320913C
:10C690004B12211135C042EC5BE961E077279C0128
:10C6A000220F331F820F931F092E000CAA0BBB0B06
:10C6B0000296A11DB11D840F951FA61FB71FABBF0A
:10C6C000FC01879102EC1BE921E0332740913012F5
:10C6D00093E0499FA0011124052E000C660B770BF7
:10C6E0004E5F5F4F6F4F7F4F040F151F261F371F81
:10C6F0002BBFF8010791801718F01F910F912CCED6
:10C700001F910F910895833091F028F4813049F002
:10C71000823051F00895853081F060F0863081F0EC
:10C72000089589E090E00EC08AE090E00BC08BE0B5
:10C7300090E008C08CE090E005C08DE090E002C081
:10C740008EE090E0A2CF8F929F92AF92BF92CF9255
:10C75000DF92EF92FF920F931F93CF93DF93EC0141
:10C76000A62E80914B1281116BC042EC5BE961E017
:10C7700077276E01CC0CDD1CCC0EDD1E0D2C000CC1
:10C78000EE08FF08D701C6010296A11DB11D480F92
:10C79000591F6A1F7B1F6BBFFA01879142EC5BE94F
:10C7A00061E07727B090301293E0B99E80011124A8
:10C7B000012E000C220B330B0E5F1F4F2F4F3F4FEC
:10C7C000400F511F621F731F6BBFFA01479148173B
:10C7D00008F036C080902E1290902F1200914412D3
:10C7E00010914512B401C8010E944F43882321F0E3
:10C7F000B401C8010E94674382EC9BE9A1E0BB271A
:10C800008C0D9D1DAE1DBF1DABBFFC0167917691C8
:10C8100082E00E947381B0922D12C0933012AA2040
:10C8200079F010922C122CEA31E642E350E060E0FD
:10C8300070E0C8010E94B64390932F1280932E128D
:10C84000DF91CF911F910F91FF90EF90DF90CF90EC
:10C85000BF90AF909F908F900895CF92DF92EF920C
:10C86000FF9280914B12811134C080914A1288232B
:10C8700081F161E08EE090E066DF60914812709196
:10C880004912CB01A0E0B0E0C0904612D090471210
:10C89000E12CF12CC816D906EA06FB0664F4BC01AB
:10C8A000CD016C197D098E099F090E941D55C60E88
:10C8B000D71EE81EF91E2DE234E6B701A6018091CD
:10C8C0004412909145120E94B64390934312809374
:10C8D0004212FF90EF90DF90CF900895CF92DF92B9
:10C8E000EF92FF9280914B12811134C080914112DE
:10C8F000882381F161E08DE090E025DF60913F12B7
:10C9000070914012CB01A0E0B0E0C0903D12D090F9
:10C910003E12E12CF12CC816D906EA06FB0664F497
:10C92000BC01CD016C197D098E099F090E941D551E
:10C93000C60ED71EE81EF91E2EE634E6B701A60184
:10C9400080914412909145120E94B64390933C12FC
:10C9500080933B12FF90EF90DF90CF900895CF929D
:10C96000DF92EF92FF9280914B12811134C080913F
:10C970003A12882381F161E08CE090E0E4DE60917E
:10C98000381270913912CB01A0E0B0E0C09036129D
:10C99000D0903712E12CF12CC816D906EA06FB0616
:10C9A00064F4BC01CD016C197D098E099F090E94B8
:10C9B0001D55C60ED71EE81EF91E2FEA34E6B70134
:10C9C000A60180914412909145120E94B643909323
:10C9D000351280933412FF90EF90DF90CF9008953E
:10C9E00080914B1281112CC080913312882341F029
:10C9F00080913A12811104C081E080933A12AFDF36
:10CA000080913212882361F080914B12811108C00D
:10CA100080914112811104C081E0809341125EDF58
:10CA200080913112882361F080914B12811108C0EE
:10CA300080914A12811104C081E080934A120DCF87
:10CA400008958091D0069091D106DC01ED91FC9182
:10CA50000084F185E02D19958091D0069091D10642
:10CA6000DC01ED91FC910480F581E02D1994809119
:10CA70000702813019F485E080930702089510922F
:10CA8000CB06089580913306882371F01092330607
:10CA90008091D606882341F064ED73E18091D4063D
:10CAA0009091D5060C94B956089580917E0F8330ED
:10CAB00099F08091330681110FC081E08093330695
:10CAC0008091D606882341F06FEB73E18091D40604
:10CAD0009091D5060C94B956089580913306882319
:10CAE00019F080E090E0CECF80E090E0DECF809142
:10CAF0003206833079F083E0809332068091D60647
:10CB0000882341F06EEA73E18091D4069091D506B6
:10CB10000C94B956089580913206823079F082E003
:10CB2000809332068091D606882341F06DE973E147
:10CB30008091D4069091D5060C94B95608958091B1
:10CB40003206813079F081E0809332068091D606FA
:10CB5000882341F06CE873E18091D4069091D5066A
:10CB60000C94B95608958091070180FF1BC08091F5
:10CB7000D606882351F08BE59BE00E940F98811127
:10CB800008C08091670B811104C08BE59BE00C9479
:10CB9000753E6DE274E18091D4069091D5060E94B5
:10CBA000B956F3CF08958091070181FF1BC0809192
:10CBB000D606882351F08AE29BE00E940F988111EB
:10CBC00008C08091360B811104C08AE29BE00C946E
:10CBD000753E60E074E18091D4069091D5060E9484
:10CBE000B956F3CF08958091070180FF17C0809157
:10CBF000D606882331F08BE59BE00E940F988823AE
:10CC000021F08BE59BE00C94239867E174E180911F
:10CC1000D4069091D5060E94B956F3CF089580911D
:10CC2000070181FF17C08091D606882331F08AE280
:10CC30009BE00E940F98882321F08AE29BE00C94ED
:10CC400023986AEE73E18091D4069091D5060E94F4
:10CC5000B956F3CF08950E940F3C80913406882383
:10CC600061F18091000B811128C08091CC06811167
:10CC700024C081E08093CC060E94B49280915F062C
:10CC8000882319F010925F060CC08091D006909115
:10CC9000D106DC01ED91FC910088F189E02D61E085
:10CCA00019958091D606882341F061E673E1809161
:10CCB000D4069091D5060C94B9560895CF93DF937E
:10CCC0008091070180FD2AC0C0916B06D0916C064F
:10CCD00080916F06882371F08EE30E94F2598130B3
:10CCE00092402CF010926C0610926B060AC081E004
:10CCF00090E003C08EE30E94F25990936C068093FB
:10CD00006B0680916B0690916C068C179D0719F449
:10CD100010926D0603C081E080936D06DF91CF9184
:10CD20000895CF93DF938091070181FD2AC0C091C0
:10CD30006506D091660680916906882371F08FE3BD
:10CD40000E94F259813092402CF0109266061092A7
:10CD500065060AC081E090E003C08FE30E94F259AB
:10CD600090936606809365068091650690916606AD
:10CD70008C179D0719F41092670603C081E0809319
:10CD80006706DF91CF91089580917E0F833041F146
:10CD90002CF48130A9F0823099F02DC086305CF5FA
:10CDA0008091C5069091C606DC01ED91FC9104804E
:10CDB000F581E02D19958091C3069091C40614C0A9
:10CDC0008091C9069091CA06DC01ED91FC91048026
:10CDD000F581E02D19958091C7069091C80604C091
:10CDE0008091C5069091C606DC01ED91FC9104800E
:10CDF000F581E02D19958091D0069091D106DC0146
:10CE0000ED91FC91E45BFF4F0190F081E02D1995CD
:10CE10008091D0069091D106DC01ED91FC910284C5
:10CE2000F385E02D60E070E019940E940F3C809142
:10CE300034068823D1F08091CC068823B1F010927B
:10CE4000CC060E94829280915F06882389F010921E
:10CE50005F068091D606882341F065E773E18091F3
:10CE6000D4069091D5060E94B9561092CC0608952A
:10CE70008091D0069091D106DC01ED91FC91008863
:10CE8000F189E02D60E01995E4CFCF93DF93C09155
:10CE90007112D0917212BE018DE89BE00E944F4347
:10CEA000882329F0BE018DE89BE00E946743109221
:10CEB000721210927112DF91CF9108950F931F9308
:10CEC000CF93DF938091830F9091840FA091850F72
:10CED000B091860F181619061A061B060CF044C0EE
:10CEE0000E940F3C809134068823C9F10091711291
:10CEF00010917212B8018DE89BE00E944F43882385
:10CF0000D9F0EBE8FDE0C0E0D0E08191919180178D
:10CF1000910769F40E945689CC0FDD1FCC0FDD1FED
:10CF2000C357D44F688379838A839B831DC021961E
:10CF3000CE31D10551F718C04091830F5091840F25
:10CF40006091850F7091860F23EA38E68DE89BE0AB
:10CF50000E94B643909372128093711205C0DF91C4
:10CF6000CF911F910F9191CFDF91CF911F910F9191
:10CF700008958091000B811148C00E940F3C809160
:10CF8000DE0D8823B1F080913406882391F0109251
:10CF900034061092DE0D0E94363C80915C1288238C
:10CFA00041F06CE373E180915A1290915B120E9400
:10CFB000B9568091620690916306806290936306F1
:10CFC000809362068091CC06882311F081E001C035
:10CFD00080E00E94339681E080935F0626DF809197
:10CFE000940F81110FC080914A06882359F021E2E5
:10CFF00035E644E650E060E070E08DE89BE00E949A
:10D00000B64301C01EDDC0DE59CF0895BDDE0E94CB
:10D010001E8B0E940F3C809134068111AADF809103
:10D02000D2069091D306DC01ED91FC910480F5814C
:10D03000E02D19958091CE069091CF06DC01ED91FF
:10D04000FC910480F581E02D199580915F0F882374
:10D0500059F080914B0690914C06DC01ED91FC91CA
:10D060000480F581E02D1994089580910C028823A5
:10D0700059F00E94178F20E030E040E050E40E9419
:10D0800020B787FF3BC008950E94178F20E030E053
:10D090004AE754E40E9485B70E9498B92091DF0FB7
:10D0A0003091E00F4091D9066217730710F44423C2
:10D0B00059F1442309F446C00E94178F20E030E064
:10D0C0004AE754E40E9485B70E9498B92091DF0F87
:10D0D0003091E00F62177307A8F11092D90681E032
:10D0E0008093D8068091D606882361F164E474E1C8
:10D0F0008091D4069091D5060C94B95610920C02EA
:10D1000081E08093D806089581E08093D90610923B
:10D11000D8068091D606882391F063E674E1809169
:10D12000D4069091D5060E9448550E94799860E6F1
:10D1300074E18091D4069091D5060E94B95666DFBD
:10D140000C94318C08950E940F3C80913406882302
:10D1500069F00FDF8091D606882341F06CE473E11B
:10D160008091D4069091D5060C94B956089580917B
:10D17000000B81115EC08091CD06823068F08091F5
:10D18000D606882309F455C06AEF72E18091D4066F
:10D190009091D5060C94B9560E940F3C8091DE0DFB
:10D1A000882309F446C080913406811142C081E091
:10D1B000809334061092DE0D0E94363C80915C1202
:10D1C000882341F06BEE72E180915A1290915B12CC
:10D1D0000E94B95680916206909163068061909397
:10D1E0006306809362068091D0069091D106DC019F
:10D1F000ED91FC910280F381E02D19958091CD068F
:10D20000811116C04091790F50917A0F81E080937F
:10D210005F064115510559F060E070E02BE236E6FB
:10D220008DE89BE00E94B6430E94829201C013DD0C
:10D2300045CE0895AF92BF92CF92DF92EF92FF92C8
:10D240000F931F93CF93DF939091691291110BC0AD
:10D250002091DC063091DD0630936812209367122E
:10D2600091E09093691290915F1291110BC02091FF
:10D27000DA063091DB0630935E1220935D1291E066
:10D2800090935F12A0906712B090681200915D12A7
:10D2900010915E12D091D606843608F047C0C82F90
:10D2A000682F70E080E090E00E9424B720E030E03A
:10D2B00048EC52E40E942BB96B017C01B501BB0C18
:10D2C000880B990B0E9426B79B01AC01C701B601E0
:10D2D0000E9485B70E9493B97093DD066093DC06C7
:10D2E000B801110F880B990B0E9426B79B01AC0166
:10D2F000C701B6010E9485B70E9493B97093DB06FF
:10D300006093DA06DD2371F16AEC72E18091D40654
:10D310009091D5060E9448556C2F8091D40690912B
:10D32000D5060E943F4868EC72E10CC0B092DD0661
:10D33000A092DC061093DB060093DA06DD2391F061
:10D340006CED72E18091D4069091D506DF91CF917A
:10D350001F910F91FF90EF90DF90CF90BF90AF9013
:10D360000C94B956DF91CF911F910F91FF90EF90E0
:10D37000DF90CF90BF90AF900895CF93823069F443
:10D380009091720F20916F0F3091730F4091700F39
:10D390005091710F60916E0F0CC090916C0F2091A5
:10D3A000690F30916D0F40916A0F50916B0F609132
:10D3B000680F60939B135093981340939913309385
:10D3C000971320939A1390939C13909100028917BE
:10D3D000B9F0809300029091D606992389F0C82F66
:10D3E0006FEA72E18091D4069091D5060E9448556B
:10D3F0006C2F8091D4069091D506CF910C9428483B
:10D40000CF910895833079F030F4813051F082303B
:10D4100091F48BE30BC0843041F0853061F482E4F9
:10D4200005C08CE303C080E401C081E40E949858E9
:10D4300021E0892B09F420E0822F0895E3DF91E0B9
:10D44000892708952F923F924F925F926F927F9219
:10D450008F929F92AF92BF92CF92DF92EF92FF9204
:10D460000F931F93CF93DF9300D01F92CDB7DEB7FA
:10D470005C01CCDD0E94D08D0E94058E8091D40687
:10D480009091D5060E94A6560E94C17524E0A2166E
:10D49000B10409F49CC00CF04FC0A3E0AA16B1047B
:10D4A00009F03CC18CE190E00E9499BA9C838B8387
:10D4B00084EF95E0AB81BC8111969C938E9313967B
:10D4C000BC92AE92129781E09FEF15969C938E933B
:10D4D00014978FEF90E017969C938E93169719965A
:10D4E0001C921E92189758961C925897CD010E9434
:10D4F0000B8388EE95E0EB81FC8191838083E09142
:10D500008E13F0918F13D08C00915C1110915D11EE
:10D5100016950795E0905A11F0905B11F694E794F8
:10D5200060E675E18091D4069091D5060E94B956C7
:10D53000812C9924939412C1B5E0AB16B10409F47F
:10D54000A6C0E6E0AE16B10409F0E8C08CE190E0B8
:10D550000E9499BA9C838B8384EF95E0AB81BC8158
:10D5600011969C938E931396BC92AE92129781E083
:10D570009FEF15969C938E9314978FEF90E01796DC
:10D580009C938E93169719961C921E9218975896F4
:10D590001C925897CD010E940B8388EE95E0EB8199
:10D5A000FC8191838083E091C006F091C106D08C0C
:10D5B00000919B1110919C1116950795E09099117F
:10D5C000F0909A11F694E79463E975E1A0C08CE1BC
:10D5D00090E00E9499BA9C838B8384EF95E0AB81A5
:10D5E000BC8111969C938E931396BC92AE92129727
:10D5F00081E09FEF15969C938E9314978FEF90E0A8
:10D6000017969C938E93169719961C921E921897B4
:10D6100058961C925897CD010E940B8388EE95E096
:10D62000EB81FC81918380830091711110917211C3
:10D6300016950795E0906F11F0907011F694E794AD
:10D6400080913F0F8C50823040F4E091D206F091EF
:10D65000D306D08C63ED75E15AC080917E0F823085
:10D6600009F07AC080913D0F8C3009F075C0E091CF
:10D67000C006F091C106D08C63EB75E18091D406B1
:10D680009091D5060E94B9568824839466C08CE197
:10D6900090E00E9499BA9C838B8384EF95E0AB81E4
:10D6A000BC8111969C938E931396BC92AE92129766
:10D6B00081E09FEF15969C938E9314978FEF90E0E7
:10D6C00017969C938E93169719961C921E921897F4
:10D6D00058961C925897CD010E940B8388EE95E0D6
:10D6E000EB81FC8191838083E091CE06F091CF069F
:10D6F000D08C009186111091871116950795E090B6
:10D700008411F0908511F694E79463E775E18091B8
:10D71000D4069091D5060E94B9561EC067E475E103
:10D720008091D4069091D5060F900F900F900F9096
:10D73000DF91CF911F910F91FF90EF90DF90CF90ED
:10D74000BF90AF909F908F907F906F905F904F9021
:10D750003F902F900C94B956812C912C0E94C1754A
:10D760006AE375E18091D4069091D5060E94B9567E
:10D770006EE275E18091D4069091D5060E944855DD
:10D78000B8018091D4069091D5060E94A24962E228
:10D7900075E18091D4069091D5060E944855B70155
:10D7A0008091D4069091D5060E94A24966E175E168
:10D7B0008091D4069091D5060E9448558D2D0E94E7
:10D7C0009D758091D4069091D5060E94A656AB8196
:10D7D000BC81ED91FC9111970280F381E02DCD0188
:10D7E0001995CA2C8A2D0E9429828D3D9540A8F456
:10D7F00064E378E08A2D0E942182EB81FC81F78A24
:10D80000E68AB70182810E9439826CED75E08A2D2B
:10D810000E942582DD20C1F01AC064E873E08A2DE1
:10D820000E942582AB81BC8157961C930E9356971C
:10D83000B80112968C910E9439826CED75E08A2DA8
:10D840000E942182DD2019F03324339401C0312C51
:10D8500021E02983212C2A830E94245D80910511D7
:10D86000882359F1AB81BC81ED91FC9111976091B6
:10D870000A1170910B110190F081E02DCD011995E5
:10D880008C2D0E9429828D3DB5E09B075CF4843885
:10D89000E3E09E0784F08C018D3D954074F00CED23
:10D8A00015E00BC07C01853398403CF064E3E62E24
:10D8B00068E0F62E02C004E813E02A8121111FC09F
:10D8C0008091FB108823C9F1E0910211F0910311BE
:10D8D000858196814091FE105091FF109C0121534B
:10D8E0003109421753074CF1C196841795072CF163
:10D8F0000E9456896415750586059705F0F080919C
:10D90000FB108823C1F04091FE105091FF10E09170
:10D910000211F0910311858196819C01285C3109E7
:10D92000421753072CF088539F4F841795071CF418
:10D9300081E0382605C021E02A83222009F47CC03A
:10D94000332009F445C0DD20F9F064E873E08C2D44
:10D950000E942582992009F458C06091590F709156
:10D960005A0F41E08C2D0E94E0810E949296AB817B
:10D97000BC8112968C910E94298208171907ACF37A
:10D980008C2D0E94B38141C064E378E08C2D0E940D
:10D9900021829920B1F06091590F70915A0F40E0A7
:10D9A0008C2D0E94E0810E949296AB81BC811296E0
:10D9B0008C910E9429828E159F05ACF38C2D0E94BC
:10D9C000B381EB81FC81F78AE68AB701828110C0BE
:10D9D000DD20B1F064E378E08C2D0E942182AB81E0
:10D9E000BC815796FC92EE925697B70112968C9195
:10D9F0000E9439826CED75E08C2D0E94258212C048
:10DA000064E873E08C2D0E942582EB81FC81178BEA
:10DA1000068BB80182810E9439826CED75E08C2DF5
:10DA20000E9421820E9456892B013C01F8EC4F0E86
:10DA3000511C611C711C1A8229812223D9F1809109
:10DA4000F1108823A9F14091F4105091F510E09164
:10DA5000F810F091F910858196819C01285C3109BC
:10DA6000421753072CF088539F4F8417950704F5EE
:10DA700081E0D8268091D4069091D506DD2039F03A
:10DA800067E075E10E94B95682E090E006C065EF5C
:10DA900074E10E94B95681E090E00E94D88D0E9406
:10DAA0005689AB81BC815896DC922224239403C012
:10DAB000212C1EC0212C8091F110882309F46FC203
:10DAC000E091F810F091F910858196814091F41061
:10DAD0005091F5109C0121533109421753070CF462
:10DAE0005EC2C19621E02983841795070CF457C2C2
:10DAF0000E941C850E94EA488DE89BE00E94E74353
:10DB000080911A0B882309F4A7CE80911C0B8823DF
:10DB100009F4A2CE0E94EA480E94604C8823D1F307
:10DB200084E0A816B104D9F134F4B3E0AB16B10423
:10DB300009F438C1C4C1E5E0AE16B10409F4CDC0A2
:10DB4000F6E0AF16B10409F0BAC110934D0F00937F
:10DB50004C0FF0924F0FE0924E0FD092500FB80141
:10DB60008CE291E00E947B48B7018EE291E00E9436
:10DB70007B486D2D80E391E00E94D749B80186E093
:10DB80000E945881B70186E00E943D81E091C00665
:10DB9000F091C106D08E6CED75E086E091C08820D2
:10DBA000C1F010934D0F00934C0FF0924F0FE09285
:10DBB0004E0FD092500FB8018CE291E00E947B484A
:10DBC000B7018EE291E00E947B486D2D80E391E0E9
:10DBD00017C01093410F0093400FF092430FE09253
:10DBE000420FD092440FB80180E291E00E947B483E
:10DBF000B70182E291E00E947B486D2D84E291E0C2
:10DC00000E94D749B80184E00E945881B70184E09E
:10DC10000E943D81882049F0E091C006F091C10644
:10DC2000D08E6CED75E084E04BC0E091D206F091AF
:10DC3000D306D08E80913F0F8D3029F4E09173127E
:10DC4000F0917412D08E6CED75E084E00E94398200
:10DC500066E970E080E090E00E941E8980913F0FAD
:10DC60008D3011F584E00E942982A091D206B091F6
:10DC7000D3068D3D95404CF0ED91FC9111970190AC
:10DC8000F081E02D6FEF7FEF08C0ED91FC911197CF
:10DC90000190F081E02D61E070E0CD011995809157
:10DCA000D2069091D3066FC08091D2069091D30690
:10DCB000DC01ED91FC910480F581E02D1995FFC008
:10DCC0000E94398266E970E080E090E00E941E893F
:10DCD0008091C0069091C106EBCF1093480F00933E
:10DCE000470FF0924A0FE092490FD0924B0FB801C4
:10DCF00087E291E00E947B48B70189E291E00E94AF
:10DD00007B486D2D8BE291E00E94D749B80185E0F8
:10DD10000E945881B70185E00E943D81E091CE06C6
:10DD2000F091CF06D08E6CED75E085E00E943982CF
:10DD300066E970E080E090E00E941E8980913E0FCD
:10DD40008D3059F585E00E942982A091CE06B091D0
:10DD5000CF068D3D95404CF0ED91FC9111970190CF
:10DD6000F081E02D6FEF7FEF08C0ED91FC911197EE
:10DD70000190F081E02D61E070E0CD011995809176
:10DD8000CE069091CF06DC01ED91FC910190F081DF
:10DD9000E02D60E070E0199592C08091CE069091E0
:10DDA000CF0686CF10935C0F00935B0FF0925E0F4F
:10DDB000E0925D0FD092550FB8018BE391E00E9485
:10DDC0007B48B7018DE391E00E947B486D2D85E390
:10DDD00091E00E94D749B80183E00E945881B701C1
:10DDE00083E00E943D818091550FE0918E13F09168
:10DDF0008F13808F8091550F0E94464883E00E94C8
:10DE000029822091550F222369F1B9E0BC1538F021
:10DE100020915C1130915D113695279502C02EEE50
:10DE200032E08217930709F44AC06091590F70914C
:10DE30005A0F41E083E00E94E0810E949296EB81BC
:10DE4000FC8182810E94298208171907B4F383E0BC
:10DE50000E94B381AB81BC8157961C930E93569759
:10DE6000B80129C029E02C1508F49BC020915A1153
:10DE700030915B11369527958217930701F16091D8
:10DE8000590F70915A0F40E083E00E94E0810E9498
:10DE90009296EB81FC8182810E9429828E159F05DA
:10DEA000B4F383E00E94B381AB81BC815796FC92AE
:10DEB000EE925697B70112968C910E94398280910A
:10DEC000D4069091D5060E94A6565BD6B4E0AB1658
:10DED000B10459F0E5E0AE16B10451F0F3E0AF162D
:10DEE000B10471F46BEA74E105C06BED74E102C03A
:10DEF00062EC74E18091D4069091D5060E94B956E7
:10DF000040D660EA74E18091D4069091D5060E94D3
:10DF1000B95664E974E18091D4069091D5060E94C7
:10DF20004855B8018091D4069091D5060E94A24927
:10DF300068E874E18091D4069091D5060E94485516
:10DF4000B7018091D4069091D5060E94A2496CE752
:10DF500074E18091D4069091D5060E9448558D2D8C
:10DF6000ECD58091D4069091D5060E94A6560F90CC
:10DF70000F900F900F90DF91CF911F910F91FF9015
:10DF8000EF90DF90CF90BF90AF909F908F907F9059
:10DF90006F905F904F903F902F900C94018E19825C
:10DFA000A7CD2AEC38E068CF089508950895089524
:10DFB0000895623039F0633041F0613041F44093AC
:10DFC0003312089540933212089540933112089508
:10DFD000623069F06330A1F06130D1F450933712B0
:10DFE000409336123093391220933812089550938B
:10DFF0003E1240933D123093401220933F120895F9
:10E00000509347124093461230934912209348127E
:10E010000895FC018581089508950895089508954F
:10E0200020914B12211102C0FC01628308952091BE
:10E030004B12211102C0FC016483089520914B1200
:10E04000211102C0FC016383089508950895809111
:10E050004B12811102C00C94B43F0895089580E0E2
:10E060000895089508950895089508950895809154
:10E070004B12811104C08FE090E00C944563089529
:10E0800020914B12211108C0FC018481882321F0CA
:10E0900082E090E00C944563089520914B12211189
:10E0A00008C0FC018381882321F081E090E00C947A
:10E0B0004563089580914B12811104C08BE090E07C
:10E0C0000C944563089580914B12811105C060E066
:10E0D00080E190E00C94A363089580914B1281112C
:10E0E00005C060E08FE090E00C94A36308958091F8
:10E0F0004B12811127C06330A1F028F4613049F040
:10E10000623059F008956530A1F078F06630A9F0DA
:10E11000089560E089E090E013C060E08AE090E05C
:10E120000FC060E08BE090E00BC060E08CE090E01E
:10E1300007C060E08DE090E003C060E08EE090E01A
:10E140000C94A363089580914B12811127C0633012
:10E15000A1F028F4613049F0623059F0089565303B
:10E16000A1F078F06630A9F0089561E089E090E0D0
:10E1700013C061E08AE090E00FC061E08BE090E0C6
:10E180000BC061E08CE090E007C061E08DE090E0C2
:10E1900003C061E08EE090E00C94A36308952091A9
:10E1A0004B12211109C0FC018281882329F061E012
:10E1B00088E090E00C94A363089520914B12211104
:10E1C00009C0FC018481882329F061E082E090E0AD
:10E1D0000C94A363089520914B12211109C0FC01F6
:10E1E0008381882329F061E081E090E00C94A363AF
:10E1F000089580914B12811105C061E086E090E0A6
:10E200000C94A363089580914B12811105C060E0C6
:10E210008BE090E00C94A363089580914B128111E0
:10E2200005C061E087E090E00C94A36308958091BD
:10E230004B12811105C061E085E090E00C94A3636E
:10E240000895CF93DF93FC0125812223A1F1EC01F6
:10E2500080914B1281112EC0609134127091351251
:10E2600080914412909145120E94674310923A1295
:10E2700080914B1281110CC060913B1270913C1245
:10E2800080914412909145120E946743109241126E
:10E2900080914B1281110CC0609142127091431217
:10E2A00080914412909145120E94674310924A1245
:10E2B0001092050E1D82DF91CF910895CF93DF93C9
:10E2C000FC01258121111EC0EC0180914B128111AE
:10E2D00017C08091050E811113C020EF34E648EB82
:10E2E0005BE060E070E080914412909145120E94E2
:10E2F000B643909335128093341281E08093050EDB
:10E3000081E08D83DF91CF910895862F90914B12FC
:10E31000911102C00C9483630895CF93C1E0809162
:10E320004B12811103C08C2F0E948363CF5FC730D3
:10E33000B1F7CF91089580914B12882329F06CEDAD
:10E3400075E081E00C94738184E090E00C94456367
:10E3500080914B12882329F068EE73E081E00C94E1
:10E36000738160E084E090E00C94A36380914B1291
:10E3700081111BC08091090E8823B9F068EE73E00B
:10E3800081E00E9473811092090E24EB3FE348E97B
:10E390005AE360E070E080914412909145120E942F
:10E3A000B6439093080E8093070E08956CED75E0C8
:10E3B00080E00C94738124EF31E0DB010E9493BA7A
:10E3C0002FEF30E040E050E00E9469B8CA01B90187
:10E3D00064527A4F8F4F9F4F80E00C9473818091ED
:10E3E0004B12882339F060ED77E081E00E94738161
:10E3F0000C94BE4361E083E090E00C94A363209111
:10E400004B12211109C02091060E222329F00296F9
:10E410000E94D0431092060E089520914B122223A1
:10E4200089F06FE676E080E00E9473812BEB3FE39A
:10E4300042E350E060E070E0809144129091451218
:10E440000C94B6432091060E211106C002960E943C
:10E45000D04381E08093060E089580E00E949A8167
:10E4600081E00E949A8180914B12811103C082E069
:10E470000E949A816CED75E080E00E9473816CEDE2
:10E4800075E081E00E94738180914B1281110DC073
:10E4900082EC9BE9A1E0BB27ABBFFC0167917691C1
:10E4A00082E00E9473810C94AC610895FC01808924
:10E4B00091899387828782899389958784878489C4
:10E4C000958997878687089526E00C943358809124
:10E4D000D7068093D606089580919D12882359F01F
:10E4E00080919B1290919C12DC01ED91FC91048033
:10E4F000F581E02D1994089580919D12882369F08B
:10E5000080919B1290919C12DC01ED91FC91019005
:10E51000F081E02D6FEF73E01994089580919D12C2
:10E52000882389F080919F12882321F080E090E079
:10E53000D3DF03C080E090E0DFDF90919F1281E0A5
:10E54000892780939F12089520919D12222369F0BC
:10E55000A0919B12B0919C12ED91FC9111970190AA
:10E56000F081E02DBC01CD011994089580919A129B
:10E57000882359F08091981290919912DC01ED91C5
:10E58000FC910480F581E02D1994089580919A12F0
:10E59000882369F08091981290919912DC01ED9195
:10E5A000FC910190F081E02D6FEF73E019940895D4
:10E5B00080919A12882389F080919E12882321F0FD
:10E5C00080E090E0D3DF03C080E090E0DFDF909157
:10E5D0009E1281E0892780939E12089520919A12BD
:10E5E000222369F0A0919812B0919912ED91FC91BB
:10E5F00011970190F081E02DBC01CD01199408958F
:10E6000020919712222369F0A0919512B091961251
:10E61000ED91FC9111970190F081E02DBC01CD01AD
:10E620001994089520919412222369F0A0919212D6
:10E63000B0919312ED91FC9111970190F081E02D32
:10E64000BC01CD011994089520919112222369F003
:10E65000A0918F12B0919012ED91FC9111970190C1
:10E66000F081E02DBC01CD011994089520918E1206
:10E67000222369F0A0918C12B0918D12ED91FC9142
:10E6800011970190F081E02DBC01CD0119940895FE
:10E6900020918B12222369F0A0918912B0918A12E5
:10E6A000ED91FC9111970190F081E02DBC01CD011D
:10E6B0001994089520918812222369F0A09186125E
:10E6C000B0918712ED91FC9111970190F081E02DAE
:10E6D000BC01CD011994089520918512222369F07F
:10E6E000A0918312B0918412ED91FC911197019049
:10E6F000F081E02DBC01CD01199408958091D006E0
:10E700009091D106DC01ED91FC91E05AFF4F019010
:10E71000F081E02D19948091D0069091D106DC0112
:10E72000ED91FC91E25AFF4F0190F081E02D199498
:10E730008091D0069091D106DC01ED91FC91E45AD4
:10E74000FF4F0190F081E02D199480915F0F8111AE
:10E7500017C080914B0690914C06DC0156962D9186
:10E760003C915797ED91FC910190F081E02D1216AC
:10E7700013061CF460E070E002C06FEF70E01994C3
:10E78000089580915F0F81110DC080914B0690918B
:10E790004C06DC01ED91FC910190F081E02D60E0F0
:10E7A00070E01994089580915F0F81110DC08091E0
:10E7B0004B0690914C06DC01ED91FC910190F081AB
:10E7C000E02D6FEF70E0199408958091D7068823AB
:10E7D00061F00E945E85029741F06EE876E18091DB
:10E7E000D4069091D5060C94B9560895CF93DF9333
:10E7F0002091A2123091A31228173907D1F09093DB
:10E80000A3128093A2122091D606222391F0EC014C
:10E810006FE576E18091D4069091D5060E94485527
:10E82000BE018091D4069091D506DF91CF910C94D2
:10E830008445DF91CF910895CF93DF932091A0126B
:10E840003091A11228173907D1F09093A11280932B
:10E85000A0122091D606222391F0EC0165E476E126
:10E860008091D4069091D5060E944855BE018091B2
:10E87000D4069091D506DF91CF910C948445DF9119
:10E88000CF91089520919712222339F0BC018091F5
:10E890008112909182120C947D800895209194129F
:10E8A000222339F0BC0180917F12909180120C9448
:10E8B0007D80089520919112222339F0BC0180912E
:10E8C0007D1290917E120C947D80089520918E127D
:10E8D000222339F0BC0180917B1290917C120C9420
:10E8E0007D80089520918B12222339F0BC01809104
:10E8F000791290917A120C947D800895209188125B
:10E90000222339F0BC0180917712909178120C94F7
:10E910007D80089520918512222339F0BC018091D9
:10E920007512909176120C947D800895CF92DF92AB
:10E93000EF92FF9220910002213019F420916B0F89
:10E9400004C02230C9F52091710F2223A9F19C0146
:10E95000211584E0380710F02FEF33E0ADE0B0E090
:10E960000E94B7B82FEF33E040E050E00E9469B852
:10E9700069017A018FEFC81AD80AE80AF80A80916B
:10E980009C138C15C9F0C0929C138091D6068823E5
:10E9900099F06EE276E18091D4069091D5060E94BE
:10E9A00048556C2D8091D4069091D506FF90EF903C
:10E9B000DF90CF900C942848FF90EF90DF90CF909D
:10E9C0000895CF92DF92EF92FF92209100022130C2
:10E9D00019F42091680F04C02230C9F520916E0F00
:10E9E0002223A9F19C01211584E0380710F02FEFB4
:10E9F00033E0ADE0B0E00E94B7B82FEF33E040E085
:10EA000050E00E9469B869017A018FEFC81AD80AEC
:10EA1000E80AF80A80919A138C15C9F0C0929A13EB
:10EA20008091D606882399F067E176E18091D4063B
:10EA30009091D5060E9448556C2D8091D4069091F6
:10EA4000D506FF90EF90DF90CF900C942848FF9070
:10EA5000EF90DF90CF90089581E08093CD060E94E3
:10EA600015678091D606882341F06DEF75E180919E
:10EA7000D4069091D5060C94B956089583E08093FE
:10EA8000CD060E942B668091D606882341F06AE06D
:10EA900076E18091D4069091D5060C94B9560895EC
:10EAA00082E08093CD060E942B668091D606882353
:10EAB00041F060EF75E18091D4069091D5060C94F9
:10EAC000B95608950C9473968091010281110C94AB
:10EAD00057960C9473960C94579684E60C941A6986
:10EAE00089E10C941A6982E30C941A698BE40C9402
:10EAF0001A69682F8091D4069091D5060E943F48EC
:10EB00006CE876E18091D4069091D5060C94485536
:10EB10002091D4063091D506882319F066EB77E072
:10EB200002C06AEB77E0C9010C944855F1DF80918F
:10EB3000D4069091D5060C94A6562091D406309117
:10EB4000D506882319F061E876E102C066E876E12F
:10EB5000C9010E9448558091D4069091D5060C9425
:10EB6000A6566FE776E18091D4069091D5060C9475
:10EB700048556BE776E18091D4069091D5060C94C8
:10EB80004855CF93CDE269E776E18091D406909124
:10EB9000D5060E944855C150B1F78091D406909196
:10EBA000D5060E94A6568091D4069091D506DC0128
:10EBB000ED91FC910680F781E02DCF9119940F9390
:10EBC0001F93CF93DF938C01FC01178A168AEC0107
:10EBD000699640E068E0CE010E94EB5C4FE766E09A
:10EBE000CE010E94EB5C40E06CE0CE010E94EB5C49
:10EBF0004FE767E0CE010E94EB5C0E945689F80166
:10EC0000648F758F868F978FDF91CF911F910F91B2
:10EC10000895EF92FF920F931F93CF93DF938C0190
:10EC2000FC01778B668B0E94B94EEC01F801828162
:10EC300093818830910531F57801F9E1EF0EF11CEF
:10EC4000D7FF06C06AE0C1388FEFD80754F001C083
:10EC500068E02C2F9D2FC038D1052CF02FE790E0D5
:10EC600002C021E89FEF422F592F57FF03C0519553
:10EC700041955109C7010E94EB5CCD2B69F54FE727
:10EC800066E027C0099741F57801E9E1EE0EF11C35
:10EC9000D7FF06C06EE0C138FFEFDF0754F001C0B8
:10ECA0006CE02C2F9D2FC038D1052CF02FE790E081
:10ECB00002C021E89FEF422F592F57FF03C0519503
:10ECC00041955109C7010E94EB5CCD2B29F44FE718
:10ECD00067E0C7010E94EB5C0E945689F801648FCF
:10ECE000758F868F978FDF91CF911F910F91FF9036
:10ECF000EF900895CF93DF93EC018091A5128111DD
:10ED000009C06A8D7B8DCE0149960E94B94881E089
:10ED10008093A51221E83FEF3B872A878FE790E099
:10ED20009D878C871F861E86398B288B9B8B8A8BB1
:10ED30001D8A1C8ADF91CF9108950F931F93CF9363
:10ED4000DF93EC011F8A1E8A8C01075E1F4F40E093
:10ED500060E0C8010E94C58340E064E0C8010E94F1
:10ED6000C5830E9456896C8F7D8F8E8F9F8FDF9118
:10ED7000CF911F910F910895CF93DF93EC017F8B7B
:10ED80006E8B0E94B94E9C018A819B8188309105CF
:10ED9000C1F437FF06C061E021388FEF38074CF02F
:10EDA00001C060E0A901203831052CF04FE750E0A8
:10EDB00002C041E85FEF57FF1FC0519541955109CF
:10EDC0001BC00997E9F4922F832F2038310514F0E6
:10EDD0009FE780E0492F582F41388FEF580714F4F0
:10EDE00041E85FEF57FF03C0519541955109632FEB
:10EDF000661F6627661F6C5FCE0149960E94C58319
:10EE00000E9456896C8F7D8F8E8F9F8FDF91CF915F
:10EE100008950F931F93CF93DF93EC010E945689BF
:10EE20000C8D1D8D2E8D3F8DDC01CB01801B910B38
:10EE3000A20BB30B853F9140A105B10540F06E894F
:10EE40007F89CE01DF91CF911F910F9195CFDF91F7
:10EE5000CF911F910F9108950F931F93CF93DF933D
:10EE6000EC018091A412811112C00A8D1B8D6AEAF7
:10EE700070E0C8010E947680D801ED91FC91068077
:10EE8000F781E02DC801199581E08093A4124AE032
:10EE90006EE0CE0149960E94C58321E83FEF3B8793
:10EEA0002A878FE790E09D878C871F861E86398B87
:10EEB000288B9B8B8A8B1D8A1C8ADF91CF911F9197
:10EEC0000F9108950F931F93CF93DF93EC011F8A47
:10EED0001E8A8C01075E1F4F40E060E0C8010E945F
:10EEE000898340E064E0C8010E9489830E945689BA
:10EEF0006C8F7D8F8E8F9F8FDF91CF911F910F91A0
:10EF00000895CF93DF93EC017F8B6E8B0E94B94EF7
:10EF10009C018A819B8188309105C1F437FF06C02E
:10EF200061E021388FEF38074CF001C060E0A901A3
:10EF3000203831052CF04FE750E002C041E85FEF88
:10EF400057FF1FC05195419551091BC00997E9F41E
:10EF5000922F832F2038310514F09FE780E0492F4E
:10EF6000582F41388FEF580714F441E85FEF57FFEF
:10EF700003C0519541955109632F661F6627661F8F
:10EF80006C5FCE0149960E9489830E9456896C8FDE
:10EF90007D8F8E8F9F8FDF91CF9108950F931F9359
:10EFA000CF93DF93EC010E9456890C8D1D8D2E8D21
:10EFB0003F8DDC01CB01801B910BA20BB30B853F76
:10EFC0009140A105B10540F06E897F89CE01DF91A6
:10EFD000CF911F910F9195CFDF91CF911F910F91FD
:10EFE00008950F931F93CF93DF93EC01E8A1F9A14C
:10EFF00080819181A281B3818E01075E1F4F8115AF
:10F000009649A105B10509F450C040E056E960E019
:10F0100070E08FEB97E058DA64E170E080E090E018
:10F020000E941E89E8A1F9A180819181A281B3810A
:10F0300081152BE49207A105B105E9F068F480364B
:10F0400029E09207A105B105A1F080389542A105FC
:10F05000B105C1F442E012C0811521EE9207A1056D
:10F06000B10559F08115924CA140B10559F445E024
:10F0700005C041E003C043E001C046E06FE0C801C5
:10F080000E9489838FEB97E00E945D53E8A1F9A16C
:10F0900040815181628173818FEB97E015DA64E1E1
:10F0A00070E080E090E00E941E894AE06EE0C801B6
:10F0B0000E94898341E067E1C8010E9489834AA1D7
:10F0C00068E1C8010E9489834BA18FEF840F8E31C4
:10F0D00008F04CE066E1C8010E94898342E863E0E1
:10F0E000C8010E94898321E83FEF3B872A878FE789
:10F0F00090E09D878C871F861E86398B288B9B8B83
:10F100008A8B1D8A1C8ADF91CF911F910F910895E0
:10F110000C94B3650C94F3650C94D3650C940F6652
:10F120000C94BF8C0C94FA8C8091A912882319F04E
:10F130000E94BF8C02C00E94FA8C9091A91281E0BB
:10F1400089278093A912089580910002813011F4DB
:10F1500082E001C081E00C94BD6982E00C94BD693D
:10F1600081E00C94BD690C94AD0D8091D606882386
:10F1700041F06BED77E18091D4069091D5060C9427
:10F18000B95608958091D606882341F06BEC77E15B
:10F190008091D4069091D5060C94B956089580912B
:10F1A000D0069091D106DC01ED91FC91EC5BFF4F14
:10F1B0000190F081E02D19958091D606882341F0C9
:10F1C0006AE577E18091D4069091D5060C94B95602
:10F1D0000895CF93DF93CDB7DEB765970FB6F89458
:10F1E000DEBF0FBECDBF8091C30E9091C40E2091A3
:10F1F000C10E3091C20E3A8329839C838B8381E0B8
:10F200008D8B82E08F938DB79EB745970FB6F8949C
:10F210009EBF0FBE8DBFADB7BEB7119685E1FE0193
:10F22000319601900D928A95E1F78AE29BE00E9467
:10F23000DF3C0FB6F894DEBF0FBECDBF8091D6067F
:10F24000882381F062E877E18091D4069091D50619
:10F2500065960FB6F894DEBF0FBECDBFDF91CF919C
:10F260000C94B95665960FB6F894DEBF0FBECDBFAD
:10F27000DF91CF910895CF93DF93CDB7DEB7659738
:10F280000FB6F894DEBF0FBECDBF8091C30E909134
:10F29000C40E2091C10E3091C20E3A8329839C8303
:10F2A0008B8381E08D8B82E08F938DB79EB74597DE
:10F2B0000FB6F8949EBF0FBE8DBFADB7BEB7119607
:10F2C00085E1FE01319601900D928A95E1F78BE57B
:10F2D0009BE00E94DF3C0FB6F894DEBF0FBECDBFAF
:10F2E0008091D606882381F060EB77E18091D40687
:10F2F0009091D50665960FB6F894DEBF0FBECDBFD0
:10F30000DF91CF910C94B95665960FB6F894DEBF95
:10F310000FBECDBFDF91CF9108950E94BF8C409169
:10F32000E40F5091E50F60E070E02AEF3CE88DE8D3
:10F330009BE00E94B6439093BD138093BC138091D1
:10F34000D606882341F06DE077E18091D406909154
:10F35000D5060C94B95608950E94FA8C4091E40F9A
:10F360005091E50F60E070E02FEB3CE88DE89BE00A
:10F370000E94B6439093BD138093BC138091D60630
:10F38000882341F06AEF76E18091D4069091D5060A
:10F390000C94B956089580916F06882339F08BE557
:10F3A0009BE00E94753E23EF35E606C08BE59BE0AF
:10F3B0000E94239823EB35E64CE251E060E070E0D8
:10F3C0008DE89BE00E94B6438091D606882341F0E9
:10F3D0006DE977E18091D4069091D5060C94B956E9
:10F3E000089580916906882339F08AE29BE00E94A3
:10F3F000753E2FE036E606C08AE29BE00E94239825
:10F4000023ED35E64CE251E060E070E08DE89BE0F2
:10F410000E94B6438091D606882341F06FE677E1DB
:10F420008091D4069091D5060C94B95608958BE539
:10F430009BE00E940F9881110C94B3650C94F365C6
:10F440008AE29BE00E940F9881110C94D3650C9482
:10F450000F6669E081E00C94B29168E081E00C9461
:10F46000B29167E081E00C94B29161E081E00C948C
:10F47000B29169E080E00C94B29168E080E00C9475
:10F48000B29167E080E00C94B29161E080E00C946E
:10F49000B2918CE00C94FF918BE00C94FF918AE088
:10F4A0000C94FF9189E00C94FF9188E00C94FF91FB
:10F4B00087E00C94FF9186E00C94FF9185E00C941A
:10F4C000FF9184E00C94FF9183E00C94FF9182E023
:10F4D0000C94FF9181E00C94FF918CE00C942692A7
:10F4E0008BE00C9426928AE00C94269289E00C948E
:10F4F000269288E00C94269287E00C94269286E06F
:10F500000C94269285E00C94269284E00C9426922A
:10F5100083E00C94269282E00C94269281E00C9475
:10F5200026928CE00C944D928BE00C944D928AE0E4
:10F530000C944D9289E00C944D9288E00C944D927D
:10F5400087E00C944D9286E00C944D9285E00C94EB
:10F550004D9284E00C944D9283E00C944D9282E0A5
:10F560000C944D9281E00C944D920C946A920C9400
:10F570007692CF93DF938091BB13882321F1109271
:10F58000BB1360E088E00E94C058C091BC13D091CA
:10F59000BD13BE018DE89BE00E944F43882329F0F4
:10F5A000BE018DE89BE00E9467438091D6068823C8
:10F5B00071F061E477E18091D4069091D506DF91F6
:10F5C000CF910C94B956DF91CF910C944E98DF9166
:10F5D000CF9108958091BB13811102C00C944E9875
:10F5E0000895CF93DF938091BE13882311F10E9479
:10F5F000BF8C1092BE13C091BC13D091BD13BE013D
:10F600008DE89BE00E944F43882329F0BE018DE8DE
:10F610009BE00E9467438091D606882371F068E2E0
:10F6200077E18091D4069091D506DF91CF910C942B
:10F63000B956DF91CF910C940F8DDF91CF91089542
:10F640000C940F8D8091AA12882319F00E94BF8C10
:10F6500002C00E94328E9091AA1281E08927809385
:10F66000AA1208950C94328E0C94458E0C945C8EE4
:10F670008091A812882319F00E94458E02C00E9432
:10F680005C8E9091A81281E089278093A81208953A
:10F690000C94868E0E94868E8091D0069091D10621
:10F6A000DC01ED91FC9104A0F5A1E02D19940C94DE
:10F6B000C38E8091A712882319F00E94868E02C003
:10F6C0000E94C38E9091A71281E089278093A71290
:10F6D00008950C94DF8E0C94FB8E8091A6128823E3
:10F6E00019F00E94DF8E02C00E94FB8E9091A6123C
:10F6F00081E089278093A61208950E944C8B809107
:10F70000D6068823D1F02091BD0F8091D406909128
:10F71000D506211107C02091C00F211103C064EA52
:10F7200076E109C02091010B222319F063EE76E106
:10F7300002C06FEC76E10C94B95608958091010BEC
:10F7400081110C94448B0C944C8B0E94448B8091BF
:10F75000D606882341F06EEE76E18091D406909132
:10F76000D5060C94B95608950C941C9680915612A7
:10F7700081110C9406960C941C960C9406960E948B
:10F780004B8D8091D0069091D106DC01ED91FC91DA
:10F7900002A0F3A1E02D199408950895FC0182813F
:10F7A00093818830910529F410922B0110922A013F
:10F7B0000895099721F410922901109228010895C3
:10F7C000FC01178A168A6CED75E0828152C6CF93D0
:10F7D000DF93EC011F8A1E8A8A81C5D58B8D882311
:10F7E00029F08A8136D69A8F898F1B8EDF91CF912F
:10F7F0000895DF92EF92FF920F931F93CF93DF93C1
:10F80000EC018A81893008F495D5DD8C6B8D7C8D77
:10F81000098D1A8DEA80FB8089E08E1508F466C098
:10F820000F30110538F001369DE6190728F000E683
:10F830001DE602C00FE010E06F30710538F0613650
:10F840008DE6780728F060E67DE602C06FE070E0A4
:10F8500080E090E00E9424B720E030E04AE754E4E2
:10F860000E942BB920E030E04CE852E40E9485B7BA
:10F870009B01AC0160E070E08AEF94E40E942BB938
:10F880000E9493B9FF2425E12E9DF0012F9DF00DDC
:10F890001124E85EFE4EDD2071F023813481AB013E
:10F8A00077FF04C044275527461B570B8827992705
:10F8B000841B950B0AC025813681AB0177FF04C0FC
:10F8C00044275527461B570BCA014FB7F89455E1FB
:10F8D0005E9DF0015F9DF00D1124E85EFE4E108BE1
:10F8E0000787328B218B948B838B4FBF9D8D6B8DC4
:10F8F0007C8D8A819923E9F08A3058F495E1899FBB
:10F90000F0011124E85EFE4E0581168116950795DB
:10F9100002C00EEE12E041E053D561E070E080E0FD
:10F9200090E00E941E898A8194D508171907A8F3D0
:10F930001CC08A3058F495E1899FF0011124E85EDB
:10F94000FE4E038114811695079502C00AEC18E05B
:10F9500040E036D561E070E080E090E00E941E89D2
:10F960008A8177D580179107A8F38A81FCD4B801E2
:10F970008A81DF91CF911F910F91FF90EF90DF90DF
:10F9800078C5CF93DF93EC018A81893008F4D2D413
:10F9900048EE53E05B874A8720ED37E03D872C87B0
:10F9A0008CED95E09F878E87598B488B3B8B2A8BFC
:10F9B0009D8B8C8BDF91CF910895CF93DF93EC01DA
:10F9C0007F8B6E8B888599856817790759F48A81B2
:10F9D000CAD48B8D882321F18A813BD59A8F898F58
:10F9E0001B8E1EC0CE010E94B94EEA81EA30B0F4EF
:10F9F0009C01C39714F022E330E02E3C8FEF3807D0
:10FA000014F42EEC3FEF8FB7F89495E1E99FF001E5
:10FA10001124E85EFE4E318720878FBF81E08B8FF7
:10FA2000DF91CF910895CF93DF93EC018BA19CA13F
:10FA3000892B11F01CA21BA29B0177FF03C03195FB
:10FA400021953109B901CE010E94B94E90932D0143
:10FA500080932C019F8B8E8B0E9456896F8F78A389
:10FA600089A39AA3DF91CF9108950F931F93CF930A
:10FA7000DF938C01FC01778B668B0E94B94EEC0101
:10FA8000F8018281938188309105D1F4D7FF06C0B7
:10FA900060E08AE00E94C05861E005C061E08AE051
:10FAA0000E94C05860E086E00E94C058D7FF03C0A3
:10FAB000D195C195D109D0932B01C0932A011BC0C8
:10FAC0000997C9F4D7FF06C060E08DE00E94C058D6
:10FAD00061E005C061E08DE00E94C05860E08BE00D
:10FAE0000E94C058D7FF03C0D195C195D109D093CA
:10FAF0002901C0932801DF91CF911F910F910895A3
:10FB0000CF93DF93EC018A81893008F413D42EEC73
:10FB10003FEF3B872A8782E390E09D878C871F8693
:10FB20001E86398B288B9B8B8A8B1D8A1C8A6EEED6
:10FB300072E08A818AD46AEC78E08A8182D48CED82
:10FB400095E09A8F898F1B8EDF91CF910895CF9387
:10FB5000DF93EC018BA19CA1892B11F01CA21BA2AD
:10FB6000CE010E94567210922D0110922C011F8A14
:10FB70001E8A0E9456896F8F78A389A39AA3DF916A
:10FB8000CF9108950F931F93CF93DF93FC0123A18F
:10FB900034A1232B91F1EC010E9456890F8D18A1FD
:10FBA00029A13AA1DC01CB01801B910BA20BB30B65
:10FBB0004097A105B10508F18BA19CA10197E9F43B
:10FBC0006E897F89615071097F8B6E8BCE0116160D
:10FBD00017062CF0DF91CF911F910F91B8CF0E94A3
:10FBE000B94E90932D0180932C019F8B8E8B0E9498
:10FBF00056896F8F78A389A39AA3DF91CF911F9124
:10FC00000F910895CF93DF93EC018D8D9E8D1B8610
:10FC10001A869D878C871F861E86198A188A9B8B59
:10FC20008A8B1D8A1C8A61E08CE20E94EF588A81CF
:10FC30009B81089721F410922D0110922C011CA297
:10FC40001BA2DF91CF910895CF93DF93EC0121E0C8
:10FC50003FEF3B872A878FEF90E09D878C871F8639
:10FC60001E86398B288B9B8B8A8B1D8A1C8A61E0B0
:10FC70008AE00E94EF5861E086E00E94EF5861E060
:10FC80008DE20E94EF5861E08DE00E94EF5861E044
:10FC90008BE00E94EF5861E08EE20E94EF588A816B
:10FCA0009B818830910529F410922B0110922A0132
:10FCB00006C0099721F41092290110922801DF91C2
:10FCC000CF9108950F931F93CF93DF93EC010E9480
:10FCD00056890C8D1D8D2E8D3F8DDC01CB01801B37
:10FCE000910BA20BB30B853F9140A105B10548F0E4
:10FCF0006E897F89CE01DF91CF911F910F910C9476
:10FD00000976DF91CF911F910F9108956F927F92A5
:10FD10008F929F92AF92BF92CF92DF92EF92FF921B
:10FD20000F931F93CF93DF938091B9139091BA13E0
:10FD3000DC01ED91FC910084F185E02D1995B12C49
:10FD4000181619060CF0D1C0AA24A3948091B913F7
:10FD50009091BA13DC01ED91FC910084F185E02DC6
:10FD60001995892B09F4C1C0C091051381E08C0F4E
:10FD7000809305138091B9139091BA13DC01ED9132
:10FD8000FC910284F385E02D1995EC2FF0E0EB5304
:10FD9000FD4E80838A30D1F6E0900513F12C10924D
:10FDA000D90D1092D80D1092D40D1092D50D10923D
:10FDB000D60D1092D70D1092D30D1092D20D109235
:10FDC000D10D85ECC82E82E1D82E00E010E0D0E005
:10FDD000C0E00E151F050CF06CC0F60191916F018B
:10FDE0009D3009F463C09C3789F19A3009F052C004
:10FDF000D33009F059C0CC2309F456C06C2E712CB5
:10FE0000C30101970E94154C7093D90D6093D80DD2
:10FE10000E9456896093DB117093DC118093DD1191
:10FE20009093DE118091AB12882309F45BC080901F
:10FE3000D80D9090D90DB8016619770985EC92E13B
:10FE40000E94ED608816990679F54CC08C2F90E0E1
:10FE5000FC01EB5EF14F1082D13099F068F0D230A6
:10FE6000B1F40E94154C6093D40D7093D50D80931E
:10FE7000D60D9093D70D0BC00E94154C6093D10DF9
:10FE800006C00E94154C7093D30D6093D20DDF5FB6
:10FE9000C0E00CC00F3311053CF4EC2FF0E0EB5E3A
:10FEA000F14F9083CF5F02C01092C4120F5F1F4FBB
:10FEB00090CF8091C41281110EC08091CE0D90918F
:10FEC000CF0D01969093CF0D8093CE0D60E087E823
:10FED0000E94909702C0BB24B3941092C512109256
:10FEE000051334CFA092C412E1CF8B2DDF91CF91B7
:10FEF0001F910F91FF90EF90DF90CF90BF90AF9048
:10FF00009F908F907F906F900895CF931092D00D17
:10FF10001092CD0D1092CF0D1092CE0D61E089E3BD
:10FF20000E94C0580E9490608091B9139091BA13BA
:10FF3000DC01ED91FC910084F185E02D1995892B70
:10FF400061F08091B9139091BA13DC01ED91FC91AD
:10FF50000284F385E02D1995E7CF0E940C988091DB
:10FF6000B9139091BA13DC01ED91FC910680F781F1
:10FF7000E02D19951092DA110E9456896093DB11D9
:10FF80007093DC118093DD119093DE11C1E0BEDE31
:10FF900081110E94FA300E94D0604ED58091CE0D22
:10FFA0009091CF0D0A9724F48091DA11882331F0D3
:10FFB00060E08AE80E949097C093D00D8091D00DA8
:10FFC000882329F38091CD0D882341F047ED51E03E
:10FFD00060E070E080E29EE00E9439B860E089E372
:10FFE0000E94C05860E08AE3CF910C94C058EF9211
:10FFF000FF920F931F93CF93DF9300D000D0CDB724
:020000021000EC
:10000000DEB76DE276E0CE0101960E9409550D81C2
:100010001E81F02EEE24E3948091B9139091BA13CF
:10002000DC01ED91FC910084F185E02D1995892B7F
:1000300021F18091B9139091BA13DC01ED91FC91FB
:100040000284F385E02D19958F3439F4E092C312C0
:100050008093B812E092B712DFCF9091C312992328
:10006000D9F2E091B71291E09E0F9093B712F0E0B1
:10007000E854FD4E80839F1578F28091B7128F155A
:1000800010F4F12C21C04BE050E06CEA72E1CE019B
:1000900001960E94754BA8EBB2E1EDE2F6E0FF2479
:1000A000F3941127CF018D5296408017910734F4B5
:1000B0009D9181919817B1F3F12CF4CF1092B81261
:1000C0001092C3121092B712CE0101960E94D95419
:1000D0008F2D26960FB6F894DEBF0FBECDBFDF91F1
:1000E000CF911F910F91FF90EF900895DC01ED915A
:1000F000FC910190F081E02D1994CF93DF93EC01F6
:100100007F8B6E8B0E94B94EBC018A81DF91CF91AB
:10011000B0C1482F50E095E1899FF0011124E85EBD
:10012000FE4E2181328180859185280F391F838180
:1001300094818217930728F08581968128173907C3
:10014000E8F485E1849FF001859FF00D1124E85EBD
:10015000FE4E858196812817390728F5258136813D
:1001600085E1849FF001859FF00D1124E85EFE4E2D
:100170008285823019F411861086128685E1849F6B
:10018000F001859FF00D1124E85EFE4E328321833D
:100190008091840090918500280F391F3093890049
:1001A0002093880008958381948182179307C0F675
:1001B00023813481D5CF8091100B811157C0E091FC
:1001C000F810F091F910858196819093F510809345
:1001D000F4101092F7101092F610E0910211F091C5
:1001E0000311858196819093FF108093FE101092E9
:1001F000011110920011E0910C11F0910D11858107
:100200009681909309118093081110920B1110920E
:100210000A11E0911611F091171185819681909342
:10022000131180931211109215111092141182E182
:1002300090E09093EC108093EB1081E08093F110AC
:100240008093FB108093051180930F118093ED1024
:1002500080E090E021E0FC01E956FF4E2183079603
:1002600084359105C1F781E08093100B08951092B9
:10027000111108951092071108956E3E22E0720741
:1002800038F06B3C98E0790728F06AEC78E002C01F
:100290006EEE72E0660F771F9FB7F89425E1829F9C
:1002A000F0011124E85EFE4E748363839FBF0895BE
:1002B0006E3E22E0720738F06B3C98E0790728F038
:1002C0006AEC78E002C06EEE72E0660F771F9FB7AF
:1002D000F89425E1829FF0011124E85EFE4E7683BA
:1002E00065839FBF0895660F771F282F30E095E143
:1002F000899FF0011124E85EFE4E85819681681782
:10030000790718F46581768107C083819481861707
:10031000970710F4638174818FB7F89495E1929FE9
:10032000F001939FF00D1124E85EFE4E728361830D
:100330008FBF0895982F8FB7F89425E1929FF00111
:100340001124E85EFE4E21E027838FBF41B121E0FA
:1003500030E0B90102C0660F771F9A95E2F7CB0132
:10036000842B81B908958A3058F49FB7F89425E119
:10037000829FF0011124E85EFE4E118610869FBF19
:1003800008951F93CF93DF9325E1829FC00111242D
:10039000EC01C85EDE4E8A8581110EC01FB7F8944D
:1003A00081E08A8789899A899A8389837FD76B8735
:1003B0007C878D879E871FBFDF91CF911F91089506
:1003C000CF93DF938A30D0F56233710538F0613610
:1003D0009DE6790728F060E67DE602C062E370E002
:1003E000D42FC82F80E090E00E9424B720E030E0B6
:1003F0004AE754E40E942BB920E030E04CE852E494
:100400000E9485B79B01AC0160E070E08AEF94E444
:100410000E942BB90E9493B99B01DD2321F0222772
:100420003327261B370B8FB7F89495E1C99FF0014E
:100430001124E85EFE4E318720878FBFDF91CF9178
:1004400008958A3008F419CF08958A3008F430CF1F
:1004500008958A3058F495E1899FF0011124E85EEF
:10046000FE4E8181928196958795089580E090E077
:1004700008958A3008F437CF08951F920F920FB66F
:100480000F9211240BB60F920F931F932F933F934C
:100490004F935F936F937F938F939F93AF93BF938C
:1004A000CF93EF93FF9380915613893048F01092C9
:1004B00056138091C711882399F08091C0110DC007
:1004C000E0915613E15025E1E29FF0011124E85E2E
:1004D000FE4E8781882321F0808192B1892782B9DD
:1004E000E091561385E1E89FF0011124E85EFE4E8D
:1004F0008781882321F0808192B1892B82B9E09194
:100500005613C5E1CE9FF0011124E85EFE4E8085B2
:100510009185892B09F04CC0E0915613CE9FF001D4
:100520001124E85EFE4E8285813009F05FC0BED6A0
:10053000E0915613CE9FF0011124E85EFE4E038534
:10054000148525853685E0915613CE9FF001112440
:10055000E85EFE4E0784F089E02DAB01BC01401B34
:10056000510B620B730BCF01A0E0B0E0841795072D
:10057000A607B707D8F5E0915613A0915613CA9F66
:10058000D0011124A85EBE4E53968D919C91549734
:10059000CE9FF0011124E85EFE4E91878087E091A6
:1005A0005613CE9FF0011124E85EFE4E82E0828752
:1005B00080915613AEDD809156138F5F8093561352
:1005C000FF91EF91CF91BF91AF919F918F917F91CB
:1005D0006F915F914F913F912F911F910F910F90CC
:1005E0000BBE0F900FBE0F901F901895E091561301
:1005F000809184009091850025E1E29FF001112413
:10060000E85EFE4E21813281820F931F9093890014
:1006100080938800D0CF1F93CF93DF9380915513A1
:10062000811173C0109256139FB7F89485E128EB9F
:100630003BE04CED55E064E971E1A1E0B0E0E09110
:100640005613E93008F052C0E09156138E9FF00126
:100650001124E85EFE4E32832183E09156138E9F73
:10066000F0011124E85EFE4E56834583E091561357
:100670008E9FF0011124E85EFE4E74836383E09147
:100680005613F0915613ED0101C0CC0FFA95EAF71D
:100690008E9FF0011124E85EFE4EC083E091561358
:1006A0008E9FF0011124E85EFE4E1782E0915613F2
:1006B0008E9FF0011124E85EFE4E11861086E091B7
:1006C00056138E9FF0011124E85EFE4E1286E091D3
:1006D00056138E9FF0011124E85EFE4E148A138A91
:1006E000E0915613EF5FE0935613A9CF9FBF8FB7EA
:1006F000F89420EA3FE03093C2112093C111109288
:10070000C0118FBF81E080935513DF91CF911F916E
:1007100008950F931F93CF93DF938C01C62FD42F8F
:10072000DC0111968D919C911297DC01ED91FC9169
:100730000190F081E02DD8016C911995F80181812B
:100740009281DC01ED91FC910190F081E02D6C2F04
:100750001995F80181819281DC01ED91FC91019064
:10076000F081E02D6D2F1995F80180816C2F70E0DC
:10077000680F711D6D0F711D6F77772781819281D1
:10078000DF91CF911F910F91B1CC0F931F93CF9316
:10079000DF938C01C62FD42FDC0111968D919C9193
:1007A0001297DC01ED91FC910190F081E02DD801D0
:1007B0006C911995F80181819281DC01ED91FC9198
:1007C0000190F081E02D6C2F1995F80181819281C3
:1007D000DC01ED91FC910190F081E02D6D2F1995D8
:1007E000F80180816C2F70E0680F711D6D0F711D15
:1007F0006F77772781819281DF91CF911F910F9140
:1008000075CC4F925F926F927F92AF92BF92CF92D0
:10081000DF92EF92FF921F93CF93DF93DD24D39467
:1008200045E0C42EC2E0D0E053E0E52EF12CAA242E
:10083000A394B12C8091391390913A13DC01ED917E
:10084000FC910084F185E02D1995892B09F4D1C024
:10085000109130018091391390913A13DC01ED91A0
:10086000FC910284F385E02D199596B3B39A2091FB
:100870008400309185002059384E30938D002093AC
:100880008C00212F2C7119F0109254132AC093FB65
:10089000992790F9E0915413E11116C0992351F270
:1008A0008F3041F6D092541380933B1380913713CD
:1008B00090913813892B09F0BDCFB0923813A092D4
:1008C000371310923613B6CF992381F01092541338
:1008D000109236138091371390913813029709F0D4
:1008E000A9CFF0923813E0923713A4CF91E09E0F76
:1008F00090935413F0E0E55CFC4E8083993109F04D
:1009000099CF811173C08091521382FF05C0F0927C
:100910003813E09237136AC083FDF9CF8091371303
:1009200090913813019761F4809136138F5F809313
:100930003613843058F0D0933813C093371306C061
:10094000D0933813C0933713109236138091351318
:100950008F5F8093351390913413981708F044C03B
:10096000D0923313A3E1B3E1ECE3F3E140E050E0D4
:10097000BA0110E0CF01FC011B3098F401964080D1
:10098000512C612C712C012E04C0440C551C661C8A
:10099000771C0A94D2F74429552966297729185FCC
:1009A000EACF9A013770205E3340C29EC001C39ED9
:1009B000900D112497FD079623E0959587952A952C
:1009C000E1F784529A4F8D939D931B503BE07695AF
:1009D0006795579547953A95D1F783E1A333B807C3
:1009E00049F61092351302C010923313109254132B
:1009F00021CFDF91CF911F91FF90EF90DF90CF90AB
:100A0000BF90AF907F906F905F904F9008958091CE
:100A1000160B833031F480911113909112130C94C2
:100A2000EF3708958091160B823029F480910F13CF
:100A300090911013E6CE0895F5DFE9CF1092F110F2
:100A40001092FB101092051110920F111092ED10E0
:100A500080E090E0FC01E956FF4E11820796843554
:100A60009105C1F708958091160B823039F08330DB
:100A700049F0813049F480910C1301C080E18093EA
:100A8000120B04C08EE0FBCF1092120B8091120B60
:100A900008958091160B823039F0833049F081300F
:100AA00059F480910B130895BDDF8091331308959D
:100AB000AEDF80910A13089580E008958091160BAF
:100AC000823049F0833069F0813089F480910613D7
:100AD000909107130895A6DF8091371390913813F2
:100AE000089595DF8091081390910913089581E08E
:100AF00090E008958F929F92AF92BF92CF92DF9233
:100B0000EF92FF921F93CF93DF93EC0111E08E8160
:100B10009F81892B09F410E02C813D81E885F985BE
:100B2000C580D680878190E0A601480F591F241701
:100B3000350764F180850D2C000CEE08FF08A90133
:100B4000330F660B770B0380F481E02D9A01AB0124
:100B50002C193D094E095F09882329F0A1E0BFEF58
:100B60000E9491B804C0AFEFB0E00E9485B84F0179
:100B7000FF0FAA08BB08A50194012C193D094E09D5
:100B80005F090E9469B83F832E834BC0A601481BB2
:100B9000590B421753070CF43FC080850D2C000CF5
:100BA000EE08FF08A901330F660B770B8180928056
:100BB000092C000CAA08BB089A01AB0128193909B5
:100BC0004A095B09882399F0A1E0BFEF0E9491B820
:100BD000A7019601281939094A095B090E9469B8D9
:100BE000DA01C90181509F4FAF4FBF4F12C0AFEF25
:100BF000B0E00E9485B8A7019601281939094A0971
:100C00005B090E9469B8DA01C9018F5F9109A109E6
:100C1000B1099F838E8305C01F821E82111101C0FE
:100C200019828E819F81009789F08F3F910519F07D
:100C300014F08FEF90E081305FEF950714F481E0BE
:100C40009FEF9F838E8381E018271A83DF91CF91D6
:100C50001F91FF90EF90DF90CF90BF90AF909F904B
:100C60008F90089510924A061092440610923B0607
:100C700010924506109246061092470610924806BA
:100C800081E08093FE0A409150065091510660E049
:100C900070E021E536E880913C0690913D060C9489
:100CA000B6438091010B882361F18091030A811181
:100CB0001CC01092450A1092460A1092470A1092E0
:100CC000480A1092490A10924A0A10924D0A8091DD
:100CD000FC0A9091FD0ADC01ED91FC910190F081FC
:100CE000E02D19951092FE0A089521E536E845E0B9
:100CF00050E060E070E080913C0690913D060C94DD
:100D0000B643089560915F137091601380913C0623
:100D100090913D060E944F43882319F081E0809313
:100D20005E13089560E087E00E94C0581092FF0AA9
:100D3000089561E087E00E94C05881E08093FF0A37
:100D40000895CF93DF9380916C13811110C084EFCD
:100D500091E090936B1380936A138BE290E09093F1
:100D600069138093681381E080936C1320C0809195
:100D70006813909169138532910514F0049709C0A6
:100D80008331910514F0029704C0823091052CF054
:100D900001979093691380936813809168139091E1
:100DA000691397FF04C01092691310926813C091E1
:100DB0006713CC2311F0B6DF01C0BBDF81E08C27C5
:100DC00080936713C0916A13D0916B131C161D0694
:100DD00054F010926C13A6DF21E137E84AEF50E09F
:100DE00060E070E007C021EA36E8AE010D2E000C8D
:100DF000660B770B80913C0690913D060E94B643AE
:100E00009093661380936513809168139091691392
:100E1000C81BD90BD0936B13C0936A13DF91CF918A
:100E200008950F931F93CF93DF938091000B882336
:100E300029F0DF91CF911F910F9183CF009165131E
:100E400010916613C0913C06D0913D06B801CE01C9
:100E50000E944F43882321F0B801CE010E946743CE
:100E6000DF91CF911F910F915DCFCF92DF92EF92E3
:100E7000FF921092000B2091400630914106409164
:100E80004206509143066091450670914606809156
:100E90004706909148060E94C6B86B017C0120E08D
:100EA00030E0A9010E9420B787FD09C0C092450625
:100EB000D0924606E0924706F092480608C010928B
:100EC0004506109246061092470610924806FF907B
:100ED000EF90DF90CF90A5CFEF92FF921F93CF932B
:100EE000DF9300D0CDB7DEB784E689838CE38A83B5
:100EF00088E28B83109161131330E8F4E12EF12C1A
:100F000010FF02C00FDF01C014DFE1E0F0E0EC0FE2
:100F1000FD1FEE0DFF1D408150E060E070E02CE60B
:100F200037E880913C0690913D060E94B6431F5FD2
:100F30001093611303C0F6DE109261130F900F90AF
:100F40000F90DF91CF911F91FF90EF9008958091C6
:100F5000FF0A882311F0E6DE01C0EBDE9091FF0A64
:100F600081E089278093FF0A08950F931F93CF9301
:100F7000DF939091641380914A0691112AC08823CF
:100F800009F44FC00091621310916313C0913C06A5
:100F9000D0913D06B801CE010E944F43882321F035
:100FA000B801CE010E946743C4DE25EB37E842EC6E
:100FB00051E060E070E080913C0690913D060E9417
:100FC000DF43909363138093621381E080936413F3
:100FD00053C0882329F0DF91CF911F910F91B7CF94
:100FE0008091FF0A8823B9F36091621370916313B3
:100FF00080913C0690913D060E94674325EB37E8BF
:1010000044E150E060E070E080913C0690913D0644
:101010000E94DF43909363138093621310926413D2
:101020002BC0C0910D02D0910E022297D0930E02D8
:10103000C0930D021C161D0674F4BE01772787E0CD
:101040000E942B59CC2321F081E08093FF0A14C029
:101050001092FF0A11C06091621370916313809126
:101060003C0690913D060E9467435CDE8FEF90E066
:1010700090930E0280930D02DF91CF911F910F91FB
:1010800008950F931F93CF93DF9300915A131091FC
:101090005B13C0915C13D0915D13C00FD11FD0932F
:1010A0005D13C0935C13BE01772787E00E942B5924
:1010B000CC2321F081E08093FF0A02C01092FF0A46
:1010C00010161106ECF58091581390915913C8171A
:1010D000D9070CF485C080915E13882371F01092BB
:1010E0005913109258138CEF9FEF90935B138093DA
:1010F0005A1381E08093571373C068E770E080E073
:1011000090E00E941D55DC01CB010A96A11DB11D86
:10111000909359138093581368E270E080E090E058
:101120000E941D55DC01CB010A96A11DB11D662749
:101130007727681B790B70935B1360935A1350C029
:10114000012B09F44DC080915813909159138C17BD
:101150009D070CF445C080915713882311F100912D
:101160005F1310916013C0913C06D0913D06B80109
:10117000CE010E944F43882399F1B801CE010E940D
:101180006743D0DD10925D1310925C1310925713D9
:1011900080914A06882321F1DF91CF911F910F9111
:1011A000E4CE69E670E080E090E00E941D55DC012D
:1011B000CB018A569F4FAF4FBF4F909359138093E7
:1011C000581368E270E080E090E00E941D55DC0159
:1011D000CB010A96A11DB11D90935B1380935A1306
:1011E000DF91CF911F910F91089560E088E00C94FA
:1011F000C0583FB7F8948091721390917313A091E7
:101200007413B091751326B5A89B05C02F3F19F034
:101210000196A11DB11D3FBFBA2FA92F982F882776
:10122000820F911DA11DB11DBC01CD0142E0660FD1
:10123000771F881F991F4A95D1F708958F929F9223
:10124000AF92BF92CF92DF92EF92FF926B017C013F
:10125000D0DF4B015C01C114D104E104F104E9F0D9
:10126000C8DFDC01CB0188199909AA09BB09883EAE
:101270009340A105B10578F321E0C21AD108E10835
:10128000F10888EE880E83E0981EA11CB11CC114E1
:10129000D104E104F10421F7DECFFF90EF90DF905D
:1012A000CF90BF90AF909F908F9008952FB7F894F4
:1012B00060916E1370916F13809170139091711300
:1012C0002FBF08951F920F920FB60F9211242F93E4
:1012D0003F938F939F93AF93BF9380916E139091A1
:1012E0006F13A0917013B091711330916D1323E0BF
:1012F000230F2D3720F40196A11DB11D05C026E84E
:10130000230F0296A11DB11D20936D1380936E13C0
:1013100090936F13A0937013B09371138091721315
:1013200090917313A0917413B09175130196A11D40
:10133000B11D8093721390937313A0937413B093A1
:101340007513BF91AF919F918F913F912F910F9006
:101350000FBE0F901F9018950F931F93CF93DF939D
:101360000091651310916613C0913C06D0913D0623
:10137000B801CE010E944F438823A1F0B801CE01ED
:101380000E94674322E836E848EB5BE060E070E0EB
:1013900080913C0690913D060E94B643909366135F
:1013A0008093651360915F137091601380913C0688
:1013B00090913D060E944F4381114BC010925E13E5
:1013C0008FEF90E090935D1380935C13B2DC68E73D
:1013D00070E080E090E00E941D55DC01CB010A9690
:1013E000A11DB11D909359138093581368E270E0CA
:1013F00080E090E00E941D55DC01CB010A96A11D02
:10140000B11D66277727681B790B70935B13609378
:101410005A1321E438E844E150E060E070E0809144
:101420003C0690913D060E94DF43909360138093A9
:101430005F1322E836E848EB5BE060E070E0809103
:101440003C0690913D060E94B643909366138093AC
:101450006513DF91CF911F910F9108958F929F9205
:10146000AF92BF92CF92EF92FF920F931F93CF93C1
:10147000DF9320915B06223008F07AC07B018C015B
:101480008090450690904606A0904706B09048068A
:1014900020E030E0A901C501B4010E9420B7181670
:1014A00054F520E030E0A901C501B4010E94C4B99F
:1014B000181654F420E030E048E452E4C501B401C9
:1014C0000E9420B71816D4F420E030E048E452E43B
:1014D000C501B4010E94C4B918169CF420E030E0A4
:1014E00048EC52E4C501B4010E9420B787FF09C04F
:1014F000CBE4D0E008C0C0E0D0E005C0C2E3D0E05B
:1015000002C0C4E6D0E08FEF8C0D823070F42097DB
:1015100039F06C2FC8010E942C4E6C2FC7010DC0F2
:10152000C8010E945672C70116C08DEF8C0D833022
:10153000F8F4209779F06C2FC801DF91CF911F91BB
:101540000F91FF90EF90CF90BF90AF909F908F90B2
:101550000C942C4EC801DF91CF911F910F91FF90F9
:10156000EF90CF90BF90AF909F908F900C94567259
:10157000DF91CF911F910F91FF90EF90CF90BF908F
:10158000AF909F908F9008958F929F92AF92BF924D
:10159000CF92DF92EF92FF92C0904506D090460620
:1015A000E0904706F090480620E030E0A901C7012E
:1015B000B6010E94C4B920E030E040E05FE387FD5F
:1015C0000BC0C701B6010E94C7B84B015C010E9465
:1015D00093B997FD27C010C0C701B6010E94C6B8D5
:1015E0000E9493B997FD1EC065367105810591056E
:1015F000DCF424E6822F14C0C501B4010E9493B923
:1016000065367105810591057CF420E030E040E00D
:101610005FE3C701B6010E94C7B80E9493B984E690
:10162000861B03C084E601C080E0FF90EF90DF904E
:10163000CF90BF90AF909F908F9008950F931F937E
:10164000CF93DF930091350610913606C0913C068A
:10165000D0913D06B801CE010E944F43882321F06E
:10166000B801CE010E9467438091000B882339F0B6
:101670001092000BDF91CF911F910F91D2CBDF9190
:10168000CF911F910F910895EC981092010B68EC87
:1016900070E082E00C94CF4480915406811105C023
:1016A00080915806811101C0EFCF8091FC0A909182
:1016B000FD0A0E943C5281E08093010B64E670E0D9
:1016C0000C94CF4460E089E30E94C05860E08AE354
:1016D0000E94C05860E085E30E94C05860E085E049
:1016E0000E94C05860E084E00E94C05860E087E03B
:1016F0000E94C05859980895CF93C09112026C2F40
:1017000089E30E94C05881E0C8276C2F8AE30E94B9
:10171000C058C0931202CF910895CF93DF93C09128
:1017200011026C2F89E30E94C058D1E0DC276D2F95
:101730008AE30E94C0586C2F85E30E94C0586D2F29
:1017400085E00E94C0586D2F84E00E94C0586C2F25
:1017500087E00E94C058CC2311F0599801C0599AD3
:101760009091110281E0892780931102DF91CF913E
:101770000895CF93DF9380918B1381110DC0109248
:101780008A131092891381E090E0909388138093DC
:10179000871380938B1336C08091891390918A139D
:1017A000863191057CF18F38910534F4809187134F
:1017B00090918813019609C08D3521E0920754F469
:1017C0008091871390918813029690938813809349
:1017D000871318C0863222E0920734F48091871371
:1017E000909188130496F1CF883E93403CF4809109
:1017F0008713909188138A5B9F4FE7CF10928813CD
:10180000109287138ADFC0918913D0918A13C93E41
:1018100083E0D80754F010928B1354DF21E33CE8A7
:1018200048EE53E060E070E007C029EB3BE8AE0112
:101830000D2E000C660B770B8DE89BE00E94B643E3
:1018400090938613809385138091871390918813CA
:101850008C0F9D1F90938A1380938913DF91CF91F2
:101860000895CF93DF938091D906882319F0DF91F3
:10187000CF917FCFC0918513D0918613BE018DE8A3
:101880009BE00E944F43882329F0BE018DE89BE036
:101890000E946743DF91CF9115CFCF93C091821300
:1018A0006C2F70E088E00E942B5989E180938113AE
:1018B00090911002992311F0CD5F01C0C350C093E5
:1018C000821380918213873970F0992321F08FEF72
:1018D0008093821308C08D3D30F086E98093821397
:1018E00088E780938113809182138F3F19F41092BF
:1018F000100205C08A3118F481E0809310024091F3
:10190000811350E060E070E02DE43CE88DE89BE05E
:101910000E94B6439093BD138093BC13CF9108955A
:10192000CF92DF92EF92FF92CF93DF93EC019C0175
:10193000AFEFB0E00E94B7B8CC24CA9423E0D22E17
:10194000E12CF12CA70196010E9469B8B90188E049
:101950000E942B599E01A4E6B0E00E94B7B8A701EF
:1019600096010E9469B88091EA0F82132093EA0FD2
:10197000DF91CF91FF90EF90DF90CF900895CF93BC
:10198000DF93C091BC13D091BD13BE018DE89BE0E5
:101990000E944F43882329F0BE018DE89BE00E94FE
:1019A000674360E088E00E94C0588091D606882393
:1019B000D1F08091BE13882319F06DE878E10DC055
:1019C0008091BB13882319F064E778E106C0809109
:1019D000BF13811108C065E678E18091D40690912B
:1019E000D5060E94B9561092BE131092BB13DF9118
:1019F000CF91089561E088E00E94C0588091D6069A
:101A0000882361F08091BE13811108C067E578E1F9
:101A10008091D4069091D5060C94B9560895809182
:101A2000BE13811110C0ABDF81E08093BE138091A3
:101A3000D606882341F06CEB78E18091D406909132
:101A4000D5060E94B95680918013882329F060E062
:101A500088E00E94C05801C0CDDF9091801381E0E2
:101A6000892780938013882329F04091E60F5091B5
:101A7000E70F04C04091E80F5091E90F60E070E07B
:101A80002FE03DE88DE89BE00E94B6439093BD13A4
:101A90008093BC130895CF9380917E1381110FC062
:101AA00081E080937E138091D606882341F065E221
:101AB00078E18091D4069091D5060E94B956C091E4
:101AC0007D136C2F85E00E94C0584091EF0F50E0CD
:101AD00060E070E02BE43DE88DE89BE00E94B643B7
:101AE00090937C1380937B1381E06C2F6827609325
:101AF0007D13CF910895CF93DF93C0918313D0913D
:101B00008413BE018DE89BE00E944F43882361F05F
:101B1000BE018DE89BE00E946743109284131092EF
:101B20008313DF91CF91CECDDF91CF910895609156
:101B30008313709184138DE89BE00E944F438111C1
:101B40002EC060E089E30E94C05860E08AE30E94F2
:101B5000C05860E085E30E94C05860E085E00E94C4
:101B6000C05860E084E00E94C05860E087E00E94B6
:101B7000C05859988091EC0F882319F02DE83BE864
:101B800002C02CE73BE842E350E060E070E08DE803
:101B90009BE00E94DF439093841380938313089506
:101BA00060E08AE30C94C05861E08AE30C94C0586A
:101BB0000F931F93CF93DF938C01C1E0D0E00C17FC
:101BC0001D078CF0F1DF64E670E080E090E036DB2A
:101BD000E7DFC017D1072CF46AE570E080E090E001
:101BE0002DDB2196ECCFDF91CF911F910F910895BE
:101BF00083E090E0DDCF82E090E0DACF81E090E01A
:101C0000D7CF60E089E30C94C05861E089E30C947D
